:020000040800F2
:1000000000000120D13F0008972700089927000829
:100010009B2700089D2700089F270008000000007C
:10002000000000000000000000000000A127000800
:10003000A327000800000000A5270008A727000844
:100040002140000821400008A9270008214000089D
:1000500021400008214000082140000821400008FC
:1000600021400008CD270008214000082140000859
:100070002140000821400008B5270008C1270008DA
:1000800021400008214000082140000821400008CC
:100090000000000021400008214000082140000825
:1000A00021400008214000082140000821400008AC
:1000B000214000082140000821400008214000089C
:1000C000214000082140000821400008214000088C
:1000D000214000082140000821400008214000087C
:1000E0002140000821400008D527000821400008D1
:1000F000214000080000000000000000214000082E
:100100002140000821400008E127000821400008A4
:10011000214000082140000821400008214000083B
:10012000214000082140000821400008214000082B
:080130002140000821400008F5
:1001380010B5054C237833B9044B13B10448AFF319
:1001480000800123237010BDBC08002000000000BF
:100158005039010808B5034B1BB103490348AFF3F5
:10016800008008BD00000000C008002050390108C8
:1001780014214160704714207047406A704700009E
:10018800790100087F01000883010008990100082F
:1001980010B5044604F1100000F05CFCC4F8F80047
:1001A8000148C4F87C0110BD88010008F8B5E6B024
:1001B80004460D4616461F460A4906A800F0CAFE20
:1001C80070996F9A05910492009733466E996D9ACB
:1001D800039102922A466C990191214600F060F839
:1001E80067B0F0BD94010008F8B5E6B004460D46C6
:1001F80016461F46094906A800F0ACFE6F996E9A8C
:100208000491039200976D996C9A0291019233467A
:100218002A46214600F087F867B0F0BD940100082F
:1002280038B500281CBF01680029184A23D1184B8B
:100238001C684FF6F0710C404CF24025AC421FBFD1
:100248001B6819404CF27024A14212D1114D296843
:1002580079B911490B68C3F30B03B3F58A6F1FBF54
:100268000968C1F30B0140F28343994204BF01219D
:10027800117028B905E0094B994204BF012111709A
:100288004068BDE8324001F099BE00BFD8080020A0
:1002980000ED00E0002004E00010005C000037489A
:1002A8002DE9F04104460D46216816464A681F4666
:1002B80090478046B8F5403F2ED122680A99936846
:1002C800204698478046B8F5403F25D12368089ACC
:1002D8000799D3F80CC02046E0478046B8F5403F60
:1002E8001AD12368069A39461F692046B8478046BE
:1002F800B8F5403F10D1236829465D69324620464B
:10030800A8478046B8F5403F06D123680B9A09995B
:100318009D692046A847804621680A68204690477C
:100328004046BDE8F0812DE9F04104460D462168BC
:1003380016464A681F4690478046B8F5403F2ED17A
:1003480022680A999368204698478046B8F5403F46
:1003580025D12368089A0799D3F80CC02046E047AE
:100368008046B8F5403F1AD12368069A39461F6976
:100378002046B8478046B8F5403F10D12368294643
:100388005D6932462046A8478046B8F5403F06D109
:1003980023680999DD6900222046A847804621681C
:1003A8000A68204690474046BDE8F0814FF4403047
:1003B80070470000F0B50C4685B0114600281A4673
:1003C8001CBF0568002D0B4B11D082B104B971B95F
:1003D8000D9860B10F9E0E9F0A9B0290049603979A
:1003E8000B980C9E009001962046A8470346184695
:1003F80005B0F0BD020003002DE9F04F0646D0B06D
:100408000868F56DD6F860E0726EB76EF36E00BAE4
:1004180000906C46486800BA60600DF14008886832
:1004280000BAA060C86800BAE060086900BA206134
:10043800486900BA6061886900BAA061C86900BAF1
:10044800E061086A00BA2062486A00BA6062886A95
:1004580000BAA062C86A00BAE062086B00BA2063FA
:10046800486B00BA6063886B00BAA063C86B00BAB7
:10047800E063402058F80C1C58F820CC58F838ACE9
:100488008CEA010158F840CC8AEA01018CEA01099A
:100498004FEAF979401E48F8049BEBD187EA02003D
:1004A80000EA0E00784010EBF5610098DFF824C4EC
:1004B80041186144C81882EABE032B404FEAF06134
:1004C80053405918636859186144CF194FEAB50366
:1004D80083EABE01014081EABE0111EBF765A1681C
:1004E8004D196544A91883EAB0023A404FEAF1650C
:1004F8005A405519E26855194FEAB70282EAB0071F
:1005080065440F4005EBBE0E97EAB00717EBFE6592
:1005180027697D194FEAB10782EA0701654401EAB4
:100528000E01EB18514011EBF36561694D194FEA63
:10053800BE0187EA010E65440EEA030E15EBB00012
:100548008EEA070E0EEBF065D4F818E075446544A2
:10055800AA1881EAB30505404FEAF26E4D40AE4451
:10056800E569AE44E64477444FEAB00080EAB30E4A
:100578000EEA020E8EEAB30E0EEBF765D4F820E011
:1005880075446544691880EAB2053D404FEAF16E4A
:100598004540AE44656AAE44E6440EEBB3034FEA09
:1005A800B70787EAB20E0EEA010E8EEAB20E0EEB1C
:1005B800F365D4F828E075446544281887EAB1053E
:1005C8001D404FEAF06E7D40AE44E56AAE44E64415
:1005D8000EEBB2024FEAB30383EAB10E0EEA000E45
:1005E8008EEAB10E0EEBF265D4F830E0754465443E
:1005F800EF1983EAB00515404FEAF76E5D40AE4447
:10060800656BAE44E6440EEBB1014FEAB20282EAF2
:10061800B00E0EEA070E8EEAB00E0EEBF165D4F8B6
:1006280038E075446544EB1882EAB7050D404FEA97
:10063800F36E5540AE44E56BAE44E6440EEBB000B5
:100648004FEAB10181EAB70E0EEA030E8EEAB70E41
:100658000EEBF065D4F840E07544654481EAB30ECA
:10066800AA180EEA000E4FEAF2658EEA010E7544EA
:10067800DDF844E04FEAB000754480EAB30E654403
:100688000EEA020E15EBB7078EEAB30E0EEBF7650E
:10069800DDF848E04FEAB202754480EA020E65448C
:1006A8000EEA070E69188EEA000E0EEBF165DDF80A
:1006B8004CE07544654405EBB3034FEAB70E1427C5
:1006C8000DF1500CDFF810528EEA010B82EA0B0B89
:1006D8000BEBF36A5CF804BBDA44AA44504483EA9F
:1006E800B10B4FEAF06A8EEA0B0BDA445CF804BBF4
:1006F800DA44AA44524480EAB30B4FEAF26A8BEA1E
:10070800B10BDA445CF804BBDA444FEAB000AA44FF
:1007180080EA020BD6448BEAB30B0BEBFE6A5CF85B
:1007280004BBDA444FEAB202AA4482EA0E0B0AEB8F
:10073800B10180EA0B0B0BEBF16A5CF804BBDA44FD
:100748007F1DAA44282F0AEBB3034FEABE0EBBD382
:100758003C2F61D3502F4DD204EB870CC7F15407BF
:100768005E4CA7FB04A504465D4FA8088EEA010A63
:1007780082EA0A0A5CF804BB0AEBF3655D447D195A
:100788002C1983EAB10A4FEAF4658EEA0A0A55443D
:100798005CF804AB5CF804BB55447D19AA1884EADC
:1007A800B30A4FEAF2658AEAB10A55445D444FEA52
:1007B800B4047D1984EA020AAE448AEAB30A0AEB51
:1007C800FE655CF804AB55444FEAB2027D1982EA33
:1007D8000E0A15EBB10184EA0A0A5CF804BB0AEBBD
:1007E800F1655D447D1915EBB303401E4FEABE0E5B
:1007F800BCD12046F46D1B19F365336EC9183166F8
:10080800716E71447166B36ED218B266F16E40189B
:10081800F06650B0BDE8F08F4EEA010B0EEA010A0F
:100828000BEA020B4BEA0A0A0AEBF36554F827A015
:10083800DFF8B0C0554443EAB10B654403EAB10A96
:100848000BEA0E0B28184BEA0A0A7F1C0AEBF06524
:1008580054F827A0554440EAB30B654400EAB30AAC
:100868000BEAB10BAA184BEA0A0A7F1C0AEBF265DD
:1008780054F827A055444FEAB00040EA020B6544FB
:1008880000EA020A0BEAB30BAE444BEA0A0A7F1CE1
:100898000AEBFE6554F827A055444FEAB20242EA33
:1008A8000E0B654402EA0E0A0BEA000B15EBB101C8
:1008B8004BEA0A0A7F1C0AEBF16554F827A0554455
:1008C8007F1C65443C2F05EBB3034FEABE0EA3D350
:1008D80040E700BF9979825AA1EBD96ECDCCCCCC38
:1008E800D6C162CADCBC1B8F00B581B00168074A5B
:1008F800914200D110B9064801B000BD7C2112F028
:100908008DFF4FF4003001B000BD00BFFC090008A6
:10091800030002002DE9F0410B4A92E8F85188B033
:10092800694681E8F8510268084B9A4200D118B923
:10093800074808B0BDE8F0811422083000F04FFBEA
:1009480008B0BDE8F08100BFDC090008FC09000818
:1009580003000200152904D20268044B9A4200D110
:1009680008B903487047083000F048BBFC09000884
:100978000300020010B481B013460268074CA2427B
:1009880000D118B901B010BC0548704701B000F19A
:10099800240210BC083000F035BB00BFFC09000879
:1009A8000300020010B481B013460268074CA2424B
:1009B80000D118B901B010BC054870470A4601B00B
:1009C80000F1240110BC083000F070BBFC090008DD
:1009D800030002000123456789ABCDEFFEDCBA981E
:1009E80076543210F0E1D2C300000000000000008D
:1009F80000000000F10800081D0900085D09000852
:100A08007D090008AD09000801040008790F0008F5
:100A1800C50F0008810F0008F0B5A3B004460B48C5
:100A280002900D4616461F46094B0822402104A88D
:100A380000F0D1FA28980190009733462A462146BB
:100A480002A800F01BF823B0F0BD00BFFC090008A5
:100A5800100A000810B5040008BF002408D0054893
:100A6800054B20600822402104F1080000F0B3FA89
:100A7800204610BDFC090008100A00082DE9F041C5
:100A880004460E46216817464A681D469047804628
:100A9800B8F5003F19D1226806999368204698470F
:100AA8008046B8F5003F10D123683146DE683A46E3
:100AB8002046B0478046B8F5003F06D12368079A1C
:100AC80029461D692046A847804621680A682046AD
:100AD80090474046BDE8F08110B500F033FA4FF476
:100AE800403400280EBF034C4FF4C07112F096FE3C
:100AF800204610BD0200030010B5044600F022FA9B
:100B080008B9054810BD0021A160D0F87C21116802
:100B180088474FF4403010BD0200030070B504460A
:100B28000D4600F00FFA064E40B1D0F87C0141683E
:100B38008847A84224BF65604FF44036304670BDF0
:100B4800020003002DE9FF4715000C4600D02CB128
:100B5800064600F0F7F95FEA000801D16448C3E0EF
:100B6800D8F8F80001684A689047B0F5003F17D1F7
:100B7800D8F87C118A68404690478146B9F1810FC0
:100B880080F09E80A94508F1FC0A17D2D8F8F80031
:100B98000368D3F80CC02A462146E047B0F5003F69
:100BA80040F08E80D8F8F8000368D3F810C06A4681
:100BB8005146E047B0F5003F76D10AE0002004E056
:100BC800215C0AF800100098401C00900098A84288
:100BD800F6D34FF0000C4749474A484B01AC009800
:100BE800844558D2D3E9007001ADC5E9007010788A
:100BF80000281ABF042086464FF0000E085854F803
:100C08000E5028443E4D05600127D0F800E087606B
:100C1800019D4F681AF80C007D408EEA050585F0A5
:100C2800040E65680F687D4085F0FC05754485F005
:100C3800A30568400AF80C000CF1010CCFE7D3E9D2
:100C4800004501A8C0E9004510782E4D002814BFC2
:100C58004FF0040E4FF0000E01A8744651F80EE054
:100C68000459A6440127CEF80050DEF80040CEF81B
:100C780008704D68019F40687D406C400D68684071
:100C880084F0040480F0FC00041984F057040AF886
:100C98000C400CF1010CCC45D1D3D8F8F800016810
:100CA8004A689047B0F5003F0AD1D8F8F8000368C1
:100CB800D3F80C804A465146C047B0F5003F01D0F2
:100CC800114811E0002006E05AF8201081F06A313E
:100CD8004AF82010401CB0EB990FF5D3B06840F0EB
:100CE8000100B0604FF4403004B0BDE8F08700BFA9
:100CF80002000300E8390108D8080020240F000882
:100D0800ADBE4ED70DBE75A10100030038B50C4627
:100D1800017A1546CA0702D500F014F908B908483F
:100D280032BDD0F8F80003682146DC682A46A0479F
:100D3800B0F5003F01D0034832BD4FF4403032BD1A
:100D480002000300010003002DE9F84191B00546B7
:100D58000E461746402101A812F060FD297AC807FF
:100D680004D5284600F0EEF8040002D1DFF8A4808C
:100D78004BE0D4F8F800DFF8A0800368D3F810C07F
:100D88006A4601A9E047B0F5003F3ED1D4F8F80023
:100D980001684A689047B0F5003F36D1D4F87C1115
:100DA8008A6820469047D4F8F830024618461B68EF
:100DB800D3F80CC004F1FC01E047B0F5003F24D1A2
:100DC800D4F87C0141688847D4F8F83002461846C0
:100DD8001B68D3F80CC001A9E047B0F5003F14D157
:100DE800D4F8F8000268696893689847B0F5003F3E
:100DF8000BD1D4F8F80003681C693A463146A0477D
:100E0800B0F5003F08BF4FF44038404612B0BDE887
:100E1800F08100BF02000300010003002DE9F84142
:100E2800A5B0074688461646402115A812F0F6FCDC
:100E380000220492402105A812F0F0FC387AC1077C
:100E48005ED5384600F07EF8050059D0D5F8F80090
:100E58002D4C0368D3F810C06A4605A9E047B0F5E1
:100E6800003F3CD1D5F8F80001684A689047B0F5D2
:100E7800003F34D1D5F87C118A6828469047D5F8C8
:100E8800F830024618461B68D3F80CC005F1FC017F
:100E9800E047B0F5003F22D1D5F87C01416888478A
:100EA800D5F8F830024618461B68D3F80CC005A9D7
:100EB800E047B0F5003F12D1D5F8F800026879682C
:100EC80093689847B0F5003F09D1D5F8F800036852
:100ED8001D6904AA15A9A847B0F5003F01D020460E
:100EE8000FE00A4B0A490B4A0396029101924046C9
:100EF8001C68049B009415AA796800F0E5F900E0E5
:100F0800054826B0BDE8F08101000300F03901086A
:100F1800936E030026C703000200030004B001011A
:100F280000170145E10A0008010B0008250B00081D
:100F3800B50300084D0B0008150D0008510D0008F9
:100F4800250E00080168024A914218BF0020704728
:100F58002C0F000810B5040008BF002404D0034873
:100F68002060204609688847204610BD2C0F0008DD
:100F780020225C3012F050BCF0B58468A30800222F
:100F880004F0030407E000F15C0555F8226035BA67
:100F980041F82250521C9A42F5D300220BE000F18E
:100FA8005C0502EB830755F82360D500C5F11805E9
:100FB800EE40CE55521CA242F1D3F0BD30B5C46804
:100FC80003690022E31AD5188C5C0544521C082AD0
:100FD8002C77F8D330BD0360C1600261704738B523
:100FE800044615460022626023685A68904700202C
:100FF8006061A061A5604FF4003032BD81604FF49C
:10100800003070472DE9F84304462079D4F80C8065
:10101800450748BF244845D466691D46A8F1010024
:1010280000EAD60306EBC506B6EBC50F666102D229
:10103800A669761CA6611746A66906EB5576A661D1
:101048000E46E918884225D2A8EB03094A463146DC
:10105800F81812F0E1FB2268136839460FE042469F
:10106800384612F0D9FB23681A683946204690475B
:1010780007E0311811F00300F1D122681368204607
:101088009847484600EB0809A9F10101A942F0D3A5
:10109800002300E000202A1A3118F81812F0BCFBCF
:1010A8004FF40030BDE8F283040002002DE9FC4F44
:1010B800024685B0D0681369DFF86CC1DFF86C812F
:1010C800A0EB030A506840F004005060002703A812
:1010D80002900DF10C0ED8E9003403A8544DC0E974
:1010E80000342878534D00280CBF00230423994668
:1010F8005CF803305EF80940234401261D601C6833
:101108009E60DCF80430039DDCF80090DEF8046093
:101118005D406540484C654089EA0606474C664094
:101128007519474C6540D8E9006B03AC0028C4E941
:10113800006B0EBF002404200424029E5CF800000B
:10114800345920183F4C04600126046886600398CF
:10115800029E43406340384C7068634089EA00004F
:10116800364C6040034438484340280018BF0120EB
:101178005B1E9B41042F2CBFC0B2D80F02F1140391
:1011880053F8200007F00303C3F10303DB00D84042
:101198000DF807007F1C082F9DD315460C466A6979
:1011A800AB69E868D20842EA4372401E00EA0207C7
:1011B800002302409B420AD8524508D28020E055BD
:1011C8007F1C574516D2AAEB0701E01910E08020D2
:1011D800E05500E0E355E8687F1C8742FAD32A68A7
:1011E800136828469847BAF1000F03D051462046A5
:1011F80012F014FB2A68069E059F936869462846E4
:1012080098472A68D2F8009021462846C8472B6894
:10121800DA683946284690470EB1A86830604FF41E
:10122800003007B0BDE8F08FE83901085412000813
:10123800D80800205FC5109304850012FC68017A65
:10124800C0F524FF24AF33D426AF698B04B0010165
:1012580000170145F8B501240094002300240DE08F
:10126800009D065D0F5D7E40F643761CF60F86F006
:10127800010635400095641C009DEB189442EFD39D
:101288001846F2BDF8B5002301240094002A11E0A5
:10129800009C85188F1815F8016C17F8015C6E40D2
:1012A800F643761CF60F86F0010634400094009C45
:1012B800E318521EECD11846F2BD00005D1200087A
:1012C8008D120008010000002DE9F84F1D46DDF8D9
:1012D80028900B9F0D9C4FF0FF3300930E469246CB
:1012E800D9F800B0804632465146D847834664B3A1
:1012F800D9F8043032465146404698476FEA0B0207
:10130800521C42EA0B0200996FEAD2735B1C194027
:10131800C2430091521C024300996FEAD2735B1CCE
:101328001940009186F05531484087EA000181F064
:101338005531216080F05531C943491C0843009A52
:101348006FEAD070401C82430092D9F80800012847
:1013580009D17540E943491C0D4300986FEAD572DD
:10136800521C90430AE0F11C85EA9102D243521CB8
:10137800154300986FEAD5735B1C984386F0AA362C
:10138800009086EA0B0686F0AA33F243DB430C98FA
:10139800C2F3C0725B1C42EAD3720099D243521C5A
:1013A80091430091774000998843009987F0AA37C4
:1013B8000F403843BDE8F28F034613F8012B002A8B
:1013C800FBD1181A0138704781F0004102E000BFD4
:1013D80083F0004330B54FEA41044FEA430594EAED
:1013E800050F08BF90EA020F1FBF54EA000C55EA28
:1013F800020C7FEA645C7FEA655C00F0E2804FEAF9
:101408005454D4EB5555B8BF6D420CDD2C4480EADA
:10141800020281EA030382EA000083EA010180EA0A
:10142800020281EA0303362D88BF30BD11F0004F58
:101438004FEA01314FF4801C4CEA113102D040428E
:1014480061EB410113F0004F4FEA03334CEA1333C9
:1014580002D0524263EB430394EA050F00F0A780E1
:10146800A4F10104D5F1200E0DDB02FA0EFC22FADC
:1014780005F2801841F1000103FA0EF2801843FAD0
:1014880005F359410EE0A5F120050EF1200E012AC1
:1014980003FA0EFC28BF4CF0020C43FA05F3C018FF
:1014A80051EBE37101F0004507D54FF0000EDCF178
:1014B800000C7EEB00006EEB0101B1F5801F1BD321
:1014C800B1F5001F0CD349085FEA30004FEA3C0C25
:1014D80004F101044FEA445212F5800F80F09A801B
:1014E800BCF1004F08BF5FEA500C50F1000041EB1F
:1014F800045141EA050130BD5FEA4C0C404141EB23
:101508000101013C28BFB1F5801FE9D291F0000F1D
:1015180004BF01460020B1FA81F308BF2033A3F1CC
:101528000B03B3F120020CDA0C3208DD02F1140CC3
:10153800C2F10C0201FA0CF021FA02F10CE002F1FE
:101548001402D8BFC2F1200C01FA02F120FA0CFCF7
:10155800DCBF41EA0C019040E41AA2BF01EB045140
:10156800294330BD6FEA04041F3C1CDA0C340EDC3E
:1015780004F11404C4F1200220FA04F001FA02F381
:1015880040EA030021FA04F345EA030130BDC4F13F
:101598000C04C4F1200220FA02F001FA04F340EA34
:1015A8000300294630BD21FA04F0294630BD94F0E5
:1015B800000F83F4801306BF81F480110134013DCC
:1015C8004EE77FEA645C18BF7FEA655C29D094EA3D
:1015D800050F08BF90EA020F05D054EA000C04BFBB
:1015E8001946104630BD91EA030F1EBF00210020A6
:1015F80030BD5FEA545C05D14000494128BF41F045
:10160800004130BD14F580043CBF01F5801130BDA8
:1016180001F0004545F0FE4141F470014FF0000033
:1016280030BD7FEA645C1ABF194610467FEA655CE4
:101638001CBF0B46024650EA013406BF52EA033586
:1016480091EA030F41F4002130BD00BF90F0000F74
:1016580004BF0021704730B54FF4806404F13204B0
:101668004FF000054FF0000150E700BF90F0000F69
:1016780004BF0021704730B54FF4806404F1320490
:1016880010F0004548BF40424FF000013EE700BF60
:1016980042004FEAE2014FEA31014FEA02701FBFF0
:1016A80012F07F4393F07F4F81F06051704732F022
:1016B8007F4208BF704793F07F4F04BF41F4002179
:1016C800704730B54FF4607401F0004521F00041D7
:1016D8001CE700BF50EA010208BF704730B54FF061
:1016E80000050AE050EA010208BF704730B511F062
:1016F800004502D5404261EB41014FF4806404F19A
:1017080032045FEA915C3FF4D8AE4FF003025FEA1F
:10171800DC0C18BF03325FEADC0C18BF033202EBA3
:10172800DC02C2F1200300FA03FC20FA02F001FAFD
:1017380003FE40EA0E0021FA02F11444BDE600BFA0
:101748004FF0FF3C06E000BF4FF0010C02E000BF85
:101758004FF0010C4DF804CD4FEA410C7FEA6C5C68
:101768004FEA430C18BF7FEA6C5C1BD001B050EA0B
:10177800410C0CBF52EA430C91EA030F02BF90EAF6
:10178800020F0020704710F1000F91EA030F58BFB5
:10179800994208BF90422CBFD8176FEAE37040F017
:1017A800010070474FEA410C7FEA6C5C02D150EAB5
:1017B800013C07D14FEA430C7FEA6C5CD6D152EA70
:1017C800033CD3D05DF8040B704700BF8446104635
:1017D80062468C461946634600E000BF01B5FFF734
:1017E800B7FF002848BF10F1000F01BD4DF808ED04
:1017F800FFF7F4FF0CBF012000205DF808FB00BFD5
:101808004DF808EDFFF7EAFF34BF012000205DF82E
:1018180008FB00BF4DF808EDFFF7E0FF94BF01207B
:1018280000205DF808FB00BF4DF808EDFFF7CEFF7C
:1018380094BF012000205DF808FB00BF4DF808EDBB
:10184800FFF7C4FF34BF012000205DF808FB00BF8C
:101858004FEA410212F5001215D211D56FF47873D0
:10186800B3EB625212D94FEAC12343F0004343EA73
:10187800505311F0004F23FA02F018BF404270474E
:101888004FF00000704750EA013005D111F00040D8
:1018980008BF6FF0004070474FF00000704700BF6E
:1018A80080F0004002E000BF81F0004142001FBF0D
:1018B8005FEA410392EA030F7FEA226C7FEA236C16
:1018C8006AD04FEA1262D2EB1363C1BFD21841400B
:1018D80048404140B8BF5B42192B88BF704710F0A1
:1018E800004F40F4000020F07F4018BF404211F044
:1018F800004F41F4000121F07F4118BF494292EAAC
:10190800030F3FD0A2F1010241FA03FC10EB0C00D7
:10191800C3F1200301FA03F100F0004302D5494264
:1019280060EB4000B0F5000F13D3B0F1807F06D311
:1019380040084FEA310102F10102FE2A51D2B1F109
:10194800004F40EBC25008BF20F0010040EA0300FE
:101958007047490040EB0000013A28BFB0F5000F7E
:10196800EDD2B0FA80FCACF1080CB2EB0C0200FA34
:101978000CF0AABF00EBC25052421843BCBFD04083
:101988001843704792F0000F81F4000106BF80F4FD
:1019980000000132013BB5E74FEA41037FEA226CC0
:1019A80018BF7FEA236C21D092EA030F04D092F08B
:1019B800000F08BF0846704790EA010F1CBF0020BF
:1019C800704712F07F4F04D1400028BF40F000401C
:1019D800704712F100723CBF00F50000704700F03C
:1019E800004343F0FE4040F4000070477FEA226263
:1019F80016BF08467FEA23630146420206BF5FEA34
:101A0800412390EA010F40F4800070474FF0000333
:101A180004E000BF10F0004348BF40425FEA000CFA
:101A280008BF704743F0964301464FF000001CE0A2
:101A380050EA010208BF70474FF000030AE000BFF8
:101A480050EA010208BF704711F0004302D5404236
:101A580061EB41015FEA010C02BF844601460020A8
:101A680043F0B64308BFA3F18053A3F50003BCFAC3
:101A78008CF2083AA3EBC25310DB01FA02FC634470
:101A880000FA02FCC2F12002BCF1004F20FA02F277
:101A980043EB020008BF20F00100704702F120026A
:101AA80001FA02FCC2F1200250EA4C0021FA02F2CB
:101AB80043EB020008BF20EADC7070474FEA40029F
:101AC800B2F1FE4F0FD34FF09E03B3EB12620DD964
:101AD8004FEA002343F0004310F0004F23FA02F0CE
:101AE80018BF404270474FF00000704712F1610F75
:101AF80001D1420205D110F0004008BF6FF000404C
:101B080070474FF00000704753B94AB9002908BF21
:101B180000281CBF4FF0FF314FF0FF3000F06AB9CA
:101B2800ADF1080C6DE904CE00F006F8DDF804E02C
:101B3800DDE9022304B070472DE9F047089D0C4603
:101B4800002B4ED194468C458646B2FA82F262D971
:101B58004AB1C2F12003914020FA03F30CFA02FCC7
:101B6800194300FA02FE4FEA1C471FFA8CF6B1FB34
:101B7800F7F44FEA1E4307FB141143EA014304FB41
:101B880006F199420AD91CEB030304F1FF3080F0F7
:101B98001281994240F20F81023C6344591A1FFA9C
:101BA8008EF3B1FBF7F007FB101143EA014300FB8A
:101BB80006F69E420AD91CEB030300F1FF3180F0C0
:101BC800FC809E4240F2F980634402389B1B40EA45
:101BD800044000211DB1D3400022C5E90032BDE810
:101BE800F0878B4205D90DB1C5E9000100210846EF
:101BF800F5E7B3FA83F1002946D1A34202D3904214
:101C0800C0F0F080861A64EB03030120002DE6D0B3
:101C1800C5E90063E3E7002A40F09080A1EB0C04DB
:101C28004FEA1C481FFA8CF70121B4FBF8F64FEA7B
:101C38001E4308FB164443EA044307FB06F0984298
:101C480008D91CEB030306F1FF3402D2984200F2D4
:101C5800CD8026461C1A1FFA8EF3B4FBF8F008FB59
:101C6800104443EA044300FB07F79F4208D91CEBE2
:101C7800030300F1FF3402D29F4200F2B0802046F5
:101C8800DB1B40EA0640A5E7C1F120068B4022FA9B
:101C980006F71F4320FA06FC04FA01F343EA0C0393
:101CA800F44000FA01F8380C4FEA1349B4FBF0FE8F
:101CB8001FFA87FC00FB1E4449EA04440EFB0CF99A
:101CC800A14502FA01F20AD93C190EF1FF3A80F057
:101CD8008480A14540F28180AEF1020E3C44A4EB21
:101CE80009041FFA83F9B4FBF0F300FB134449EA33
:101CF800044403FB0CFCA44507D93C1903F1FF304D
:101D080067D2A44565D9023B3C4443EA0E40A0FB98
:101D18000293A4EB0C049C42CE469C4651D34ED071
:101D280055B1B8EB0E0364EB0C0404FA06F6CB408D
:101D38001E43CC40C5E90064002150E7C2F12003EE
:101D480020FA03F10CFA02FC24FA03F394400C4342
:101D58004FEA1C4800FA02FE1FFA8CF7B3FBF8F0B2
:101D680008FB1031230C43EA014300FB07F19942B9
:101D780008D91CEB030300F1FF362CD299422AD96B
:101D8800023863445B1AA4B2B3FBF8F108FB1133C1
:101D980044EA034401FB07F3A34208D91CEB0404FB
:101DA80001F1FF3613D2A34211D902396444E41A6F
:101DB80041EA004139E70446F0E6084606E7C84527
:101DC800AED2B9EB020E63EB070C0138A8E7314637
:101DD800EDE7034699E73046D4E7D6467FE7634404
:101DE80002384DE70646234608460FE7023E63449D
:101DF80030E700BF704700BF1348144A08B54FF0DA
:101E08000043C0E900230422426101220023C26189
:101E18004FF480510722C0E90233C0E90933C0E911
:101E28000C1203610383837680F8203080F82C300D
:101E3800826380F83C30C36404F092FE18B1BDE8B8
:101E4800084000F0DDBB08BDDC080020002401408C
:101E58000268084B9A4282B00AD14FF0B0431A6E1A
:101E680042F400721A661B6E03F400730193019B1F
:101E780002B07047002401400268054B9A4201BF36
:101E88004FF0B042136E23F400731366704700BF1F
:101E98000024014030B585B000240546CDE9014451
:101EA8000394FFF7A9FF144805F0EEF908B100F014
:101EB800A7FB1148039401A9CDE9015404F0AEFF32
:101EC80008B100F09DFB0C4805F008F908B100F0D6
:101ED80097FB4FF0FF31084804F042FF064805F031
:101EE800B5F9054804F096FF0446034805F058F98B
:101EF800204605B030BD00BFDC080020014B024A77
:101F08001A607047DC0800200024014008B5094821
:101F1800FFF7C0FF68B1084BB3F8AA304FF6FF725D
:101F2800934216BF40F6E442044B5343B3FBF0F32D
:101F380098B208BD002000B40075FF1FD8084C00F7
:101F480013B50023ADF80630FFF7E0FF0446194843
:101F5800FFF7A0FF184BB3F8C820B3F8A8108A42BF
:101F680004FB00F018D040F6E443B0FBF3F3642020
:101F78005B1A4343521A93FBF2F31E331BB2ADF8BC
:101F88000630BDF806305BB21B02ADF80630BDF86E
:101F9800060000B202B010BD4FF47A7240F6FF732B
:101FA800B0FBF3F35343A3F53923A3F50C6340F6D1
:101FB800C412E0E7001000B00075FF1F4FF0B043F7
:101FC80082B09A6A22F480529A629A6C42F48052E1
:101FD8009A649B6C03F480530193019B002002B028
:101FE80070474FF0B04307B59A6C42F004029A6408
:101FF8009A6C02F004020192019A9A6C42F0010272
:102008009A649B6C002203F00103114600930E2092
:10201800009B05F0D7F90E2005F006FA00221146BC
:102028000F2005F0CFF90F2003B05DF804EB05F0A1
:10203800FBB9000008B505F0D1FB10B16FF0040042
:1020480008BD064B9A6942F040429A614CF2FA3256
:102058001A6105F0D5FB0028F2D0EFE700400058E0
:10206800F0B585B000230D4600930646A8B3FFF7E8
:10207800E1FF044670BB05F0B1FB88BB1A481B4A58
:1020880002230193D0F8E01506F1784302EA812192
:10209800B3FBF1F701FB1733DB0A0293D0F8E00535
:1020A80005F178410139314402EA8022B1FBF2F0AE
:1020B80002FB1011C3EBD1230133694601A8039336
:1020C80005F01EFC20B1022814BF6FF001040124A2
:1020D80005F096FB204605B0F0BD6FF00504F9E762
:1020E8006FF00404F6E700BF0070FF1F00FCFF0359
:1020F800014B186000207047400900202DE9F04F7F
:10210800B0F1006F89B006460F469046C0F0C08017
:10211800DFF89091644DD9F8E03505EA832303F19F
:102128000063013B984200F2B380002900F0B380BD
:1021380040EA02035B0740F0AE80FFF77BFF0446EE
:1021480090BB05F04BFB002840F0A880D9F8E015BB
:10215800009705EA812106F17842B2FBF1F301FB11
:10216800132208F17843013B3344B3FBF1F001FB40
:102178001033DB0A01334FEAD22AA3EBD222012A19
:10218800039388BFC6F30A050AF58037C6F108032A
:102198008CBFC5F500654546FF02B3460693039B11
:1021A8009A4505D305F02CFB204609B0BDE8F08F11
:1021B800A6F10803069A1A4495421CD8009B049578
:1021C8000193CDF814B04FF00009059B09EB03010A
:1021D800049B99453DD3009BAB442B44A8EB0505D4
:1021E800B5F5006F009328BF4FF400650AF1010AA6
:1021F80007F50067D3E753F8081F5A68B2F1FF3FA5
:1022080008BFB1F1FF3FD5D0284B186810B96FF05F
:102218000504C7E727B14FF40062394610F08CFE79
:10222800DFF888900099D9F80030CBF30A001844F9
:10223800AAB210F081FE4FF400613846FFF710FF94
:1022480000BBD9F8003001934FF40063059704935D
:10225800B9E7019B07914B4402930120D3E900237E
:1022680005F008FB88B90799019BD1E9000259F8E4
:102278000310029B5B689A4208BF884205D109F1A6
:102288000809A2E76FF001048CE76FF0030489E7FF
:102298004FF0FF3488E76FF0050485E76FF004041A
:1022A80082E700BF0070FF1F00FCFF034009002009
:1022B800B1F1006F70B510D30B4BD3F8E0650B4B41
:1022C80003EA862303F10063013B994205D838B13C
:1022D80092B210F031FE002070BD4FF0FF30FBE7E6
:1022E8006FF00500F8E700BF0070FF1F00FCFF0358
:1022F800B0F1006F10B40DD3084BD3F8E045084B8C
:1023080003EA842303F10063013B984202D810BC1E
:10231800FFF7A6BE4FF0FF3010BC70470070FF1FDC
:1023280000FCFF034FF0B04382B0DA6C0243DA647A
:10233800DB6C03400193019B02B07047F0B50120AC
:1023480087B000242E4DCDE90444FFF7EBFF0220AF
:10235800FFF7E8FF0420FFF7E5FF0DEB00014FF65C
:10236800FF7203232846CDE90123039405F016FBE9
:1023780001A9244805F012FB01A94FF0904005F08F
:102388000DFB4FF0B0422846D36C23F00403D3640E
:102398002021012205F028FC01224FF400714FF0A2
:1023A800904005F021FC0220FFF7BCFF08214FF404
:1023B8000413CDE901130646049001A92846012714
:1023C800039405F0EBFA202301A92846CDE901374B
:1023D800CDE9037405F0E2FA102301A92846CDE9F6
:1023E8000137CDE9036405F0D9FA224621460920D0
:1023F80004F0E8FF092005F017F807B0F0BD00BFAA
:10240800000400480008004808B51248124A134B57
:10241800C0E9002300230122C0E90232C0E90433E5
:10242800C0E90633036205F05BFD08B100F0E8F887
:102438000848002105F0D4FE08B100F0E1F805488D
:10244800002105F0F3FE18B1BDE8084000F0D8B847
:1024580008BD00BF040A0020005800405D3E30203F
:1024680070B596B005461422002103A811F0A0F912
:102478003822002108A811F09BF92A68304B9A42AB
:102488005BD18023089308A84FF440230E9306F0ED
:102498003BFC08B100F0B4F84FF0B0444FF4C05022
:1024A800E36C43F00103E364E36C03F0010302937C
:1024B800029B12230026CDE903030323CDE905631C
:1024C8004FF09040042303A9079305F067FAA36D22
:1024D800DFF870C043F48003A365A36D1A4C03F4BE
:1024E80080030193019B26620D23C4E900C32046A3
:1024F8008023C4E90266C4E90436C4E9066604F028
:10250800F3FF08B100F07CF8104AEC63A562104CA8
:102518000E23C4E900231021002380222046C4E9A9
:102528000213C4E90423C4E90633236204F0DCFF80
:1025380008B100F065F8AC63A56216B070BD00BFC5
:102548000058004044000240A409002058000240FE
:102558004409002000B59BB04822002108A811F0CA
:1025680027F91822002102A811F022F905F084FEAB
:102578004FF0B0420120D2F8903023F01803C2F88F
:102588009030D2F8003423F4C06343F40073C2F8E7
:102598000034D2F8003403F4C0630193019B242370
:1025A800089381230B930023CDE91003B02208A8D8
:1025B800CDE9122305F0EAFF08B172B6FEE74F2312
:1025C800CDE90230CDE90400CDE90600022102A8D8
:1025D80006F076FA08B172B6FEE71BB05DF804FBA8
:1025E80008B504F083FAFFF7B5FFFFF7A7FEFFF77A
:1025F800F8FCFFF709FF00F008FD00F00DFDFCE70F
:1026080072B6FEE70F4808B50F4B03601F238360BF
:102618004FF080420023C0E90433C0E907238361F7
:102628004FF48073436206F0F1FC08B1FFF7E8FF4E
:10263800044806F017FE18B1BDE80840FFF7E0BFF0
:1026480008BD00BF580A00200028004010B5044605
:1026580090B03822002102A811F0AAF82268194B7C
:102668009A422CD14FF48033029302A84FF480731E
:102678000F9306F049FB08B1FFF7C2FF4FF0B043D4
:102688000220D3F8902042F40042C3F890209A6DBB
:1026980042F480629A659B6D002203F480631146C0
:1026A8000193019B04F08EFE022004F0BDFE00227F
:1026B8002A20114604F086FE2A2004F0B5FE10B048
:1026C80010BD00BF0028004010B50E4C0022204667
:1026D800102105F089FA4FF6FF714FF0904005F090
:1026E80009FA20464FF6FF7105F004FA06484FF63E
:1026F800FF7105F0FFF904F00FFABDE8104005F08E
:10270800E3BD00BF000400480008004804F00BBA0D
:1027180010B5104C00222046102105F065FA4FF63E
:10272800FF714FF0904005F0E5F920464FF6FF7134
:1027380005F0E0F908484FF6FF7105F0DBF904F001
:10274800EBF9064B0120BDE81040C3F8880005F0FE
:10275800FDBD00BF00040048000800480004005800
:1027680008B504F0E0F9FFF7E9FDFFF73AFCBDE82A
:102778000840FFF749BE08B504F0CEF9BDE80840A7
:102788000121002005F080BD04F0CDB97047FEE7B7
:10279800FEE7FEE7FEE7FEE77047704770477047C1
:1027A800014806F085BD00BF580A0020014804F022
:1027B800A7BF00BFA4090020014804F0A1BF00BFC3
:1027C80044090020082005F01DBA0000014806F061
:1027D800A3BB00BF580A0020014806F092BF00BF03
:1027E800BC0A00202DE9F04389B080460020109EE5
:1027F8000790894615461F46FDF712FDF0B9104CA3
:10280800CDE90090CDE9020407AB0E4805931423E7
:1028180004933A46434629460068FDF7CBFD234614
:10282800324604F1140153F8044B42F8044B8B422E
:10283800F9D1079B337509B0BDE8F0830120FAE7A9
:10284800A60A0020E43901081FB50E4C00233C22DB
:1028580002A8CDE902336275237500F0B7F80423A6
:1028680003AA009412210848FFF7BCFF0749142265
:10287800204610F08DFFB0FA80F35B09637504B051
:1028880010BD00BF900A00200C3A0108E50D002099
:10289800054808B50823036006F050FD18B1BDE8E7
:1028A8000840FFF7ADBE08BDBC0A00204FF0B0439A
:1028B80007B55A6E42F001025A665B6E002203F0B9
:1028C8000103019311463220019B04F07BFD322065
:1028D80003B05DF804EB04F0A7BD00000CB407B525
:1028E800054A05AB1021019310F030FE03B05DF8E6
:1028F80004EB02B0704700BF1E3A010830B585B03E
:10290800044602A80D4610F04DFCBDF90C30064AED
:1029180000931021029B2046FFF7E0FF2046FEF7B8
:102928004BFD288005B030BD1E3A01084FF0B0427B
:1029380010B5936823F40043936010F0BBFC0D4B73
:1029480001241C7010F088F90B4810F09FF90B4B0C
:102958004FF400421A61002010F09EF9FFF7CEFAFA
:1029680000F0B4F810F092FA21462046BDE8104075
:1029780010F0ACBAC80A0020052900080040005829
:1029880010F0BABA08B5FFF7C1FA40F6B833984262
:102998000CD8B0F5E16F0BD3FE23A0F5E1605843E6
:1029A8004FF49663B0FBF3F0C0B208BDFE20FCE71D
:1029B8000020FAE77FB5684600F06CF80198FFF749
:1029C8007DF800B207B05DF804FB0000194A38B57D
:1029D800D2F88035591C044619D104F0ABF80546E5
:1029E80004F0B4F8054404F0ABF82B0EE3712B0C9B
:1029F800A3712B0A6371030EE370C0F30742C0F39F
:102A080007232571C0B2A2706370207038BD190AFF
:102A1800C3718171190C1B0E41710371D2F8843591
:102A2800C370D2F88405C0F30722C0F30743000E31
:102A3800E9E700BF0070FF1F38B5094BD3F88035B0
:102A480003600133054609D104F074F8044604F024
:102A580077F8444004F07AF844402C6038BD00BF51
:102A68000070FF1F0121022010F01ABA0021022075
:102A780010F016BA00207047024B187808B100F021
:102A88005DB87047C80A002082B00190019802B072
:102A980000F0F0B810B50446FFF752FA074BA360F0
:102AA80040F30F20FEF7B6FF054B064A2360064B9E
:102AB8006060C4E90323002010BD00BF0000484245
:102AC80000007A440D093E00AB0305000020704762
:102AD800014B1868704700BFCC0A002003207047DC
:102AE80008B501464FF47A7200238002890DFFF77A
:102AF8000BF808BD4FF47A73A0FB0303800A40EA81
:102B080083507047034B98689A689042FBD1C04342
:102B1800704700BF0028004008B5FFF7F3FF014BDE
:102B2800186008BDCC0A002008B5FFF7EBFF024B80
:102B38001B68C01A08BD00BFCC0A0020024B1878D9
:102B480008B1FFF7DFBF7047D00A002010B5074B68
:102B5800074C0122DA654FF48071204606F0A2F98D
:102B68004FF0FF332363002010BD00BF0028004052
:102B7800580A002002460021014806F0AABB00BFFF
:102B8800580A002002460121014806F0A2BB00BFF6
:102B9800580A002010B58CB02C220021044601A848
:102BA80010F006FEFFF7D2FF0C4B0D481B681C44C3
:102BB8000023089306934FF00053E4430793012240
:102BC8004FF4807301A902940B9306F07FFA08B1C1
:102BD800FFF716FD00200CB010BD00BFCC0A002086
:102BE800580A002038B50546FFF78CFF0221044635
:102BF800074806F075FBC4F309024FF47A71A2FB8B
:102C08000121920AA30A2A8043EA805038BD00BFF6
:102C1800580A00200148002106F062BB580A00202B
:102C28000148012106F05CBB580A0020F8B50F4D99
:102C38002E78CEB90E4C4FF0FF372763FFF7E2FC32
:102C4800FFF784FF4FF48071204606F02BF92046E9
:102C5800276306F0E9FA32462046022106F039FBDE
:102C6800FFF75AFF01232B700020F8BDD00A00207F
:102C7800580A0020014610B54FF47A7200238002EA
:102C8800890DFEF741FF0146FFF73CFF0446FFF7B9
:102C980039FF031B8B4200D310BD00BFF7E710F0CC
:102CA80011BC000010B5064C0221204606F018FBA6
:102CB8000221421C2046BDE8104006F00ABB00BFB6
:102CC800580A00201348144A08B54FF4E133C0E904
:102CD800002300230C22C0E90233C0E90523C0E920
:102CE8000733C0E90933036107F003FB08B1FFF7B5
:102CF80087FC0848002107F071FC08B1FFF780FC49
:102D0800044807F04BFC18B1BDE80840FFF778BC51
:102D180008BD00BF340B002000440040F0B597B058
:102D280004461422002103A810F042FD3822002195
:102D380008A810F03DFD2268224B9A4240D1022398
:102D4800089308A8204B0A9305F0DEFF08B1FFF7A7
:102D580057FC4FF0B04302269A6D42F400329A6550
:102D68009A6D02F400320292029ADA6C42F0010281
:102D7800DA64DB6C03F001030193019B0423002553
:102D8800CDE903360327072303A94FF090400793A3
:102D9800CDE9055704F002FE082303A94FF090403F
:102DA800CDE90337059504F0F9FD084BE3672520C5
:102DB8002A4631469C6204F005FB252004F034FBCA
:102DC80017B0F0BD0044004004000C00D40A0020F5
:102DD80002680C4B9A4210B5044612D14FF0B0422B
:102DE8000C21936D23F4003393654FF0904004F069
:102DF80081FEE06F04F0EAFBBDE81040252004F0F6
:102E080021BB10BD0044004008B50A4601460248EF
:102E180006F074FD002008BD340B002013B5114BDB
:102E2800114C18604FF40013009302AB13E906002D
:102E3800204607F057FB2368DA69D103FCD4DA6926
:102E48005202FCD59A68084842F480029A6007F05A
:102E58008FFB06490448012207F000FB002002B05E
:102E680010BD00BFC80B0020340B0020D00B002081
:102E780008B5074B1860FFF7B4F8FFF723FF054ABA
:102E8800D2F8803043F00063C2F88030002008BDDB
:102E9800CC0B00200008005808B54FF0B043084894
:102EA8009A6B42F400329A639A6B22F400329A6366
:102EB800FFF78EFF112004F0C5FA002008BD00BFFF
:102EC800340B00200268044B9A4203D1034B0020C4
:102ED8001B681847704700BF00440040CC0B002017
:102EE80002680B4B9A4210B504460FD1094B1B6878
:102EF8002BB1D0F8902012B90748012198472046F5
:102F08000549BDE81040012207F0A8BA10BD00BF6E
:102F180000440040C80B0020D00B002002480122CA
:102F2800102104F061BE00BF0004004802480022DE
:102F3800102104F059BE00BF0004004810B50A4C27
:102F480023780BB9E37C6BB1FFF77EFC0038074BA5
:102F580018BF0120400018701B78022B02BF002305
:102F68002370E37410BD00BFE50D0020D80B0020CE
:102F780038B5114C2378F3B9E37CE3B90F4D2B68CE
:102F8800012B07D92B68042B04D80D4A04210120F2
:102F980000F010FA2B68042B0DD9FFF755FC003808
:102FA800084B18BF0120400018701B78022B02BF85
:102FB80000232370E37438BDE50D0020D40B0020F6
:102FC800783A0108D80B002008B5FFF7A7FF0A20B8
:102FD800FFF75AFD01F014FABDE80840FFF7A6BF55
:102FE800022801D8FFF79ABF7047022801D8FFF7D7
:102FF8009DBF7047022803D80248102104F0F9BD8C
:10300800704700BF00040048704708B5FFF78EFC02
:10301800BDE8084000F06EBB4FF0FF300FF0D0BFA6
:103028007047704770470000014BD870704700BF69
:103038000C000020014B1874704700BF0C000020E2
:1030480008B500214FF480700FF082FF02200021A4
:103058000FF07EFFBDE80840014810F0E1B900BF5D
:10306800480D0020002101200FF072BF10B542F278
:103078001073084C002818BF03460748236010F057
:1030880081F92168044810F005FABDE810400248AB
:1030980010F0C6B908000020480D002010B5094CF2
:1030A800206023680BB9084B2360084810F06AF9C0
:1030B8002168064810F0EEF9BDE81040034810F00A
:1030C800AFB900BFB4000020A0860100DC0B0020CF
:1030D80010B5044680B190F906306BB90C4810F071
:1030E80051F90C4BE2791A700B4B1868FFF7D6FFB1
:1030F8000A4B1868FFF7BAFF00214FF480700FF0F1
:1031080027FFBDE81040002102200FF021BF00BFBB
:10311800F40B0020E20D0020B4000020080000207D
:103128000A460149FFF7C4B800F0030838B50C484F
:1031380010F028F907F0B2FE60B90A4C0A480125D8
:10314800257007F03FFD2078294607F093FA0448D8
:1031580010F066F9BDE83840044810F061B900BFC6
:10316800480D0020700000200C000020300D0020C9
:1031780007F032BF30B585B0FFF704FC044607F00E
:1031880073FB054688B100243A4810F0FBF83A4B27
:1031980038481B689C42214638BF194610F07AF916
:1031A800344810F03DF905B030BD684601F014F818
:1031B80023B203EB4303FE2203EB4313B3FBF2F307
:1031C8002E4A392111702E4950680978DBB28DF8E2
:1031D8000C3001705068457050682724847050681E
:1031E8000124C47050680371264B187818B31D70F9
:1031F800536861F07F0119703A231370052322493F
:10320800224C0978012988BF00235370637A33B1AF
:1032180007F016FB012802D1204610F0B3F81C4B2A
:103228001648D978002207F035FB0630ABD107F0F5
:1032380001FB0446A8E7174B1748197811B901781C
:103248000029DBD0002101701970536804215971DD
:10325800BDF800305168180A88715168CB71BDF803
:10326800083051681B0A0B72BDF808304B720A23EC
:10327800C5E700BF480D002008000020000000201E
:103288003C0C0020E10D0020D80B0020F40B00209E
:103298000C000020600D0020E30D002020B1037811
:1032A80013B1024810F0BCB8704700BF240C0020CE
:1032B80008B5104B0122002102201A700FF048FEB9
:1032C8000D4810F0ADF80D4B1B788BB10C4B1A78EC
:1032D80072B9DB7C63B90B4B1A68042A9EBF1A6863
:1032E80001321A600021BDE8084010200FF030BEFE
:1032F80008BD00BFE10D0020DC0B0020E20D00201E
:10330800E50D0020D40B0020044B1B78022B03D1C1
:10331800002108200FF01CBE704700BF700000207D
:1033280008B507F0C4FD80B907F08AFA01280CD166
:10333800BFF34F8F0549064BCA6802F4E062134396
:10334800CB60BFF34F8F00BFFDE708BD00ED00E085
:103358000400FA0538B504460D4607484FF40061E5
:10336800FEF7C6FF30B92A4621460348BDE8384073
:10337800FEF7C4BE38BD00BF00F0030870477047B1
:1033880070477047012808B502D008280BD008BD3F
:1033980000214FF480700FF0DBFDBDE808400021EC
:1033A80002200FF0D5BD024B01221A70EFE700BFD3
:1033B800600E002070B505460C46164607F054FA14
:1033C8000346002835D000241B480FF0DBFF1B4BB9
:1033D80019481B689C42214638BF194610F05AF814
:1033E800BDE87040144810F01BB84A68F05CD0542F
:1033F8000133DAB29442F8D8114B0D701B78012BC7
:1034080088BF00244C700F4C637A33B107F018FA68
:10341800012802D120460FF0B5FF0B4B0B48D97895
:10342800002207F037FA0630CDD107F003FA044638
:10343800CAE70649DDE700BF480D00200800002064
:10344800D80B0020F40B00200C0000200000002006
:10345800044B1B7823B9044A05210120FFF7AABFB2
:10346800704700BFD80B00207D3A010810B5002432
:1034780090B03C22214601A8009410F099F92F4BF6
:103488002022DA7219788DF8001059788DF8011019
:1034980099788DF80210D9788DF8031019798DF87C
:1034A800041059798DF8051099798DF80610D97995
:1034B8008DF80710197A8DF80810597A8DF80910C7
:1034C800997A8DF80A108DF80B2021460DF10B0220
:1034D80058180131007B02F8010F1C29F8D193F824
:1034E80028208DF8282093F829208DF8292093F892
:1034F8002A208DF82A2093F82B208DF82B2093F87A
:103508002C206AB193F83F2052B10DF12B01002213
:103518009818013290F82C0001F8010F142AF7D1FD
:1035280007484FF40061FEF7E3FE20B90448402243
:103538006946FEF7E3FD10B010BD00BF7100002022
:1035480000F80308014940220FF0F6BC00F8030810
:1035580070B52A4D28796B794D2BC0B233D1C0EBA9
:10356800001080000A2838BF0A204FF47A735843A5
:10357800234BAC791860EB794D2BE4B22BD1C4EB1B
:103588000414A40095F82C301E4E63BB95F83F3008
:103598004BBB42F21070FFF769FD3068FFF77EFD04
:1035A8002B7A194A1949DBB213706B7A184ADBB2C5
:1035B80013700023EA1892F82C20D2B2CA540133AF
:1035C800142BF7D170BD6B79482B0ABF4FF4616398
:1035D8006B795843C6E7EB79482B0ABF4FF4616310
:1035E800EB795C43CEE7FFF741FD012C38BF01249E
:1035F8004FF47A735C433460CFE700BF710000205A
:1036080008000020B4000020E40D0020E50D002093
:10361800D80B002010B590B000213C2201A80091E1
:1036280010F0C6F84022314968460FF085FC9DF835
:1036380000203AB99DF80100272803D19DF802100F
:10364800012909D0FFF712FF4FF47A70FFF71CFA2F
:10365800FFF77EFF10B010BD254B1A705870997097
:103668009DF80310D9709DF8041019719DF8051084
:1036780059719DF8061099719DF80710D9719DF838
:10368800081019729DF8091059729DF80A1099725C
:103698009DF80B1001F03F01D972D87AD1B2884257
:1036A8001BD89DF8282083F828209DF8292083F826
:1036B80029209DF82A2083F82A209DF82B2083F8BA
:1036C8002B200DF12B0100229818013211F8014F1F
:1036D80080F82C40142AF7D1BAE701F14000684479
:1036E800194410F8340C08730132D6E700F80308BF
:1036F800710000201FB5002403A92046039407F099
:10370800BBFB03A9012007F0B7FB384B38480094EE
:1037180022464FF4FA710FF0D7FD364B3648009425
:1037280022464FF4FA710FF0CFFD344B3448009421
:1037380001224FF4FA710FF0C7FD2046FEF7D8FCBE
:1037480008B1FEF75DFF2F4B009400224FF4FA6199
:103758002D480FF0B9FD2D4A002101200FF0B4FCCF
:103768002B4A002102200FF0AFFC2A4A0021042036
:103778000FF0AAFC284A002108200FF0A5FC00F051
:10378800A7FB2649264807F02DFB264807F01AFA1A
:103798001B480FF045FE244B0021187806F06AFFFD
:1037A80022490094224B0968224800220FF08CFD20
:1037B80020480FF035FEFFF72DFF1F4A002110208B
:1037C8000FF082FC1D4A00214FF480700FF07CFC42
:1037D8001B4B1C4819681C4B009400220FF074FD09
:1037E80018480FF01DFE04B010BD00BF8933000853
:1037F800240C00208B3300080C0C002085330008B3
:10380800F40B002011330008300D0020D1A9000866
:103818007D310008793100083531000800000301C6
:10382800240000200C000020700000200800002068
:1038380049300008480D0020792F0008D12F0008D2
:10384800B4000020DC0B0020B932000810B50024B9
:10385800A2B07C22214603A802940FF0A9FF5323AB
:103868008DF8083040F22713ADF80A3001238DF89F
:103878000C30ADF80440FFF785F800B200EB4000CB
:1038880000EB4010FE23B0FBF3F08DF80D0001A80B
:1038980000F0B0FCA0B958238DF80E300724802220
:1038A800002114480FF084FF224602A911480FF0A6
:1038B800B8FF104A21460120FFF77CFD22B010BD59
:1038C800430001338DF80E308DF80F0000F098FD9D
:1038D800094B1A6812128DF810201A688DF81120F9
:1038E8005A685B688DF8133012128DF812200C2478
:1038F800D5E700BF610D0020640E002030B50378C5
:10390800592B91B0044640F0FC81052959D84378D9
:10391800443B162B55D8DFE813F03D0154002D0128
:1039280054003501540054005400540092005400CF
:103938001801540054005400A30154005400AE0070
:1039480054005400540017008578482D11D1BB4A03
:1039580014210120FFF72EFD41F28830FFF794F87B
:1039680040F6B830FFF790F811B0BDE83040FFF7E7
:10397800D7BC532D0ED180220021B1480FF018FF7B
:10398800FFF764FF41F28830FFF77EF8AC4A152153
:10399800012085E0432D16D1002468468DF80040AB
:1039A80007F088F8A64A4C231370272393709DF8D4
:1039B8000030547001204133D07013710521FFF796
:1039C800F9FC11B030BD442DFBD19D4C5923237017
:1039D8005A236370A57000F0F1FB7F220021601C60
:1039E8000FF0E6FE272325700125A370E5702571E9
:1039F800FEF7C8FF9349FE23B0FBF3F00B6864227F
:103A08009BB2B3FBF2F3A3710B6800EB400000EB31
:103A180040109BB26071B3FBF2F002FB1033E3710C
:103A28004B689BB2B3FBF2F323724B689BB2B3FBB8
:103A3800F2F102FB1133637222460A21A8E7837868
:103A4800303BDBB2092BBCD87F49804A0B700B781E
:103A5800DBB253727A4A592313704D2353700B7893
:103A68000120303303219370FFF7A4FC11B0BDE8A7
:103A78003040FFF7FBBC8578482D16D1704A562395
:103A88001370002353702723937003231371182393
:103A980053710523012093711723D070D371082126
:103AA80011B0BDE83040FFF785BC432D89D1002413
:103AB80021463C2201A800940FF07AFE6846FFF7E1
:103AC80041FD634B2146732218460FF071FE9DF8A5
:103AD800002000F80C2C9DF8012000F80B2C9DF814
:103AE800022000F80A2C9DF8032000F8092C9DF804
:103AF800042000F8082C9DF8052000F8072C9DF8F4
:103B0800062000F8062C9DF8072000F8052C9DF8E3
:103B1800082000F80D5C00F8042C9DF80B509DF867
:103B2800092000F8032C9DF80A2000F8022C03A9AC
:103B38002A46A0F10D0400F8015C0FF072FE05F1B1
:103B48000D012246C9B2012039E7807839280CD8FE
:103B58003038C0B2FFF744FA394A237813706378D3
:103B68005370A3789370032112E711B0BDE8304079
:103B7800FFF76EBC80783928F7D83038C0B2FFF725
:103B880034FAE9E780783928EFD83038C0B2FFF73F
:103B980031FAE1E78378303BDAB2092AE5D8C07810
:103BA8003038C2B2092AE0D82179A1F14802D2B24C
:103BB8000B2ADAD8274D45FA02F2D507D5D40A22BE
:103BC8004D2902FB030034D13C2358434FF47A7348
:103BD8005843214B1860FFF749FA194A23781370A4
:103BE80063785370A3789370E378D37005212379B1
:103BF80013710120FFF7DEFB144B00221A702722F5
:103C08005A7001229A70DA70A278303A02EB820177
:103C1800E278303A02EB4102D2B21A7122795A7133
:103C28000E4A1278D2B21A72074A1278D2B25A726F
:103C38001CE74829CAD14FF46163C6E7833A0108F3
:103C4800610D0020640E0020D80B002071000020B8
:103C58006E0D0020DEF7FFFF08000020E40D0020B5
:103C68008278303AD3B2092B3FF67FAFC378303B26
:103C7800D9B209293FF679AF0079A0F14801C9B254
:103C88000B293FF672AF624D45FA01F1C9073FF5BE
:103C98006CAF0A214D2801FB02332DD13C2253433E
:103CA8004FF47A7253435B4A13601068FFF7F6F9D2
:103CB800594A2378137063785370A3789370E37824
:103CC800D3700521237913710120FFF773FB534B40
:103CD80000221A7027225A7001229A70DA70A2788C
:103CE800303A02EB8201E278303A02EB4102D2B27A
:103CF8009A712279DA7193E74828D1D14FF4616239
:103D0800CDE7502B48D102297FF65BAE4378303B94
:103D1800012B3FF656AE8378312B7FF452AE0B2938
:103D280004D8FFF795FB00213B4A31E63B4D0234AE
:103D3800002214F8013FA918303B0132DBB20C2AEB
:103D48000B73F6D1FFF760F9334B502227211A7015
:103D58009970002201215A70D97003F8041FA9181C
:103D68000132097B0C2A01F1300103F8011FF6D159
:103D780000232B7027236B700123AB70EB70284B4B
:103D88001B78DBB22B72274B1B78DBB26B72EA72A3
:103D9800FFF76CFB1121C7E7412B7FF412AE437884
:103DA800432B7FF40EAE16297FF40BAE1E4D421C3A
:103DB800002312F8011FE9540133142BF9D1FFF73E
:103DC800BDF81A4B5B7D012B1DD114490023EA5C19
:103DD800C8180133D2B2142B80F82C20F7D1114B1C
:103DE80000221A701B78DBB24B72FFF73FFB0A4ABE
:103DF800631E153413F8011F02F8011BA342F9D101
:103E0800054A1621C4E5074B02221A70EFE700BFE6
:103E1800DEF7FFFFB4000020610D002071000020D4
:103E2800E40D0020D80B0020E50D0020900A0020AA
:103E380037B504460D46002939D022480FF0F0FA6C
:103E48002B78A3B39CB36068237880B3032B0DD081
:103E5800392B2ED0022B2AD16178012927D00B06C5
:103E680025D403B0BDE83040FFF748BD6378012B87
:103E780007D10078012802D0022800D008B906F03E
:103E8800D3FD00240DF107008DF8074006F012FE5F
:103E98000D4A4C231370272393709DF807305470F4
:103EA800012041330521D0701371FFF783FA03B065
:103EB80030BD6378012BFAD10378044A03F001037B
:103EC8001370F4E70C0C0020610D00203C0C00205E
:103ED800034B0022C3E902220122C3E900227047F2
:103EE800FC0D002000487047FC0D00204FF0B04347
:103EF80082B0DA6C0243DA64DB6C03400193019B05
:103F080002B070472DE9F04186B000240220154D1B
:103F18000594FFF7EBFF0420FFF7E8FF124F039427
:103F28004FF4807601230DEB0001CDE901632846AB
:103F3800032304934FF4005803F030FD01A93846D9
:103F4800CDF8048003F02AFD22464146384603F0A6
:103F58004BFE28462246314603F046FE204606B070
:103F6800BDE8F0810004004800080048032810B5A7
:103F78000ED8012810D868B902460B484FF4807152
:103F880003F032FE002209484FF4005103F02CFEE2
:103F9800002010BD0122F0E7002203484FF4807191
:103FA80003F022FE0122EEE7000400480008004862
:103FB800022070470020704701207047002814BF76
:103FC80016200F20704700000D48854602F08CFD32
:103FD8000C480D490D4A002302E0D458C45004335C
:103FE800C4188C42F9D30A4A0A4C002301E0136032
:103FF8000432A242FBD30FF0E3FBFEF7F1FAFEE72F
:104008000000012000000020BC0800208C450108A9
:10401800BC0800205C2C0020FEE74FF0B04382B0C3
:10402800DA6C42F00102DA64DB6C03F001030193FD
:10403800019B02B07047000030B587B0FFF7EDFF75
:104048004FF4805101224FF0904003F0CDFD012242
:104058004FF400614FF0904003F0C6FD4FF4C05597
:104068001123CDE9015301A901234FF09040039397
:1040780003F094FC08240A2500224FF480514FF0E5
:10408800904003F0B1FD0120FEF7FEFC01224FF441
:1040980080514FF0904003F0A7FD0120FEF7F4FC9B
:1040A800013DE9D14FF400614FF0904003F096FDD7
:1040B80008B9013CDFD14FF400614FF0904003F0A4
:1040C8008DFD68BBFFF7A9FF04240123039001A914
:1040D8002A48CDE9014303F061FC284C0122042160
:1040E800204603F081FD2120FEF7CEFC00220421AA
:1040F800204603F079FD2120FEF7C6FC01220421A9
:10410800204603F071FD2120FEF7BEFC2046002268
:10411800042103F069FD4FF42570FEF7B5FCDDE7D7
:10412800FFF77BFF4FF0B04300249A6D42F4800202
:104138009A659B6D03F4800300934FF4C052009B73
:104148001223CDE901230323CDE9034304230DEB17
:1041580003014FF09040059303F020FC08480949FB
:10416800094B8460C0E900130123C0E90334C0E9A6
:104178000744446103F0B4FE07B030BD00040048B2
:104188000C0E0020005800401A091020FFF754BFF9
:1041980010B1012809D0704701394A424A414FF00D
:1041A80090404FF4007103F01FBD4B1E5A42024865
:1041B8005A412021F7E700BF0004004808B5012054
:1041C800FEF70EFF6420FEF75FFC00F019F9BDE86A
:1041D80008400120FEF709BF044B1A685B68038199
:1041E800034B028001221A70704700BF640E002042
:1041F800E30D002010B5044600F008F810F0FF00A9
:104208001CBFEE232370AA23637010BD2DE9F7436A
:1042180000242D4E2D4D346021462046FFF7B8FF6F
:1042280021460120FFF7B4FF5227A046012195F847
:10423800640185F86071C5F86881FFF7A9FF03205C
:10424800FEF722FC00228821284602F0BBFB0DF174
:104258000602C021284602F005FC78BBBDF80620FE
:104268004EF6AA639A4229D14FEA440909F1540942
:104278004946284600F030F900BB85F860910DF1F9
:104288000602C021284602F0EDFBB8B9284600F026
:10429800DFFA98B9326801231A4432600C4AC5F82B
:1042A80068311168A3400B43136005F5C8751CB14C
:1042B800306803B0BDE8F0830124B7E70021204649
:1042C800FFF766FFF1E700BF740E0020B80000207A
:1042D800700E00202DE9F74F344C054604F5487B55
:1042E8004FF00A0A4FF00E0948F2E8084FF4901709
:1042F8004FF48046D4F86831002B50D0204600F0A7
:1043080097FD0DF102020DF10101204600F058FB66
:104318000DF1030201A9204600F08CFE0021204681
:1043280000F0DEF801220021204600F09EF901226B
:104338001146204600F099F9022D0ED81C4B33F88F
:1043480015601C4B53F825701B4B53F825801B4BED
:1043580013F805901A4B13F805A0324601212046A0
:1043680000F0CCF93A460021204600F0C7F9414652
:10437800204600F0CFF84A460021204600F0CCF84D
:1043880052460121204600F0C7F80DF102020DF156
:104398000101204600F014FB0123C4F87C3104F528
:1043A800C874A345A6D103B0BDE8F08FB8000020BB
:1043B800B83A0108AC3A0108A03A01089B3A01084A
:1043C800983A010810B50B7E9BB9D0F87C21098971
:1043D80012B1C0E95E1310BD084BD0F878411A68D5
:1043E800C2F580734B4304FB02331B12C0F87831CB
:1043F800F1E70123C0F87C31EDE700BF6805002034
:104408002DE9F84FDFF8B8A02E4DFFF7BFFEDAF818
:1044180000300BB12B6813B9FFF7F8FE28602B6842
:10442800294F0024A3423C607C6042DDDFF89C8079
:10443800274D0220FFF74EFF88F80040D5F8683175
:10444800012B2ED1DFF88CB003FA04F90A26214992
:10445800284600F04DFCB0B959462846FFF7B2FF90
:104468009BF818307BB9D5F8783147F82430DAF85A
:10447800003043EA0903CAF8003098F8003043F0E6
:10448800010388F800301E20FEF7FEFA9BF818306A
:104498009BB1013E16F0FF06D9D14FF47A7347F865
:1044A80024301E20FEF7F0FA05F5C8751CB198F8FF
:1044B8000030BDE8F88F0124C0E7D5F87831EEE781
:1044C800700E00206C0E0020640E0020E30D00200A
:1044D800B8000020780E00204A088A2102F072BA3B
:1044E800152906D8044BCB40DB0702D50174002000
:1044F80070476FF0070070470B00300010B50A4690
:104508000C46092102F080FA18B9237803F0010358
:10451800237010BD01F051BE01F02EBD01F033BE75
:10452800F7B500230F46144601210DF10702064690
:104538008DF8073002F068FA0546D0B9012C9DF8CD
:10454800073025D1042F39D8DFE807F00316191CE6
:104558001F0043F010049C420BD022460121304634
:1045680002F030FA68BB716986F830413046FFF7CF
:10457800D1FF284603B0F0BD43F02804EBE743F031
:104588000404E8E743F04004E5E743F08004E2E789
:10459800042F13D8DFE807F00306090C0F0003F017
:1045A800EF04D8E703F0D704D5E703F0FB04D2E71C
:1045B80003F0BF04CFE703F07F04CCE76FF00305F7
:1045C800D7E70546D5E713B500230C460DF10702DA
:1045D80001218DF8073002F017FA78B99DF80730F5
:1045E800C3F300122270C3F3C002A270C3F38002A7
:1045F8006270C3F38012DB09E270237102B010BD50
:1046080037B50D460DF10202F821044602F02AFAE8
:1046180070B901AA0421204602F042FA40B9BDF857
:1046280002201AB1019BB3FBF2F32B602B68A36144
:1046380003B030BD037F0B700020704737B50D46BF
:104648000DF106022021044602F00CFA28B9BDF843
:10465800063023B9236A2B60207703B030BDDB0016
:104668002B60236201232377F7E70529F8B5044671
:104678000E46154633D862B100EB810301215A6B0F
:104688000023701E042807D8DFE800F010191C1F4B
:10469800260011460123F4E784F82810003D34442D
:1046A80018BF012584F82850002007E0C2F34F22E4
:1046B8004421204602F096F90028EFD0F8BD84F88E
:1046C8002A10EBE784F82B10E8E75B00FE22602154
:1046D800204602F0B0F9EFE71B01EF22F7E76FF091
:1046E8000300EBE7052996BF4018002390F828300F
:1046F800137094BF00206FF00300704770B5431823
:10470800044693F828300E4615463BB105291BD8B8
:10471800DFE801F0030912141616426304EB86045D
:104728000020656307E0C2F34F224421204602F0CF
:1047380059F90028F2D070BDC263EFE70264EDE7D3
:10474800C2F34F226421F1E76FF00300F3E737B5B6
:104758000446154605292AD8DFE801F00306141691
:104768001818436B2B601FE00DF10602442102F07C
:1047780079F9D0B9BDF8062053028AB12B60A3633A
:1047880001230FE0C36BEDE7036CEBE70DF10602C5
:10479800642102F067F940B9BDF806305B02E1E731
:1047A800A26B2A6084F82930002003B030BD6FF076
:1047B8000300FAE737B50D460DF10702012104465B
:1047C80002F022F938B99DF8073084F83031DB0956
:1047D8002B7084F84C3003B030BD2DE9F843037CCE
:1047E8000C4601F8083B0546FFF70AFF40BB20735B
:1047F80004F110012846FFF721FF08BB04F114015A
:10480800284600F019FCD8B904F1240705F1270956
:1048180004F1170806463A46B1B22846FFF797FF53
:1048280070B9013619F8013F08F8013F062E07F163
:104838000407F0D104F13C012846FFF7BBFF08B19B
:10484800BDE8F883211D2846BDE8F84301F01DBDE9
:10485800F0B50022054693B0882102F0B3F84FF472
:104868007A72A5F852214FF4C872A5F85421514A1A
:10487800C5F858210023504A85F8F030C5F8D420EF
:104888002B6202A92846FFF7A8FF044670B9ADF8C5
:10489800080002AE0FCE05F110070FC70FCE0FC7E5
:1048A8000FCE0FC796E80F0087E80F00434BC5F8F7
:1048B80034314FF4FA730126A5F838314FF42063E8
:1048C800A5F83C313246802185F85061284602F02F
:1048D80079F832460746FF21284602F073F800228D
:1048E80011460743284602F06DF83C4364B204437E
:1048F8000DF107029121284602F086F864B29DF86E
:10490800073085F83A31044332460021284602F040
:1049180059F864B204430022FF21284602F052F8F5
:1049280064B2044300228021284602F04BF864B2A6
:10493800204340B200283BD013B0F0BD0028FBD183
:10494800A1B2012228460134FFF78FFE062CF5D1CB
:104958000028F1D104466885024604212846FFF75D
:1049680084FE0028E8D1024605212846FFF77DFE8F
:104978000028E1D14FF490136B634FF4804201217A
:104988002846FFF7BBFE0028D6D14FF40C13FF22B0
:10499800C5E90F3085F830210121284602F012F8C8
:1049A800012385F832310028C6D185F81541C3E7BF
:1049B8000446C5E7856B0100A47009006400840300
:1049C800012300F069BD2DE9F0428EB00C460C239E
:1049D80004AA1421054601F0DDFF8446002860D1B1
:1049E800BDF81620BDF81830A075BDF8121020606B
:1049F80052BA5BBA6060BDF81A60B5F8520192B25B
:104A08009BB249BA5B0252022361A18276BAE26084
:104A1800B0F57A7F8BB295F831719DF81010B6B267
:104A28000AD0704300F5FA704FF47A76B0FBF6F0CE
:104A38002E7F002E39D186B2002F40D0B001C0B2EF
:104A4800B608E0750DF10F002681CDE90040284633
:104A580001F072FE844620BB9DF80FE084F818E050
:104A680005F150060FCE07AF0FC796E80700E37DA4
:104A780087E80700D4E90301A28AADF83020D4E919
:104A88000149CDE90A01CDE9084907AC8DF8333071
:104A98008DF834E00FCC50350FC597E8070086E84D
:104AA800070060460EB0BDE8F0822E8C5E43B2EB84
:104AB800262F4FEA262C04D157B948F6E0260020C5
:104AC800BFE780B25043A2EB0C06B0FBF6F0B2E7AA
:104AD80042F2B826B2E70000F7B517460E210DF1ED
:104AE80006021D460B4C064601F0BCFFBDF8063019
:104AF80004EA43433B6050B90DF106020C213046ED
:104B080001F0B0FFBDF8063004EA43442C6003B05E
:104B1800F0BD00BF0000FE1F73B590F8DA30013B0E
:104B2800022B06460C4634D801AB6A460121FFF732
:104B3800D3FF009BB3F57F0F054603D8019BB3F560
:104B48007F0F23D915BB34B11349304602B0BDE8F5
:104B5800704001F0FFBB0422FF21304601F032FF14
:104B68002A4604467021304601F02CFF2A460443A9
:104B7800FF21304601F026FF64B204432A46802113
:104B8800304601F01FFF64B2044365B2284602B004
:104B980070BD0025FAE700BF6C05002037B5044654
:104BA80001228021057C01F00DFF0122FF21204612
:104BB80001F008FF00221146204601F003FF94F897
:104BC8003A219121204601F0FDFE012200212046D4
:104BD80001F0F8FE0022FF21204601F0F3FE00223A
:104BE8008021204601F0EEFE012D24D0032D32D085
:104BF800C5BB01222946204601F0E4FE01238DF8B9
:104C08000730B0B905469DF80730DB0705F1010507
:104C18000AD548B9B5F5FA6F27D001460DF1070254
:104C2800204601F0F1FEEEE7B5F5FA6F08BF6FF028
:104C3800060003B030BD18B929462046FFF76CFFBF
:104C480002220021204601F0BDFE0028F1D10423F4
:104C580084F83231EDE718B901212046FFF75CFFEF
:104C68000422EEE76FF00700E3E76FF00600E0E7E5
:104C780038B5057C044625B1204600F03BFD28B137
:104C880038BDFFF78BFF0028F6D0F9E7002DF7D1E4
:104C9800032384F83231F3E773B506460025012271
:104CA8000B21304601F08EFE002204460B213046CF
:104CB80001F088FE0DF1070204431321304601F08C
:104CC800A3FE9DF8073064B2044301355B0760B268
:104CD800EDB205D0032D08D00028E0D002B070BD99
:104CE800032D08BF6FF00B00F8E76FF00B00F5E736
:104CF80038B50023037404460D46FFF7B9FF50B9D1
:104D080029462046FFF75FFE28B901462046BDE840
:104D18003840FFF7C1BF38BD152970B5054616469E
:104D28001C4667D10122FF2101F04CFE00221146EA
:104D38000446284601F046FE00220443FF21284687
:104D480001F040FE64B2044301228021284601F0AC
:104D580039FE64B2044302228521284601F032FE5E
:104D680064B204430422FF21284601F02BFE64B2FA
:104D780004430022CD21284601F024FE64B20443F6
:104D88001122CC21284601F01DFE64B204430722FB
:104D9800FF21284601F016FE64B204430022BE211A
:104DA800284601F00FFE64B204430622FF2128467C
:104DB80001F008FE64B204430922CC21284601F020
:104DC80001FE64B204430022FF21284601F0FAFDE7
:104DD80064B204430122FF21284601F0F3FD64B2C6
:104DE800002204431146284601F0ECFD64B220433A
:104DF80040B270BD042A17D80A2101F0E3FD00284B
:104E0800F7D1231E18BF01231B01EF228421284656
:104E180001F011FE0028ECD185F8DA600146284639
:104E2800BDE87040FFF738BF6FF00A00E1E7000007
:104E380070B594B005464022002104A80EF0B8FCD5
:104E4800002301212846ADF806308DF803308DF88F
:104E58000430029300F0A0FC95F8142195F8131182
:104E6800012A04D840F0AD80202940F2AC8001AA84
:104E780002A9284600F02BFB0446002840F09E803B
:104E880095F85031002B40F0A280D5F84C112846F7
:104E980001F060FA0446002840F09080034601467D
:104EA80004222846FFF738FF0446002840F0868091
:104EB8000122FF21284601F085FD0DF10602064674
:104EC8008421284601F0CEFD22460643FF212846CC
:104ED80001F078FD76B2064374B2002C6ED1BDF8AD
:104EE80006301B01C5F8D43004A92846FFF775FC25
:104EF8000446002862D10DF103012846FFF7FEFAA7
:104F0800044600285AD19DF8033085F8313104ACA5
:104F18000FCC05F110060FC60FCC0FC60FCC0FC66D
:104F280094E80F0086E80F000DF1030201212846DE
:104F380001F06AFD0446002840D19DF8033085F849
:104F48003031024601462846FFF7EAFA0446A8BB74
:104F5800024602212846FFF7E3FA044670BB032302
:104F6800014685F832310DF10502284601F00BF9AA
:104F7800044618BB9DF8053085F8E8300DF10502A8
:104F88000121284601F0FFF80446B8B99DF805301C
:104F980085F8E03003AA0321284600F0E7FE04461E
:104FA80060B9039BC5F8E43003AA0421284600F041
:104FB800DDFE044610B9039BC5F8DC30204614B06A
:104FC80070BD0C2951E7284600F013F954E7014950
:104FD8005DE700BF2207002013B50C460DF107025C
:104FE800132101F011FD9DF8073013F0180F03F09D
:104FF800070218BF6FF00500226002B010BD13B59C
:1050080090F8DA30042B0C4609D101A9FFF7E4FF28
:10501800019B1A1F53425341237002B010BD01AACD
:10502800142101F0F1FC0028F7D19DF8043003F0B9
:105038000103F1E700F04BBA13B50C460DF1060277
:10504800282101F00FFD78B9BDF80620C2F30B0343
:1050580012F4006F18BFA3F580534FF0FA0214BF83
:1050680013FB02F35343236002B010BDF0B54FEABF
:10507800D20C4FF0FF341C6002F00702664600278E
:105088008E4200D207B1F0BD845D664503BF14416E
:10509800E4B215463D4614F0010705D005EBC605F8
:1050A8001D6001270136EBE70135082D4FEA54044E
:1050B800F8D014F0010FF0E7034B800953F82000F3
:1050C800003818BF012070471808002010B5B1EB50
:1050D800D20F4FEAD20402F0070381BF01229A409F
:1050E800035D13438ABF03556FF03100002010BDE4
:1050F8000A460623B02101F02FBC0A460623B02138
:1051080001F048BC2DE9F04F85B00546109F0E9E72
:1051180001978A4693461C464FF00009119B994512
:1051280008D10023129A176013B36FF0310005B04D
:10513800BDE8F08F01AB3A4631465846FFF796FF77
:10514800DDF80480B8F1FF3F0FD00F9B08EB030098
:10515800FFF7B2FF504508D142462046FFF7B6FF99
:1051680008F1010709F10109D8E76FF03103D9E720
:1051780021462846FFF7BCFF0028D8D102A92846B7
:10518800FFF7BBFF02ABA2199442D0D014F8015B21
:1051980013F8011B8D42F7D0C7E770B5C02288B05D
:1051A8000E46012190F83051044601F00BFCF0B98D
:1051B80001A92046FFF79CFDC8B90122FF2120461E
:1051C80001F000FC98B93246B621204601F04AFCAD
:1051D80068B90246FF21204601F0F4FB38B92A4697
:1051E8000121204601F0EEFB08B984F8305108B0DF
:1051F80070BDF0B50F4689B01646FF21012204465E
:1052080001F0E0FB0246A8B94F21204601F0DAFB85
:1052180080B92C224E21204601F0D4FB024648B921
:10522800FF21204601F0CEFB20B9B422B62120464A
:1052380001F0C8FB0025C4F82451A4F82851DEB9B0
:10524800354607ABB422CDE903730623CDE9003216
:10525800029504F5927304F5957231462046FFF7DE
:1052680051FF30B9012384F8153184F8137184F89B
:10527800146109B0F0BD013505F1B400FFF71CFF5A
:105288000028DED12C2DF6D1DBE710B541F0010264
:105298000021044601F096FB78B9204600F02AFA6E
:1052A80058B901462046FFF7F7FC30B902460146D7
:1052B8002046BDE8104001F085BB10BD2DE9F74F31
:1052C8004FF0000B88461746FF21012205461E466F
:1052D8009DF838A09DF83C908DF807B001F072FB5E
:1052E8005A4604465946284601F06CFB5A46044380
:1052F800FF21284601F066FB64B2044364B2B8F1AA
:10530800000F32D0BAF1000F06D00C9ACB212846F4
:1053180001F07AFB204344B2B9F1000F07D00DF138
:105328000702EE21284601F06FFB204344B2012218
:10533800FF21284601F046FB0122044300212846AC
:1053480001F040FB64B204430022FF21284601F02B
:1053580039FB64B29DF807300D9A204323F01003FF
:1053680040B2137003B0BDE8F08FBAF1000F06D059
:105378003A46CB21284601F025FB204344B2B9F137
:10538800000FD4D033468022EE21284601F053FB8B
:10539800CBE72DE9F04387B09146002205460E463B
:1053A8008DF817201F4653B390F83081012211461B
:1053B800284601F007FB044648BB40212846FFF772
:1053C80064FFF0B9B9F1010F24D10DF11703CDE94C
:1053D8000294CDE900632246234649462846FFF752
:1053E8006DFF044678B947B142460121284601F0CD
:1053F800E9FA044638B985F83081002403E0984674
:10540800D4E734700446204607B0BDE8F083002393
:105418003370F8E73070E6E72DE9F043054687B0CA
:105428000E4691461F4653B390F83081022201215F
:10543800284601F0C7FA044648BB01462846FFF74C
:1054480024FFF0B9B9F1010F24D10DF11703CDE90B
:105458000249009322462346019649462846FFF70B
:105468002DFF044678B947B142460121284601F08C
:10547800A9FA044638B985F83081002403E0984633
:10548800D4E734700446204607B0BDE8F083002313
:105498003370F8E73070E6E7F8B51D461646002386
:1054A8002A4690F830710446FFF773FF70B9034637
:1054B8002A4631462046FFF7AFFF38B93A46012160
:1054C800204601F07FFA08B984F83071F8BD2DE95B
:1054D800F04F002393B0CDE90A12C0F82431A0F8A8
:1054E80028310122FF21CDE90E33B0F83C818DF837
:1054F800343004468DF8353001F064FA002840F065
:10550800F08002464F21204601F05CFA002840F066
:10551800E8802C224E21204601F054FA002840F061
:10552800E0800246FF21204601F04CFA002840F0B6
:10553800D880B422B621204601F044FA002840F071
:10554800D08002468021204601F03CFA002840F035
:10555800C88003460DF135020DA92046FFF79CFFD0
:10556800002840F0BE8004F5957307930323CDE926
:105578000203B421062304F592790EAECDE9003179
:10558800049601464B4604F595722046FFF7BAFD8E
:10559800002840F0A6800DF1360120460E9DFFF749
:1055A800FCFD002840F09D80BDF83630434541D9C8
:1055B800C4F82401A4F8280105F1B400FFF77CFD24
:1055C80008B92B2D1FD90623B42204960326CDE94A
:1055D8000032CDE90256079A4B4601212046FFF7D3
:1055E80091FD00287DD10DF1360120460E9DFFF773
:1055F800D4FD002875D1BDF83630434574D901274C
:105608004FF0010A19E00135D6E7089E099324E016
:10561800089E0A9B1E600B9B1F70012384F815319E
:105628000A9B1B6884F813310B9B1B7884F8143190
:10563800002056E000273E46BA46BDF836304345BE
:10564800E7D2A3EB080383EAE372A2EBE3725FFA03
:105658008AF70992032604F5927BDBF80000BBF871
:1056680004301090ADF844302A460FAB0798062155
:10567800FFF7FCFC0F9D6B1C39D005F1B400FFF758
:105688001BFD5045C5D1731C2A4648460893FFF7B1
:105698001DFD30BB494620460135FFF729FD00BBFB
:1056A8000DF136012046FFF778FDD0B9BDF8362058
:1056B800A2EB0803002BB8BF5B424245A5D9099A63
:1056C8009342A5D910A92046FFF712FDBDF8442042
:1056D80003461098C4F82401ABF804201846002BA0
:1056E80097D013B0BDE8F08F0746064688E76FF0FD
:1056F8003100F6E737B5002304468DF807304FF43C
:10570800FA650DF107012046FFF779FC58B99DF8B5
:105718000730012B07D0013D03D0204601F0DEF908
:10572800EFE76FF0060003B030BD02464FF080434C
:10573800934202D8002013B970479B08F8E7C118B4
:1057480091424FEA50009CBFC018521A9B08F2E7DA
:1057580073B500228321054601F034F9044690B957
:1057680006460DF107028321284601F04DF99DF800
:1057780007300343DBB204462BB90136B6F5FA6F9E
:10578800EFD16FF0060401228321284601F01AF9AF
:10579800204340B202B070BD2DE9F04F90F8F060A0
:1057A80091B04FF00009072ECDE9079904460F463E
:1057B80000F0A2820122802101F004F90122804632
:1057C800FF21204601F0FEF84A4648EA000849460B
:1057D800204601F0F7F84FFA88F848EA0008062250
:1057E800FF21204601F0EEF84FFA88F848EA000851
:1057F8000DF115028321204601F006F99DF81520C8
:105808004FFA88F848EA000842F00402832120464B
:1058180001F0D8F84FFA88F848EA00080722FF2173
:10582800204601F0CFF84FFA88F80122812148EA92
:105838000008204601F0C6F84FFA88F848EA000840
:10584800204601F04BF94FFA88F848EA000801228F
:105858008021204601F0B6F84FFA88F848EA00059A
:1058680017F0010B6DB200F01E82F20700F11E82E4
:105878006B229421204601F0A5F880462046FFF7C8
:1058880067FF06AA48EA00089021204601F008F9B7
:1058980045EA0805069B6DB224229421054320465B
:1058A800C3F3062AC3F3C03901F08CF86DB205437F
:1058B8002046FFF74DFF6DB2054306AA902120460A
:1058C80001F0EEF8069B6DB21BBA25229421054320
:1058D8002046099301F076F86DB205432046FFF79C
:1058E80037FF6DB2054306AA9021204601F0D8F88B
:1058F800069B6DB21A0E05431B0C6DB28DF828205D
:105908008DF8293017F00203029300F0DB8016F0BF
:10591800020840F0D78002229421204601F052F874
:1059280001902046FFF714FF019B0DF11602034377
:10593800902120461D4301F067F86DB27B22942127
:105948000543204601F03EF86DB205432046FFF7B7
:10595800FFFE6DB205430DF117029021204601F0BC
:1059680053F86DB2772294210543204601F02AF8B6
:105978006DB205432046FFF7EBFE6DB2054306AA5C
:105988009021204601F08CF8069B5A0E8DF82C20A9
:10599800C3F386428DF82D20C3F3C6228DF82E203E
:1059A8006DB2C3F30612DB0003F0780394210543BC
:1059B8008DF82F20204678228DF8153001F002F856
:1059C8006DB205432046FFF7C3FE6DB2054306AA34
:1059D8009021204601F064F8069B9DF8152002EB03
:1059E80053728DF83020C3F386528DF83120C3F3FB
:1059F800C6328DF83220C3F306228DF833206DB2FB
:105A0800C3F346029B0103F04003942105438DF83C
:105A18003420204679228DF8153000F0D3FF6DB27E
:105A280005432046FFF794FE6DB2054306AA902170
:105A3800204601F035F8069B9DF8152002EB93628D
:105A48008DF83520C3F3C6428DF83620C3F30632ED
:105A58008DF837206DB2C3F346129B0003F07C0328
:105A6800942105438DF8382020467A228DF8153088
:105A780000F0A8FF6DB205432046FFF769FE6DB23E
:105A8800054306AA9021204601F00AF8069B9DF8D6
:105A980015208DF83E8002EB93728DF83920C3F300
:105AA800C6526DB28DF83A20C3F3064205438DF80D
:105AB8003B20C3F34622C3F386036DB28DF83C2026
:105AC8008DF83D3017F00403019300F0F18073075F
:105AD80000F1EE807B229421204600F073FF80467F
:105AE8002046FFF735FE07AA48EA0008902120461D
:105AF80000F0D6FF45EA08084FFA88F848EA00059A
:105B08007C229421204600F05DFF6DB205432046BB
:105B1800FFF71EFE6DB2054308AA9021204600F04B
:105B2800BFFF6DB2732294210543204600F04AFF5F
:105B38006DB205432046FFF70BFE6DB2054306AA7A
:105B48009021204600F0ACFF069B6DB21B02742228
:105B58009421054320461FFA83F800F033FF6DB205
:105B680005432046FFF7F4FD6DB2054306AA9021D0
:105B7800204600F095FF6DB29DF81B3075229421E8
:105B88000543204643EA080800F01CFF6DB20543B0
:105B98002046FFF7DDFD6DB2054306AA9021204699
:105BA80000F07EFF069B6DB21B029BB27622942109
:105BB80005432046039300F005FF6DB205432046D8
:105BC800FFF7C6FD6DB2054306AA9021204600F0F6
:105BD80067FF6DB29DF81B20039B05436DB213430D
:105BE800002281212046039300F0ECFE06220543A3
:105BF800FF21204600F0E6FE6DB205430DF11502C7
:105C08008321204600F000FF9DF815206DB2054362
:105C180002F0FB028321204600F0D4FE6DB205435A
:105C28000122FF21204600F0CDFE6DB2054301227E
:105C38000021204600F0C6FE6DB205430022FF2178
:105C4800204600F0BFFE6DB20543002280212046A9
:105C580000F0B8FE6DB205436DB2039BFDB9BBF110
:105C6800000F29D1029AAABB019AAAB1720713D4CC
:105C7800079AC4F81821089AC4F81C214FEA482248
:105C8800C4F820213BB1A3F5C8534FF47A725343AB
:105C98001B095B421BB2E3603E4384F8F060284670
:105CA80011B0BDE8F08FD946DA462BE6CA4629E698
:105CB8004FF00008434693E7F007D3D40998BDF89E
:105CC800282084F813A184F81491C4F82A01A4F8B0
:105CD8002E21C7E7B107C7D49DF8162084F8F12014
:105CE8009DF8172084F8F2200BA904F1F300029321
:105CF8000DF08AFD029BB7E74D46D0E740B1013869
:105D08000023FF2803F1010203D800EB032080B22F
:105D1800704740081346F4E7C3B2000A03FA00F0DC
:105D280001307047084B5A434FF47A7302F5FA7200
:105D38004FF4FA60B2FBF0F0B2FBF3F203FB0100A0
:105D4800B0FBF2F0704700BF002F3A00064B5A43F1
:105D58004FF47A7002F5FA72B2FBF0F24A4302F598
:105D6800FA72B2FBF0F07047002F3A002DE9FF41BC
:105D780002294FF00005074616468DF80350ADF886
:105D880004501CD80DF102022946FEF7C7FB044651
:105D980030B90DF103024621384600F035FE0446BD
:105DA8009DF80300FFF7B8FF81B29DF8022038463E
:105DB800FFF7CCFF3060204604B0BDE8F08103292E
:105DC80018D10DF102022946FEF7A8FB0446002867
:105DD80046D101460DF102023846FEF79FFB044604
:105DE80028B901AA5121384600F03CFE0446BDF806
:105DF8000400D7E7042935D102A9FEF7E4FB9DF892
:105E08000B304BB30DF1020229463846FEF786FBEC
:105E1800044618BB01AA5121384600F023FE044667
:105E2800BDF80400FFF778FF85B2BCB90DF1020296
:105E380001213846FEF772FB044678B90DF10602D7
:105E48007121384600F00EFE0446BDF80600FFF743
:105E580063FF80B2401BA7E71D46E7E70020F9E78C
:105E68002846A7E728462C46A4E7F0B5022985B0BE
:105E7800054616461ED80DF105020021FEF74EFB19
:105E88000446A0B99DF8052031462846FFF74AFF89
:105E980083B2B3F5807F9ABF00F1FF32D2B2FF22FE
:105EA800A5F8D8204621284600F08CFD0446204657
:105EB80005B0F0BD032920D10DF105020021FEF740
:105EC8002DFB9DF80520044631462846FFF72AFF9A
:105ED80080B2FFF713FF0246ADF80600A5F8D80018
:105EE800002CE4D15121284600F07CFD044600280E
:105EF800DDD1C5F8E4600024D9E7042939D102A925
:105F0800FEF761FB9DF80B70B7B10DF1050200219A
:105F18002846FEF703FB04460028C8D10DF1060207
:105F28005121284600F09EFD04460028BFD1BDF847
:105F38000600FFF7F1FE87B20DF1050201212846A0
:105F4800FEF7ECFA04460028B1D19DF80520314649
:105F58002846FFF7E7FE3844FFF7D0FE71210246D6
:105F6800284600F03FFD04460028A0D1C5F8DC60B3
:105F7800C1E76FF003049AE7F0B585B000238DF808
:105F88000330D30705460F46164605D441B9A2F19A
:105F98000C03DAB2062A12D96FF0030005B0F0BD7F
:105FA800012920D1A2F10803DAB2062AF4D8062B77
:105FB80019D8DFE803F03718651886189900062BFA
:105FC80011D8DFE803F0041029102B102D00182237
:105FD8005721284600F0F6FC08225621284600F0F2
:105FE800F1FC0028DAD17408013CE4B2002F00F07B
:105FF8008E80012FD0D101AA04212846FFF7B6FED2
:1060080038B922467021284600F0DCFC002800F050
:10601800B28085F8E060C1E73022D9E74022D7E7AF
:106028005022D5E71022482100F0CCFC0822472155
:10603800284600F0C7FC022204463221284600F018
:10604800C1FC0C2204433021284600F0BBFC64B29A
:1060580004430122FF21284600F0B4FC64B2044343
:1060680064B230223021284600F0ACFC0022044300
:10607800FF21284600F0A6FC64B2204340B2B0E7F6
:106088002822482100F09EFC08224721284600F0DB
:1060980099FC032204463221284600F093FC04436D
:1060A80064B209223021284600F08CFC0122044306
:1060B800FF21284600F086FC64B2044364B2202223
:1060C800D0E73822482100F07DFC082247212846E5
:1060D80000F078FC032204463221284600F072FCC6
:1060E800044364B20822DDE74822114600F06AFC46
:1060F80008224721284600F065FC03220446322185
:10610800284600F05FFC044364B20722CAE702AAEB
:1061180003212846FFF72AFE88B903AA0221284648
:10612800FFF724FE58B922465021284600F04AFCC1
:1061380028B9029A03212846FFF797FE10B185F87F
:10614800E8602BE7039A02212846FFF78EFE85F8C0
:10615800E86000287FF422AF69692846FEF7DAF97B
:1061680000287FF41BAF024601230DF103012846E6
:10617800FFF752F912E7019A04212846FFF775FE46
:1061880085F8E060E5E713B5144629B1012910D078
:106198006FF0030002B010BD0DF10702502100F0AE
:1061A80033FC0028F6D19DF8073001335B002370DB
:1061B800F0E70DF107027021F1E7F0B5002385B093
:1061C8004FF4FA62CDE9002344F61F63994206466C
:1061D8000F4604D86FF00305284605B0F0BD02A9A4
:1061E800FEF7F1F905460028F6D19DF809209DF83B
:1061F800083013439DF80A201343A7F636341BD002
:106208006A4602213046FFF7B1FD00283BD19DF8D0
:1062180008302BB1009B03F24E239C42DAD9E41AD2
:106228009DF80A3023B3009B03F2B223B4EB430F6B
:106238004FEA4302CED9A41A9DF80B305BB101AAEC
:1062480003213046FFF792FD019B03F525739C421D
:10625800C0D9C0B9E41A9DF80C30002BBCD0A4F208
:10626800262204213046FFF700FE77610546B3E792
:106278009DF80930002BDFD0009B03F525739C4265
:10628800A8D9E41AD8E70546A6E770B54FF4FA622C
:1062980086B00023CDE9022340F636330B600C4666
:1062A80004A90646FEF78FF90546002836D19DF861
:1062B80011209DF8103013439DF81220134319D074
:1062C80002AA02213046FFF751FD002840D19DF86F
:1062D80010302BB1029B03F24E2223681344236033
:1062E8009DF81230EBB1029B03F2B222236803EB54
:1062F800420323609DF81330EBB99DF814305BB16D
:1063080001AA04213046FFF731FD019B03F2262242
:10631800236813442360D8B923687361284606B0FC
:1063280070BD9DF81130002BE4D0029B03F5257257
:1063380023681344DDE703AA03213046FFF716FD5F
:10634800039B03F525722368134423600028D4D0E7
:106358000546E3E72DE9F743002406460D462046A7
:1063680015F80480B8F1000F00D010B103B0BDE8F3
:10637800F083671CB8F1FF0F15F8079029D1A71C07
:10638800EB5DB9F1030F36D8DFE809F0020B131BF8
:10639800271D2C44E27802EB0323A6F834313C464F
:1063A800DEE7271D2C44E27802EB0323A6F83631FA
:1063B800F5E7271D2C44E27802EB0323A6F83831D1
:1063C800EDE7271D2C44E27802EB0323A6F83C31C5
:1063D800E5E7B8F1040F0ED802344246291901A89E
:1063E8000DF01FFA434601AA4946304604EB080758
:1063F80000F0B2FAD3E76FF00300D0E773B50023DB
:106408000E4613600DF1070105461446FEF712F912
:1064180040B99DF807302BB1B38A2A6A53438033B9
:106428001B0A236002B070BD13B5CB681360144615
:1064380001AAFFF7E3FF18B92368019A1344236000
:1064480002B010BDF8B5B0F85451D0F858016843FF
:106458008030000A0E464543DDE90717144652B15D
:10646800B60206EB5202B2FBF4F202EB42025243CE
:1064780002F50042140C069A534301F50042120C2F
:1064880006200332B2FBF0F2C2EBC202B2F5803F43
:1064980038BF033103F500433EBFB1FBF0F1C1EB58
:1064A800C10101F500414FEA134334BF090C1B49F0
:1064B80003FB03F338BF494303EB57030B44B3FB18
:1064C800F7F39B03FE2205F120007F33B3FBF2F3C1
:1064D8005C434FF47A7704F5FA748009B4FBF7F457
:1064E8002401FFF722F904F5FA74BC4228BF4FF4DF
:1064F800FA63064629BFB4FBF3F300205B19B4FB2B
:10650800F7F428BFB3FBF4F0FFF70FF9099B8642B5
:1065180094BF1E6018600020F8BD00BF0000F0FFA7
:106528002DE9F04F91B0054607930B6908930F4684
:10653800CB680B9393460FAAFFF776FF0EAA39464E
:106548002846FFF75BFF48BB0F9C95F8E0A0D5F8FD
:10655800DC3005934FF47A7606FB04F101F500412F
:10656800049180340E99099124F0FF010A910F914A
:106578000499D5F8E4300693BAF1080F0CBF02234A
:106588000323090C95F8E820DFF898810C9108D1CD
:10659800079BCBF80080C5F84081186011B0BDE8B2
:1065A800F08F06990D932846FFF7BCFB52460599D4
:1065B80081462846FFF7B6FB0D9B5B490C9A814440
:1065C80003FB09F94FEAC92940F2776309F5FA791B
:1065D800240AB9FBF6F903FB09F909F5FA79B9FBBD
:1065E800F6F909FB04F404F18003089C74430C4099
:1065F800B4FBF2F44D4A1B0A944228BF1446012BFF
:1066080038BF01230C204FF4167258435443FFF748
:106618008CF83B7E3A894FEA400A002B7FD14249E9
:10662800049B0B4003F5FA71414B5A4341F25C233A
:10663800B2FBF3F2099B7343B3F5481F28BF4FF42D
:106648004813A1EB4303B1FBF6F1B3FBF6F31B02CE
:10665800B3FBF1F63602C6F58036564306F500461A
:10666800360C06F5803676087643B60B4FF4487339
:10667800734303F5004304F500401B0C5B43000C17
:1066880000FB0030FFF751F803046422323341F273
:106698008837B3FBF2F340F6B532B3FBFAF302FBEB
:1066A8000377244B9F429CBF42F21073B7FBF3F76A
:1066B800DDE90532134403F5FA734FF47A7A4FF49F
:1066C800FA62B3FBFAF0B3FBF2F202F5C812B2FBBE
:1066D800F0F088BF4FF47047FFF727F8000200F585
:1066E800FA70B0FBFAF0404307FB0700FFF71DF80C
:1066F8000AFB00F0079B404528BF4046CBF8000046
:10670800C5F84001CDE902934FF448730093DDE9E1
:106718000A12019433462846FFF794FE3EE74FF4E9
:106728008036A3E7AE878F020000FFFF666666002B
:106738009A9906000F279F242DE9F04F11F0780F42
:106748008BB018BF4FF2A009C1F3C30B18BF29FAC9
:106758000BF990469A460DF10E024FF000034FF0E8
:106768000001159F8DF80E3004468DF80F308DF816
:1067780010308DF81130ADF81230099314BF09F0BC
:1067880001094FF00109FDF7ADFF9DF80E500646CF
:10679800D5B1002840F09A80149909AB05AA204683
:1067A800FFF7BEFE002840F09380149A099B53819E
:1067B800014606AA2046FDF7CAFF069D25B1059B9E
:1067C8009D422CBF0025012520B904AA022120469C
:1067D800FDF788FF9DF8106026B300287AD107AA34
:1067E80002212046FDF7B3FF88B90122FF21204688
:1067F80000F0E8F858B90DF11202B621204600F071
:1068080031F920B90246FF21204600F0DBF8BDF837
:106818001230079E5B02C4F848311EB19E422CBF5D
:106828000026012628B90DF1110203212046FDF7A3
:1068380059FF9DF8113093B100286CD1BAF1000FBF
:1068480003D04FEA0828B8FBFAFA08AA0321204621
:10685800FDF77DFF089B534594BF0023012320B912
:10686800B9F1000F38D0FF223A703A780AB9149972
:106878004A810DF10F02012120460193FDF732FFF5
:1068880008BB9DF80E20019B002A08BF0125BBF11B
:10689800040F18BF9DF80F2084F82E501ABFB2FAC3
:1068A80082F25209012284F82F209DF81020002A34
:1068B8009DF8112008BF0126002A08BF012384F88B
:1068C800306084F831300BB0BDE8F08F002581E7E7
:1068D80035467FE70026ACE70BF1FF32092A0AD8D4
:1068E800DFE802F0050505090907090B070B052272
:1068F800BAE70422B8E7012E01D10322B4E7BBF1BD
:10690800040F01D0012B01D10222ADE7012D16BFE2
:1069180000233D703B700023A7E707B502F10A0387
:10692800009393B20A4690F86011D0F85C0101F028
:1069380029FB03B05DF804FB13B502F10A0390F8D4
:1069480060410093D0F85C0193B20A4644F001011B
:1069580001F0AEFB02B010BD3F2BF8B50E46054660
:1069680011461C4611D80A4F38461A4600F8016BE2
:106978000CF057FF621C39462846FFF7CEFF002867
:1069880014BF6FF013000020F8BD6FF00300FBE7A1
:10699800940E002073B515468DF8071001220DF1ED
:1069A800070104461E46FFF7B8FF18B16FF0130041
:1069B80002B070BD324629462046FFF7BDFF0028C9
:1069C800F6D0F3E708B5064B19705A70194602223B
:1069D800FFF7A3FF002814BF6FF01300002008BDC5
:1069E800940E002008B5074B1970110A59709A7057
:1069F80019460322FFF791FF002814BF6FF0130018
:106A0800002008BD940E002037B515468DF80710F4
:106A180001220DF107010446FFF77FFF18B16FF05F
:106A2800130003B030BD012229462046FFF784FF3A
:106A38000028F6D0F3E7F7B515460DF1070206462C
:106A48000F461C46FFF7E0FF50B99DF807301D4080
:106A580044EA0502394630468DF80720FFF7B2FFB1
:106A680003B0F0BD73B514468DF8071001220DF17F
:106A780007010546FFF751FF18B16FF0130002B088
:106A880070BD064E022231462846FFF755FF002802
:106A9800F3D133885BBA2380F1E700BF940E00205E
:106AA80073B514468DF8071001220DF1070105464C
:106AB800FFF733FF18B16FF0130002B070BD064E38
:106AC800042231462846FFF737FF0028F3D1336800
:106AD8001BBA2360F1E700BF940E002008B502201E
:106AE800FBF7D2FF002008BD7047000010B5032057
:106AF80000F056FC01F03AFD064B18600F20FBF73A
:106B0800B9FF044618B9FBF741FE204610BD012421
:106B1800FBE700BF280800204FF0E022136923F0AC
:106B28000203136170474FF0E022136943F0020338
:106B380013617047014BD3F8900570470070FF1F31
:106B4800014BD3F8940570470070FF1F014BD3F831
:106B5800980570470070FF1F8068C0F38000704779
:106B6800F7B5002301930446002800F0E980856DFD
:106B780025B9FBF76DF9E56584F8545023689A68E0
:106B8800D00040F1A1809A68D10000F1B480A26DD4
:106B980042F01002A265E26D42F00102E2650125B1
:106BA8001846FFF7D9FFA26D02F01002024340F029
:106BB800C980A26D206922F4817242F00202A265A6
:106BC8009A68D2075DD4226BA67E94F82CC0003A4E
:106BD80018BF01221703D4E902120A43217E42EAB0
:106BE8008132617E42EAC13242EA4632002842EAF4
:106BF8004C02B4BF20F000414FF400113A430A435D
:106C080094F82010012903D1002E76D142F4803265
:106C1800616A21B1A66A01F4E07131430A43D96877
:106C2800E66C21F4FE3121F4FF711143D96094F828
:106C38003C206168012A01F0404C4CEA060609D163
:106C4800D4E910273A433243A66C324342EA0C0295
:106C580042F001061F693E4A3A4032431A6121F068
:106C68000042B2F1804F0CD0B1F1004F09D0394E3B
:106C7800D6F8082701F4701122F470120A43C6F8F6
:106C880008275A69666BA16B22F0070232435A61E2
:106C98005A6922F0700242EA01125A61002835D17D
:106CA8009A6A62F00F029A625B6903F007039E42D8
:106CB8003CD10023E365A36D23F0030343F00103F4
:106CC800A365284603B0F0BD9A68234922F0104214
:106CD80022F0170242F080529A60204A1268B2FBF2
:106CE800F1F2013252000192019A002A3FF44BAFAF
:106CF800019A013AF7E7002552E7A16D41F020011A
:106D0800A165E16D41F00101E16581E7B0F5001F82
:106D1800CAD19A6AE269013A92006FF00F0102F053
:106D28001C0201FA02F2216E0A43BCE7A36D23F0AC
:106D3800120343F01003A365E36D43F00103E36519
:106D48000125BEE7A36D43F01003A365F8E700BF74
:106D580002FCFF1F00200140400D0300280800200E
:106D6800F8B54569082D04460E460AD00368DB6865
:106D7800D80705D5A36D43F02003A3650120F8BD0E
:106D88000425FBF779FE074623681A682A4220D0B3
:106D9800A26D42F40072A265DA6812F4406F14D151
:106DA800A27E92B91A6812070FD51846FFF7D4FECB
:106DB80020BB5A6822F00C025A60A26D22F480723D
:106DC80022F0010242F00102A265227EFAB10020FF
:106DD800D5E7711CD9D0FBF74FFEC01BB04201D8D4
:106DE800002ED1D123681B682B40CDD1A26D84F829
:106DF800543042F00402A2650320C0E7A26D42F0BD
:106E08002002A265E26D42F00102E265DDE70C2294
:106E18001A60DCE70368186C70470000F7B50023B8
:106E2800019390F85430012B044600F0C0800568A7
:106E38000269012380F854302846FFF78DFE0028A8
:106E480040F0AF80D1E90030022822F004027ED061
:106E5800B2F1004FC3F3110E35D1AA6A42EA0E020D
:106E6800AA628A68686902EA032222F07C4222F058
:106E7800FF0220EA03210A43002B6A611DDA4D4A0A
:106E88004D4DD2F80817AB4201F0E07043D10D0226
:106E980013D4D2F8083723F0E073034343F4000314
:106EA800C2F80837454B1A68454BB2FBF3F20C237E
:106EB80002FB03330193019B53BB0020002384F89A
:106EC800543003B0F0BD226E00F01F074FF00F0CD6
:106ED8000CFA07FC6FEA0C0622EA0C0CBEF1000F54
:106EE80011D1C3F38462BA4042EA0C0222668008D8
:106EF800E26901309042B4D8A86AC3F38362BA4009
:106F080006403243ACE793FAA3F2B2FA82F2EAE718
:106F1800019B013BCEE72B4DAB420BD1C901CCD431
:106F2800D2F8083723F0E073034343F08073C2F8C4
:106F38000837C2E7244DAB42BFD14B02BDD4D2F8CB
:106F4800083723F0E073034343F48003EFE7B2F11B
:106F5800004F01BFAA6AC3F311018A43AA62002B3A
:106F6800ABDA154813498342D1F8082709D1D1F87B
:106F7800083702F0A07223F0E0731A43C1F808271B
:106F88009BE71048834204D1D1F8083702F4400245
:106F9800F1E70D48834290D1D1F8083702F0C0726A
:106FA800E9E7A26D42F02002A265184686E70220B2
:106FB80087E700BF00200140001000B0280800202B
:106FC800400D0300004000B8002000B4026838B546
:106FD80004461046FFF7C0FD08B9002038BD936885
:106FE800990707D4936823F0004323F0170343F06D
:106FF80010039360FBF740FD054623689B685B0719
:10700800EBD5FBF739FD401B0228F6D923689B68AE
:107018005A07F2D5A36D43F01003A365E36D43F05F
:107028000103E3650120D9E773B5002302680193E2
:107038009368DD07044602D5002002B070BD916850
:10704800214B194209D0A36D43F01003A365E36DEA
:1070580043F00103E3650120EFE7936823F0004361
:1070680023F0170343F001039360184BD3F8083754
:1070780018021CD4637E012BDED0FBF7FDFC144EF6
:10708800054622681368DB07D6D49368D9075FBF23
:107098009368334043F001039360FBF7EDFC401B1A
:1070A8000228EED923681B68DA07EAD4CBE7094B34
:1070B800094A1B68B3FBF2F301330193019B002BD0
:1070C800D8D0019B013BF8E7170000800020014061
:1070D800E8FFFF7F28080020400D030038B504466C
:1070E8000068FFF739FD054620BB94F85430012BA2
:1070F80020D0012384F854302046FFF795FFB0B91B
:10710800A36D226823F4706323F0010343F48073B2
:10711800A3651C23E065136084F85400936823F08A
:10712800004323F0170343F00403936038BD84F849
:107138005450FBE70220F9E7026838B59368916874
:107148000446C80701D4002038BD9907FBD49368CA
:1071580003F00503012B19D1936823F0004323F0B2
:10716800170343F00203936003231360FBF784FCC7
:10717800054623689B68DB07E5D5FBF77DFC401BCC
:107188000228F6D923689B68DA07F2D5A36D43F085
:107198001003A365E36D43F00103E3650120D3E722
:1071A80070B5044600284BD0836D43F00203836515
:1071B800FFF70CFF054668B92046FFF7BDFF0546F7
:1071C80008B90123A3652268936823F0104323F0CC
:1071D8001703936023685A6822F4677222F0030247
:1071E8005A6040F29F321A60D968164A0A40DA603B
:1071F8001A6922F040421A615A6922F007025A615C
:107208001A6A02F0F0221A625A6A02F0F0225A62EE
:10721800DA6A02F0F022DA629A6A0B4A00269E6263
:10722800D2F8083723F0FE73C2F808372046FAF779
:1072380023FEE6652666A66584F85460284670BD78
:107248000125FBE700023E830020014010B590F8BD
:107258005430012B044615D0012380F85430FFF731
:10726800B5FE58B92046FFF767FF38B9A36D23F478
:10727800807323F0010343F00103A365002384F81E
:10728800543010BD0220FCE7F7B50023019390F8B5
:107298005430012B04467FD0012380F85430FFF787
:1072A8004BFF23689A6812F00102054607D0A36DC8
:1072B80043F01003A365002384F854302DE0A16D3A
:1072C800364F21F4817141F00201A165DE68D96869
:1072D80026F4FF4626F07C0621F40041360421F00E
:1072E8000301360CD96008209968394041F0004103
:1072F80099609968002913DA01990131019101997E
:10730800B1F52E3FF5D3A36D23F0120343F010031C
:10731800A365002384F854300125284603B0F0BD46
:10732800D3F8B410013801F07F010A44DCD1996820
:107338001A48014041F001019960D3F8B41021F0D6
:107348007F0141EAD202C3F8B4209A68024042F0B1
:1073580002029A60FBF790FB074623689A68D207F7
:1073680008D4DA683243DA60A36D23F0030343F0EC
:1073780001039FE7FBF780FBC01B0228EDD92368B8
:107388009B68D907E9D5A36D43F01003A365E36DA6
:1073980043F00103E365BFE70225BEE7E8FFFF7F8F
:1073A8000749CA6822F4E0620302120403F4E063A6
:1073B800120C134343F0BF6343F40033CB607047B0
:1073C80000ED00E0164B30B5DC68C4F30224C4F1CC
:1073D8000703251D042B28BF0423062D4FF0FF3576
:1073E8008CBF033C002405FA03F321EA0303A540FC
:1073F80022EA0502A340002843EA0203ACBF00F1D9
:107408006040084A4FEA0313B8BF00F00F00DBB230
:10741800AABF00F56140135480F8003330BD00BFA7
:1074280000ED00E014ED00E0002807DB044A410904
:10743800012300F01F00834042F82130704700BF4D
:1074480000E100E000280CDB4309064900F01F00BA
:1074580020330122824041F82320BFF34F8FBFF32E
:107468006F8F704700E100E070B5D0E913456560A3
:10747800446D14B1D0E916456560D0E9105404F0A4
:107488001C060124B4406C60046863608368102B98
:107498000BBFA260A160E160E26070BD0268416C50
:1074A800D3B210B5083B1424B3FBF4F30B4CA2423F
:1074B80088BF0B4A21F0030199BF01F1804202F510
:1074C8000232521807338264064AC26403F01F036B
:1074D800012202FA03F3036510BD00BF070402404E
:1074E8001C0802408008024038B500285CD00268B9
:1074F8002E4B9A424FF014014AD82D4B1344B3FB3C
:10750800F1F32C499B00C0E91013022380F82530C1
:107518001368056923F4FF4323F070031360D0E96F
:10752800024323432B43456911682B4385692B4349
:10753800C5692B43056A2B430B431360FFF7AEFF66
:10754800B4F5804F04BF002343604368816C03F0A7
:107558007F020A60D0E91314013B032B4C601ED84C
:10756800154B1649816513449B000121013A01FA24
:1075780002F200214365C2651960114B5A64002369
:107588000122C36380F8243080F82520184638BDCE
:107598000C4B1344B3FBF1F30B499B00B3E70023F7
:1075A800C0E91533C365EAE70120F0E707040240A4
:1075B800F8FFFDBF000002403F8200104009024072
:1075C80000090240F8FBFDBF0004024038B500285E
:1075D80041D00268136823F0010313601F4B9A42DD
:1075E8004FF0140130D81E4B1344B3FBF1F31D497F
:1075F8009B00C0E91013012403F01C0304FA03F3F1
:10760800002515604B60FFF749FF836C41681D60DA
:10761800D0E913325A604A1E032A06D8124B0B448B
:107628009B0094401D60114B5C640023C363C0E958
:107638001533C0E90B33C0E90D33C36580F8253035
:1076480080F82430184638BD094B1344B3FBF1F3D6
:1076580008499B00CDE70120F5E700BF0704024079
:10766800F8FFFDBF000002403F8200100009024001
:10767800F8FBFDBF0004024070B590F82450012DBE
:1076880004463BD090F825600125AE4280F824508E
:107698004FF000062CD1022580F825500568C663F6
:1076A8002E6826F001062E60FFF7DEFE036BBBB1E5
:1076B8002B6843F00E032B60A36C1A68D20342BFF9
:1076C8001A6842F480721A60636D1BB11A6842F43A
:1076D80080721A602B6843F001032B60002070BD94
:1076E8002B6823F004032B602B6843F00A03E2E7BE
:1076F8008023C36380F824602846F0E70220EEE781
:1077080070B4426C046C036826681D6802F01C02A1
:107718000421914031420FD015F0040F0CD01A68A3
:1077280092065EBF1A6822F004021A60036B616059
:10773800002B33D070BC184702219140314217D03A
:1077480015F0020F14D01A68940606D41A6822F0AD
:107758000A021A60012280F82520114A93428CBF40
:10776800104B114B5960002380F82430C36ADFE7BF
:1077780008219140314211D029070FD5196821F00D
:107788000E011960012303FA02F26260C36380F8F4
:107798002530002380F82430436BC9E770BC70475C
:1077A8008000024000040240000002400A4A536977
:1077B80043F4802330B55361EFF3108472B600238D
:1077C800CD58C5500433B3F5807FF9D11369DB0375
:1077D800FCD484F3108830BD00400058064B5A6929
:1077E800002ABFBF054A9A6002F188329A60BABF80
:1077F8005869C00F002070470040005823016745B2
:10780800044B5A6942F000425A615869C043C00F9C
:10781800704700BF0040005870B50546FBF72CF9CB
:10782800124E04463369D90313D43369DA0744BFC7
:10783800012232614CF2FA32134011D10B4E3069F9
:1078480010F480200BD0FBF717F9001BA842F6D3E1
:1078580004E0FBF711F9001BA842E3D3032070BD35
:10786800024A1361024A01205360F8E700400058B9
:10787800D40E00202DE9F041184D98462B78012BA5
:1078880006460C46174626D001232B704FF47A7013
:1078980000236B60FFF7C0FFA0B9012E16D1104A74
:1078A800536943F0010353612760BFF36F8FC4F836
:1078B80004804FF47A70FFF7AFFF094A536923EA4F
:1078C8000603536100232B70BDE8F081394620463A
:1078D800FFF76CFFEDE70220F6E700BFD40E0020AB
:1078E80000400058054A536923F47E7343EAC000F8
:1078F80040F4803040F0020050617047004000586A
:107908002DE9F041234F3B78012B054688463FD0AF
:1079180001233B704FF47A7000237B60FFF77CFFF4
:10792800044688B92B68042B13D11B4A536943F4C6
:10793800803343F0040353614FF47A70FFF76CFF10
:107948000446154B1A681B6800233B702046BDE8A7
:10795800F0814FF0FF33C8F800306E68D5E9013286
:107968001344B3420AD93046FFF7BCFF4FF47A708C
:10797800FFF752FF50B1C8F800600446064A536941
:1079880023F47E7323F002035361DAE70136E5E757
:107998000224DBE7D40E0020004000582DE9F04F08
:1079A800524C00234FF00F090A6832FA03F501D14F
:1079B800BDE8F08F012505FA03F818EA020200F085
:1079C8008E804E68032706F003054FEA430E07FA38
:1079D8000EFC6F1E012F6FEA0C0C32D8876807EA7D
:1079E8000C0ACF6807FA0EF747EA0A078760476864
:1079F80027EA0808C6F300179F4047EA08074760C8
:107A0800C76807EA0C088F6807FA0EF747EA0807FD
:107A1800022DC76017D14FEAD30800EB880803F09E
:107A2800070AD8F820704FEA8A0A09FA0AFB27EAF7
:107A38000B0B0F6907FA0AF747EA0B07C8F820701B
:107A480001E0032DDCD1076805FA0EF507EA0C07FB
:107A58003D4316F4403F056041D023F0030707F18A
:107A6800804707F5803703F0030CBD684FEA8C0C9C
:107A78004FF0070E0EFA0CFEB0F1904F25EA0E0EED
:107A88002FD01B4DA8422ED005F58065A84214BF03
:107A98000725022505FA0CF545EA0E05BD6025689F
:107AA800D74316F4801F0CBF3D4015432560656819
:107AB80016F4001F0CBF3D4015436560D4F8805094
:107AC80016F4803F0CBF3D401543C4F88050D4F8ED
:107AD8008450B60354BF3D401543C4F88450013365
:107AE80062E70025D6E70125D4E700BF0008005863
:107AF80000040048374A2DE9F04F00234FF0010AEF
:107B08004FF0070B4FF00F0931FA03F401D1BDE82C
:107B1800F08F0AFA03FC1CEA010654D023F0030490
:107B280004F1804404F5803403F00307A568BF001E
:107B38000BFA07F8B0F1904F08EA050E45D0264D2C
:107B4800A84244D005F58065A8420CBF0225072548
:107B5800BD40754517D1D2F8805025EA0605C2F810
:107B68008050D2F8845025EA0605C2F8845015687A
:107B780025EA06051560556825EA06055560A568D5
:107B880025EA0805A560056803265C0006FA04F4E2
:107B980023FA06F6254300EB8606056003F0070581
:107BA800376AAD0009FA05F527EA050737628568DF
:107BB80025EA04058560456825EA0C054560C56821
:107BC80025EA0404C46001339EE70025C0E70125C7
:107BD800BEE700BF000800580004004803691942C6
:107BE80014BF0120002070470AB18161704781628B
:107BF8007047436901EA030221EA030141EA0241AD
:107C080081617047044AD168014208B502D0D0604A
:107C1800FBF7B8FB08BD00BF0008005803689A6965
:107C2800910744BF00229A629A69D2075EBF9A6997
:107C380042F001029A61704730B5039D04682B43F6
:107C480043EA0243064A6068C1F309010B4342EA6A
:107C5800555223F0004320EA02000343636030BD1D
:107C6800FF63FF0303682DE9F0419C6914F01004D9
:107C780005460F4616466FD010220024DA61A0464A
:107C88002B689A69900661D4B8F1000F35D044F09A
:107C9800040401202E68B369D90541BF4FF48072EE
:107CA800F26144F0010401205A0541BF4FF480629B
:107CB80044F00804F26101209B054FD54FF400738E
:107CC80044F00204F3612846FFF7A8FF736823F025
:107CD800FF7323F48B3323F4FF7323F001037360E2
:107CE8006B6C23436B64202385F84130002385F8AF
:107CF800423085F84030012032E07A1CC1D0FAF7D2
:107D0800BBFE801BB84201D8002FB9D12B68596837
:107D180095F8422098690004D2B20AD5490408D4DB
:107D2800202A06D05A6842F480425A60FAF7A4FE24
:107D380006462B689B699B06A2D4FAF79DFE801B1A
:107D48001928F6D920244FF0010899E7B8F1000F57
:107D58009DD12022DA619AE720469BE70028B2D11C
:107D6800BDE8F08170B504460D46164623689B6948
:107D78009B0701D500201BE0324629462046FFF725
:107D880071FFA0B96A1CF1D0FAF776FE801BA842F1
:107D980001D8002DEAD1636C43F0200363642023EB
:107DA80084F84130002384F8423084F840300120C0
:107DB80070BD70B504460D46164623689B699B0640
:107DC80001D5002019E0324629462046FFF74AFF30
:107DD80090B9FAF751FE801BA84201D8002DECD1CA
:107DE800636C43F020036364202384F8413000234C
:107DF80084F8423084F84030012070BD70B50446E4
:107E08000D46164623689B695B070ED43246294601
:107E18002046FFF727FF38BB23689A69910625D5C6
:107E28009A69520703D5228D0AB1002070BD9A695C
:107E380012F010021CBF1022DA614FF0200118BFA7
:107E480004226264D9615A6822F0FF7222F48B32EC
:107E580022F4FF7222F001025A60002384F84110D4
:107E680084F8423084F840300120DFE7FAF704FE56
:107E7800801BA84201D8002DC4D1636C43F02003B5
:107E88006364202384F841300023EBE72DE9F041B7
:107E9800069F0446884616461D462268936938EAB6
:107EA80003030CBF01230023B34201D0002015E0D7
:107EB8006B1CF3D0FAF7E0FDC01BA84201D8002DD7
:107EC800EBD1636C43F020036364202384F84130D2
:107ED800002384F8423084F840300120BDE8F08166
:107EE80010B5044600284AD090F8413003F0FF024C
:107EF8001BB980F84020FAF7B3FA242384F84130FC
:107F080023681A6822F001021A60626822F070621F
:107F18001A619A6822F400429A60D4E90221012980
:107F280024D142F400429A605A6842F0007242F446
:107F380000425A60DA6822F40042DA60D4E9042187
:107F48000A43A16942EA0122DA60D4E907210A4317
:107F58001A601A6842F001021A6000202023606447
:107F680084F84130206384F8420010BD42F4044292
:107F780002299A6004BF4FF400625A60D4E70120D6
:107F8800F3E700002DE9F347984690F841300A9F3F
:107F9800202B04460E46914640F0868090F84030EB
:107FA800012B00F081804FF0010A80F840A0FAF719
:107FB80063FD19230546009052464FF400412046C0
:107FC800FFF764FF18B1012002B0BDE8F087212354
:107FD80084F84130102384F842306064A4F82A8081
:107FE800638DC4F824909BB2FF2B60632F4B26D976
:107FF800FF22228500934FF0807331462046FFF719
:108008001BFE638D9BB22A4639462046FBB9FFF713
:10801800D0FE0028D7D123682021D9615A6822F0E0
:10802800FF7222F48B3222F4FF7222F001025A60AE
:1080380084F8411084F8400084F84200C4E7628D57
:1080480092B2228500934FF00073D2B2D5E7FFF7C2
:1080580089FE0028B7D1636A226813F8011B916270
:108068006362638D228D013B9BB26385638D013A08
:1080780092B29BB22285002BC3D0002AC1D10095B1
:108088003B4680212046FFF701FF00289BD1638DE6
:108098009BB2FF2B03D9FF2222850090ABE7628DAC
:1080A80092B222850090CEE702208DE70020008062
:1080B8002DE9F347984690F841300A9F202B044653
:1080C8000E46914640F0878090F84030012B00F032
:1080D80082804FF0010A80F840A0FAF7CDFC1923FE
:1080E8000546009052464FF400412046FFF7CEFE69
:1080F80018B1012002B0BDE8F087222384F841308E
:10810800102384F842306064A4F82A80638DC4F890
:1081180024909BB2FF2B6063304B26D9FF22228527
:1081280000934FF0807331462046FFF785FD638D3D
:108138009BB22A4639462046FBB9FFF73AFE00288B
:10814800D7D123682021D9615A6822F0FF7222F41E
:108158008B3222F4FF7222F001025A6084F8411037
:1081680084F8400084F84200C4E7628D92B2228508
:1081780000934FF00073D2B2D5E7FFF73FFE002817
:10818800B7D123685A6A636A1A70636A228D013309
:108198006362638D013B9BB26385638D013A92B242
:1081A8009BB22285002BC2D0002AC0D100953B4645
:1081B80080212046FFF76AFE00289AD1638D9BB282
:1081C800FF2B03D9FF2222850090AAE7628D92B285
:1081D80022850090CDE702208CE700BF00240080B4
:1081E80010B590F84120202A0346D4B21CD190F84B
:1081F8004020012A18D0242280F841200268106803
:1082080020F001001060106820F4805010601068A1
:10821800014311601168002041F00101116083F8E9
:10822800414083F8400010BD0220FCE710B590F8EB
:108238004120202A0346D4B21BD190F84020012ABD
:1082480017D0242280F841200268106820F001002D
:108258001060106820F4706040EA01211160116814
:10826800002041F00101116083F8414083F840008B
:1082780010BD0220FCE70000024A136843F4807333
:1082880013607047000400580D4B10B55B690C462D
:1082980028B99A0507D500F039F820B110BD9B051B
:1082A80001D400F02BF8074A1369012C23F00403CA
:1082B800136101D130BFF1E740BF20BF20BFEDE718
:1082C8000004005800ED00E0064A136823F0070395
:1082D80043F003031360044A136943F00403136172
:1082E80030BF70470004005800ED00E0024B1868EA
:1082F80000F4C060704700BF00040058024A1368C9
:1083080043F4804313607047000400580C4A136814
:1083180023F4804313600B4B1B6832214B430A49FB
:10832800B3FBF1F35169890500D533B9536913F4E7
:10833800007F14BF032000207047013BF2E700BF15
:10834800000400582808002040420F000B4A136818
:1083580023F0070343F002031360094B1A6901284D
:1083680042F004021A6105D130BF1A6922F00402F2
:108378001A61704740BF20BF20BFF6E700040058CD
:1083880000ED00E04FF0B0431868C0F3404070477C
:108398004FF0B0431868C0F3400070474FF0B04248
:1083A800536823F47F4343EA0023536070474FF038
:1083B800B0431868C0F34060704700007FB54FF0C5
:1083C800B0432C4AD3F80831C0F3031003F00F036D
:1083D80052F82040284A52F82330B4FBF3F4FFF750
:1083E80085FF264B054693E80700B5F5007F04ABEB
:1083F80003E9070010D0224B9C4218D303F5B703BA
:1084080003F67F539C4229D903F5741303F51063CF
:108418009C4225D802230BE01A4B9C4207D91A4BE1
:108428009C421BD903F5370303F5D853F0E7002323
:1084380004AA02EB830353F80C4C144D2B6823F069
:10844800070323432B60FAF717FB06462B6803F054
:1084580007039C4206D1002004B070BD0123E7E762
:108468000024EAE7FAF708FB801B0228EED903206C
:10847800F2E700BFC03A0108203B0108683901084B
:10848800C0CF6A00BFEA21013F9334020040005880
:108498004FF0B04310B59A68D96812F00C0205D0B5
:1084A8000C2A4AD101F00303012B51D14FF0B041FE
:1084B8002B480B6813F0080306D00B6813F0080369
:1084C80037D1D1F8941007E00C68240756BFD1F8CB
:1084D80094300968C3F3032350F82330002A0CBFF3
:1084E800184600204FF0B0418A6802F00C020C2AAE
:1084F8001ED1CA6802F00302022A2ED0032A06D12E
:108508000B68184A13F4801F174B18BF13464FF017
:10851800B042D068D168D268C0F306205843C1F38E
:1085280002130133B0FBF3F0530F0133B0FBF3F048
:1085380010BD0B68C3F30313CEE7042A05D0082A3D
:1085480006D11B6813F4801305D006480023C9E739
:1085580000231846C6E70448C4E7024BD7E700BF24
:10856800C03A01080024F4000048E80108B5FFF704
:108578008FFF4FF0B043044A9B68C3F3031352F8CC
:108588002330B0FBF3F008BD203B01082DE9F04192
:108598000446002853D04FF0B0439D68DE68036856
:1085A8009B0605F00C0506F0030668D5026A1DB1A6
:1085B8000C2D46D1012E44D1002A40D04FF0B043B3
:1085C800A16A1A68170756BFD3F894301B681B09AD
:1085D80003F0F00399421FD90846FFF7EFFE002881
:1085E8002DD14FF0B042136843F0080313601368AD
:1085F800A16A23F0F0030B431360606AFFF7CEFE15
:10860800FFF7B4FFAB4B1860AB4B1868FAF732FAB8
:10861800002834D0BDE8F0814FF0B042136843F031
:1086280008031360136823F0F0030B431360606AB8
:10863800FFF7B4FE0846FFF7C1FE0028E0D001208E
:10864800E8E74FF0B043002A54D01A6842F001021C
:108658001A60FAF711FA0746FFF79AFE002842D087
:108668004FF0B042136843F0080313601368A16A1F
:1086780023F0F0030B431360606AFFF78FFE236853
:10868800D80748D42368990700F18C8023681E070F
:1086980040F1FA80A3694FF0B046002B00F0E1806A
:1086A800D6F89430E16903F01002914200F0C480DA
:1086B80003F00302022AC2D0D80740F1B380D6F8EB
:1086C800943023F00103C6F89430FAF7D5F9074639
:1086D800D6F89430990740F1A580FAF7CDF9C31B75
:1086E800112BF5D904E0FAF7C7F9C01B0228B3D952
:1086F80003208FE71A6822F001021A60FAF7BCF922
:108708000746FFF745FE0028B9D0FAF7B5F9C01BB0
:108718000228F6D9ECE7082D03D00C2D05D1032E3D
:1087280003D16368002BADD189E74FF0B043A1684E
:108738001A6822F480120A431A606268B2F5803F10
:1087480010D11A6842F480321A60FAF795F9074690
:10875800FFF718FE002895D1FAF78EF9C01B642898
:10876800F6D9C5E7B2F5041F04D11A6842F400121D
:108778001A60E6E7196821F480311960196821F454
:1087880000111960002AE0D1FAF776F90746FFF7D9
:10879800F9FD00283FF476AFFAF76EF9C01B64289C
:1087A800F5D9A5E7042D236903D00C2D0ED1022E8F
:1087B8000CD1002B3FF443AF4FF0B04261695368CE
:1087C80023F0FE4343EA016353605FE74FF0B0468E
:1087D800BBB1336843F480733360FAF74DF9074649
:1087E80033685A0505D4FAF747F9C31B022BF7D9A2
:1087F8007EE77368626923F0FE4343EA02637360AD
:1088080044E7336823F480733360FAF735F9074691
:1088180033685B057FF53AAFFAF72EF9C31B022BD5
:10882800F6D965E74FF0B042E169D2F8943023F009
:1088380010030B43C2F894304FF0B047D7F8943088
:1088480043F00103C7F89430FAF716F90646D7F84B
:1088580094309A0718D4FAF70FF9831B112BF6D91D
:1088680046E7D6F8943023F00103C6F89430FAF7B7
:1088780003F90746D6F894309B0705D5FAF7FCF8B4
:10888800C31B112BF6D933E72368580754D50B4F70
:108898003B68D90514D4FFF7EFFCFAF7EDF8064664
:1088A8003B68DA050CD4FAF7E7F8831B022BF7D9F3
:1088B8001EE700BF280800202C08002000040058EC
:1088C800E3684FF0B046002B58D023F08003052B07
:1088D80002BFD6F8903043F00403C6F890304FF04A
:1088E800B046FAF7C9F8D6F8903043F001030746C6
:1088F800C6F8903041F28838D6F890309B0705D4F6
:10890800FAF7BAF8C31B4345F6D9F1E6E36823F052
:108918000403812B1BD1FAF7AFF8D6F8903043F057
:108928008003C6F8903007464FF0B04641F28838C9
:10893800D6F89030180504D5E36A002B4AD10020F8
:1089480068E6FAF799F8C01B4045F1D9D0E6FAF77E
:1089580093F8D6F8903023F08003C6F89030074695
:108968004FF0B04641F28838D6F890301905E3D573
:10897800FAF782F8C01B4045F6D9B9E6FAF77CF851
:10898800D6F8903023F080030746C6F8903041F2BD
:108998008838D6F890301A0516D4FAF76DF8D6F854
:1089A800903023F00103C6F8903007464FF0B048E6
:1089B80041F28836D8F890309B07BDD5FAF75CF8B5
:1089C800C31BB342F6D993E6FAF756F8C01B4045E5
:1089D800DFD98DE60C2D4ED0022B4FF0B0431A682C
:1089E80022F080721A6033D1FAF746F80546FFF78D
:1089F800DEFC38BBD4E90C314FF0B0420B43D068F1
:108A08002D4901400B43E16B0B43216C0B43616C17
:108A18000B43A16B43EA0123D360136843F08073CF
:108A28001360D36843F08053D360FAF725F80446FF
:108A3800FFF7BDFC002882D1FAF71EF8001B0A28B0
:108A4800F6D955E6FAF718F8401B0A28CFD94FE6A9
:108A5800FAF712F80446FFF7AAFC30B94FF0B04213
:108A6800164BD1680B40D36069E7FAF705F8001B8D
:108A78000A28F0D93CE6012B3FF4E1AD4FF0B043B2
:108A8800D868236B00F003029A427FF4D8AD626B7A
:108A980000F0700393427FF4D2ADA26B00F4FE4362
:108AA800B3EB022F7FF4CBAD636C00F06040C01ACB
:108AB80018BF0120AEE500BF8C80C111FCFFFEEE9F
:108AC8002DE9F0410D46044610B90120BDE8F081BA
:108AD800684E336803F007038B4216D323689A075E
:108AE80027D54FF0B047A268BB6823F0F0031343C3
:108AF800BB60F9F7C1FF0646BB68DB0319D4F9F779
:108B0800BBFF831B022BF7D911E0336823F007035F
:108B18000B433360F9F7B0FF0746336803F00703E8
:108B2800AB42DBD0F9F7A8FFC01B0228F5D9032018
:108B3800CCE72368580617D54FF0B0476269D7F8D5
:108B4800083123F00F0343EA1213C7F80831F9F785
:108B580093FF0646D7F80831D90305D4F9F78CFFF7
:108B6800831B022BF6D9E2E723685A0713D54FF087
:108B7800B047E268BB6823F4E0631343BB60F9F7CE
:108B88007BFF0646BB689B0305D4F9F775FF831B7B
:108B9800022BF7D9CBE72368180714D54FF0B04755
:108BA8002269BB6823F4605343EAC203BB60F9F748
:108BB80063FF0646BB68590305D4F9F75DFF831BBD
:108BC800022BF7D9B3E72368DA070FD4294C2368B7
:108BD80003F00703AB4239D8FFF7C8FC264B1860EF
:108BE800264BBDE8F0411868F9F744BF6268022ACD
:108BF8001DD1FFF7C7FB00283FF467AF4FF0B04621
:108C080041F28838B36823F003031343B360F9F7DC
:108C180033FF0746B368626803F00C03B3EB820FB7
:108C2800D4D0F9F729FFC01B4045F3D97FE7032AC1
:108C380002D1FFF7BCFBDEE712B9FFF7A9FBDAE7C1
:108C48004FF0B0431B685B05D8D43EE7236823F098
:108C580007032B432360F9F70FFF0646236803F049
:108C68000703AB42B8D0F9F707FF801B0228F5D9F4
:108C78005DE700BF00400058280800202C080020AD
:108C880008B5FFF773FC4FF0B043044A9B68C3F381
:108C9800022352F82330D84008BD00BF003B01082A
:108CA80008B5FFF763FC4FF0B043044A9B68C3F371
:108CB800C22352F82330D84008BD00BF003B01084A
:108CC8004FF0B043D3F89000C0F3400070474FF026
:108CD800B0410209D1F8883002F47F22000123EA6A
:108CE800020300F47F200343C1F8883070474FF037
:108CF800B041020CD1F88830120423EA020343EA97
:108D08000040C1F8880070470368DA0370B504466C
:108D180039D5FFF7B1FAF9F7AFFE614E054633686A
:108D2800DB0532D54FF0B043616BD3F8902002F4E5
:108D3800407291421DD0D3F89010D3F8902042F49D
:108D48008032C3F89020D3F8902021F4407022F4A8
:108D580080328D07C3F89020C3F8900009D5F9F741
:108D68008BFE41F288360546FFF7AAFF012840F03E
:108D780090804FF0B042616BD2F8903023F440738A
:108D88000B43C2F89030002605E0F9F775FE401B4A
:108D98000228C4D903262568E8070AD54FF0B04150
:108DA8006268D1F8883023EA124392B21343C1F8BB
:108DB8008830A9070AD54FF0B041A268D1F88830A9
:108DC80023EA124392B21343C1F88830AA0609D5A0
:108DD8004FF0B0422169D2F8883023F440630B4346
:108DE800C2F88830AB0502D5206AFFF780FF680516
:108DF80002D5606AFFF77BFF290502D5A06AFFF755
:108E080076FF6A0602D56069FFF761FF2B0602D577
:108E1800A069FFF75CFFE80502D5E069FFF757FF97
:108E2800E90610D54FF0B042E168D2F8883023F453
:108E380040730B43C2F88830B1F5807F02BFD36816
:108E480043F08073D3602A040ED54FF0B042216BF3
:108E5800D2F8883023F040430B43C2F8883019B960
:108E6800D36843F08073D3606B0410D54FF0B042E1
:108E7800E16AD2F8883023F040530B43B1F1005F28
:108E8800C2F8883003D1D36843F48033D3603046C6
:108E980070BDF9F7F1FD401BB0427FF665AF79E789
:108EA8000004005830B590F82C30012B02464FF0E2
:108EB800020022D0174B82F82D00CA24012582F81F
:108EC8002C505C6253245C62B1F5807F146B996905
:108ED80014D121F488519961596C24F0010421F0CE
:108EE800004159641463DD650A4BFF215962002073
:108EF800012382F82D3082F82C0030BD21F408516E
:108F08009961D96C24F0020421F00041D9641463FA
:108F1800D865E9E70028004070B50B4E036B756D06
:108F28001D40EA07044603D50123F365F9F7B7FEA8
:108F3800AB0704D50223F365204600F0C9F90123E5
:108F480084F82D3070BD00BF0028004038B50A4CA9
:108F5800E36823F02003E360F9F78EFD0546E36834
:108F68009B0601D5002038BDF9F786FD401BB0F5FA
:108F78007A7FF4D90320F6E700280040F8B5114DB0
:108F8800EC6814F0400406461AD1EB6843F08003FD
:108F9800EB60F9F771FD23460746EC6814F04004CE
:108FA80001D1032B01D11846F8BDF9F765FDC01BA7
:108FB800B0F57A7F234684BF032386F82D30ECE78B
:108FC8000023F0E70028004038B50F4CE36823F091
:108FD8008003E360A3699B06054606D4FFF7B6FF46
:108FE80010B1032085F82D0038BDA36923F02003B4
:108FF800A361FFF7ABFF10B1032085F82D00A3692B
:1090080043F02003A361EFE70028004038B5044689
:1090180000284BD090F82D3003F0FF021BB980F8E0
:109028002C20F9F713FB0223214D84F82D30EB682F
:10903800DB0636D4CA236B6253236B622046FFF7E4
:109048009DFF10B1FF236B6238BDAB6923F08E63BF
:1090580023F04003AB6121696368AA690B4313439A
:10906800A2691343AB61D4E9022343EA02432B61AB
:10907800D4E90931EA680B4322F4F8521343EB6050
:109088002046FFF7A1FF0028DCD1D4E90713AA691D
:109098000B4322F06042134362691343AB61FF2321
:1090A8006B62012384F82D300020CDE70120CBE747
:1090B800002800400023092803D840EA0310C0B262
:1090C80070470A380133C0B2F5E700002DE9F047D0
:1090D80090F82C30012B05464FF0020069D001238F
:1090E80085F82C304E4B85F82D00DE6806F4407666
:1090F800B6F5807F78D04C69087891F8019091F89E
:1091080002A091F82470002A55D19B6913F04003FE
:1091180008BFCB70FFF7CEFF80464846FFF7CAFF6F
:1091280002465046FFF7C6FF81463846FFF7C2FFA2
:109138000B6ACF78234343EA875343EA090343EA98
:10914800084343EA022343EA0063354ACA205062CF
:10915800532050628C6A8869B4F5807F946945D140
:1091680024F4885494610124D465B6F5807F09BF3E
:10917800CB6913640343536418BF5064284B4A688F
:109188001A672A6B42F001022A639A6942F48852EC
:109198009A61244AD2F8803043F40033C2F8803010
:1091A8001F4BFF225A620020012385F82D3085F8D5
:1091B8002C00BDE8F087B4F1803F07D0B4F5000F6C
:1091C80004D09B6913F0400308BFCB700B6ACA78C0
:1091D8001C4344EA0A0444EA004343EA092343EAF5
:1091E800825343EA0763B0E70023AEE724F4085448
:1091F80094610224D465B6F5807F09BFCB69936476
:109208000343D36418BFD064054B4A685A672A6B76
:1092180042F002022A639A6942F40852B8E700BF92
:10922800002800400008005890F82C20012A034626
:109238004FF0020012D00A4A83F82D00CA21516269
:1092480053215162916941F020019161FF215162DE
:109258000020012283F82D2083F82C00704700BFDE
:109268000028004090F82C20012A03464FF0020005
:1092780019D00D4A83F82D00CA2151625321516239
:1092880091690A4841F080019161D0F8801041F459
:109298008021C0F88010FF2151620020012283F84C
:1092A8002D2083F82C007047002800400008005843
:1092B800064B5A6D520610B5044603D54022DA65AE
:1092C800F9F7F0FC012384F82D3010BD0028004088
:1092D8007047890001F1804101F531410A6070470A
:1092E800890001F1804101F53141086870470000AB
:1092F800034AD2F8903043F40043C2F890307047E4
:1093080000040058034AD2F8903023F40043C2F80E
:109318009030704700040058074B1A6822F040024A
:109328001A6040F441704FF4B85218605A601A68D5
:1093380042F040021A6070470000015837B50546F0
:1093480000284ED0837903F0FF046BB1032C0BD0B7
:10935800254B4FF400629A612868FFF7DDFF00246F
:1093680001232B71AC602FE000236B712846F9F7BD
:109378009DFA1E4AD2F8903043F48053C2F89030D8
:10938800002CE5D102234FF0B042AB71D2F89430F3
:1093980023F40043C2F89430154B1B681C214B433F
:1093A800DB0C64214B430193019B93B90124AC600E
:1093B800FFF79EFF0C4B9A6842F400629A604FF4E4
:1093C80000629A61002CC7D00123AB71204603B01C
:1093D80030BD019B013B0193D2F894305B04E3D488
:1093E800E6E70124F2E700BF00040058000800582F
:1093F8002808002037B5174D2B6802461C20434328
:10940800DB0C6420434314480193019B93B901206A
:109418009060114C21732B681C214B43DB0C642199
:109428004B430193019B6BB9012090600A4BDB68A9
:1094380003B030BD019B013B019383689C07E4D5D1
:109448000020E6E7019B013B0193A368DB07E9D510
:10945800ECE700BF280800200000015837B5184D78
:109468002B6802461C204343DB0C64204343154809
:109478000193019BA3B901209060124CFF23237331
:109488002B681C256B43DB0C64256B430193019B04
:1094980073B9012090600B4BDB680B7003B030BDD3
:1094A800019B013B019383689C07E2D50020E4E718
:1094B800019B013B0193A368DB07E8D5EBE700BFFD
:1094C80028080020000001580E4B0F491B6818227D
:1094D800534382B01B0D6422534301934B69019A95
:1094E800C3F3800322B902238360012002B07047CE
:1094F800019A013A01924A69920701D5002BEDD1F0
:109508000020F3E7280800200004005807B5037975
:10951800012B0FD10A4B1B68182253431B0C0193D4
:10952800FFF7F0FE019B013B0193019B002BF9D152
:10953800FFF7DEFE03B05DF804EBFFF7C5BF00BF21
:1095480028080020F8B51E468379012B15460446E5
:109558000F46DAB22DD14379012B2AD0022342716A
:109568008371FFF7D3FF0D212046FFF7CBFEFFF7EE
:1095780041FF390A2046FFF73DFFF9B22046FFF7C1
:1095880039FF2E44B5420ED12046FFF7B1FEFFF752
:109598009BFFA06801230038A3714FF0000318BF98
:1095A80001206371F8BD15F8011B2046FFF722FF63
:1095B800E8E70220F6E7F8B51E468379012B154641
:1095C80004460F46DAB22FD14379012B2CD04271D1
:1095D800FFF79CFF1D212046FFF794FEFFF70AFFC7
:1095E800390A2046FFF706FFF9B22046FFF702FFC7
:1095F80000212046FFF7FEFE2E44B5420ED120463C
:10960800FFF776FEFFF760FFA06801230038A3711B
:109618004FF0000318BF01206371F8BD29462046AA
:10962800FFF71CFF0135E8E70220F6E7F8B51F460B
:109638008379012B154604460E46DAB22CD14379BC
:10964800012B29D04271FFF761FF06F0EF03A3F168
:10965800840253425341237131462046FFF752FE9C
:10966800FFF7C8FE2F44AF4210D1FFF741FE842E0A
:1096780002D02046FFF728FFA06801230038A37115
:109688004FF0000318BF01206371F8BD15F8011BE6
:109698002046FFF7AFFEE6E70220F6E7F8B51E46DC
:1096A8008379012B154604460F46DAB227D1437950
:1096B800012B24D04271FFF729FF39462046FFF7D6
:1096C80021FEFFF797FE00212046FFF793FE2E4468
:1096D800B5420ED12046FFF70BFEFFF7F5FEA06856
:1096E80001230038A3714FF0000318BF01206371F4
:1096F800F8BD29462046FFF7B1FE0135E8E702200C
:10970800F6E737B50023ADF8043001AA0223122189
:109718000546FFF7C3FFBDF80440022364BA01AA57
:10972800A4B219462846FFF781FFE20702D528466A
:1097380009F094F9A30702D5284609F095F96007BE
:1097480002D5284609F0BAF9210702D5284609F0BA
:10975800BBF9E20602D5284609F0BCF9A30602D5F2
:10976800284609F0A5F9600602D5284609F082F9CD
:10977800210606D514F4807118BF0121284609F086
:109788007FF9A20502D5284609F08AF9630402D5B3
:10979800284609F0A5F903B030BDF8B51E4683790F
:1097A800012B154604460F46DAB227D14379012B1F
:1097B80024D04271FFF7AAFE0E212046FFF7A2FD32
:1097C800FFF718FE39462046FFF714FE2E44B5422F
:1097D8000ED12046FFF78CFDFFF776FEA068012327
:1097E8000038A3714FF0000318BF01206371F8BD62
:1097F80015F8011B2046FFF7FDFDE8E70220F6E714
:10980800F8B51E468379012B154604460F46DAB291
:109818002BD14379012B28D04271FFF777FE1E2107
:109828002046FFF76FFDFFF7E5FD39462046FFF7B5
:10983800E1FD00212046FFF7DDFD2E44B5420ED1A3
:109848002046FFF755FDFFF73FFEA06801230038CB
:10985800A3714FF0000318BF01206371F8BD2946BA
:109868002046FFF7FBFD0135E8E70220F6E702682E
:1098780052E8003F23F0C00342E8003102680029A3
:10988800F5D102F1080353E8003F23F4000302F185
:10989800080C4CE800310029F3D12023C0F88830A7
:1098A8007047000010B5026852E8003F23F4907337
:1098B80042E8003102680029F5D10F4C02F1080393
:1098C80053E8003F234002F1080C4CE8003100291E
:1098D800F4D1C36E012B07D152E8003F23F01003E7
:1098E80042E800310029F7D12023C0F88C3000234A
:1098F800C366436710BD00BFFEFFFFEFF8B504461F
:109908001346D4F88850202D32D1F1B1EAB1E06F76
:10991800A4F85620A4F8542000262122C4F8906008
:109928002165C4F88820226888B1124FC762124F97
:109938000763124F2832C0E90D76FDF79DFE30B15E
:109948001023C4F89030C4F888500120F8BD23686B
:1099580040221A62226802F1080353E8003F43F0EC
:10996800800302F1080141E800300028F3D1EDE757
:109978000220EBE789990008D1990008DD990008D1
:1099880008B50346806A1B681B6813F0200317D1CB
:10999800A0F85630026802F1080353E8003F23F0AC
:1099A8008003083242E8003102680029F2D152E807
:1099B800003F43F0400342E800310029F7D108BDD9
:1099C800F9F780FAFBE7704708B5806AFFF7FBFFF5
:1099D80008BD7047806A38B50468D0F88830D0F878
:1099E8008C50A268120606D5212B04D10023A0F8BA
:1099F8005630FFF73CFFA3685B0606D5222D04D13D
:109A08000023A0F85E30FFF74DFFD0F8903043F008
:109A18001003C0F89030FFF7DCFF38BD7047000036
:109A2800D0F88C20B0F86010222A08B5036855D108
:109A38005B6A826D0B401370836D01338365B0F8E8
:109A48005E30013B9BB2A0F85E30B0F85E309BB24E
:109A5800002B42D1026852E8003F23F4907342E899
:109A6800003103680029F5D103F1080252E8002FFC
:109A780022F0010203F1080C4CE800210029F3D17F
:109A88002022C0F88C20184A41679342016705D10B
:109A9800C26E012A0ED0F9F723FA1EE05A681102A5
:109AA800F6D553E8002F22F0806243E80021002910
:109AB800F7D1EDE70022C26653E8002F22F010022A
:109AC80043E800210029F7D1DA69B0F85C10D20622
:109AD80044BF10221A62FFF7A1FF08BD9A6942F03D
:109AE80008029A61F9E700BF00800040D0F88C2096
:109AF800B0F86010222A08B5036852D15A6A11409A
:109B0800826D22F8021B8265B0F85E20013A92B29B
:109B1800A0F85E20B0F85E2092B2002A40D153E847
:109B2800002F22F4907243E800210029F7D103F1B5
:109B3800080252E8002F22F0010203F1080C4CE859
:109B480000210029F3D12022C0F88C20174A416750
:109B58009342016705D1C26E012A0ED0F9F7C0F908
:109B68001EE05A681102F6D553E8002F22F08062F1
:109B780043E800210029F7D1EDE70022C26653E847
:109B8800002F22F0100243E800210029F7D1DA69FA
:109B9800B0F85C10D20644BF10221A62FFF73EFFED
:109BA80008BD9A6942F008029A61F9E7008000400E
:109BB8002DE9F84F0368B0F86060D3F81CB01F684F
:109BC8009D68D0F88C20222A044640F0B980B0F86D
:109BD800683043B1DFF87491DFF874A14FF00008E2
:109BE8001BF0200F20D1B4F85E309BB2D3B1B4F88B
:109BF80068209A4216D9226802F1080353E8003F08
:109C080023F08053083242E8003122680029F2D15B
:109C1800504B636752E8003F43F0200342E80031AD
:109C28000029F7D1BDE8F88F2368A26D5B6A33403D
:109C38001370A36D0133A365B4F85E30013B9BB28A
:109C4800A4F85E302368D3F81CB01BF0070F2ED0A1
:109C58001BF0010F09D0F90507D501221A62D4F8C3
:109C6800902042F00102C4F890201BF0020F09D0A6
:109C7800EA0707D502221A62D4F8902042F00402BB
:109C8800C4F890201BF0040F09D0E80707D5042278
:109C98001A62D4F8903043F00203C4F89030D4F834
:109CA800903023B12046FFF794FEC4F89080B4F8B2
:109CB8005E309BB2002B93D1226852E8003F23F418
:109CC800807342E8003123680029F5D103F10802C6
:109CD80052E8002F02EA090203F1080040E80021D7
:109CE8000029F3D120225345C4F88C2061672167ED
:109CF8000AD05A68110207D553E8002F22F0806273
:109D080043E800210029F7D1E26E012A14D100228C
:109D1800E26653E8002F22F0100243E800210029F0
:109D2800F7D1DA69B4F85C10D20644BF10221A627F
:109D38002046FFF773FE53E72046F9F7D1F84FE7BF
:109D48009A6942F008029A616CE700BFFEFFFFEFD4
:109D580000800040299A00082DE9F84F0368B0F800
:109D68006060D3F81CB01F689D68D0F88C20222A48
:109D7800044640F0B780B0F8683043B1DFF870911E
:109D8800DFF870A14FF000081BF0200F20D1B4F8C5
:109D98005E309BB2D3B1B4F868209A4216D92268D3
:109DA80002F1080353E8003F23F08053083242E8E9
:109DB800003122680029F2D14F4B636752E8003F17
:109DC80043F0200342E800310029F7D1BDE8F88FBD
:109DD8002368A26D596A314022F8021BA265B4F8C3
:109DE8005E20013A92B2A4F85E20D3F81CB01BF0B2
:109DF800070F2ED01BF0010F09D0F90507D5012256
:109E08001A62D4F8902042F00102C4F890201BF0A6
:109E1800020F09D0EA0707D502221A62D4F8902067
:109E280042F00402C4F890201BF0040F09D0E807A0
:109E380007D504221A62D4F8903043F00203C4F81C
:109E48009030D4F8903023B12046FFF7C2FDC4F813
:109E58009080B4F85E309BB2002B95D1226852E80E
:109E6800003F23F4807342E8003123680029F5D1CC
:109E780003F1080252E8002F02EA090203F1080080
:109E880040E800210029F3D120225345C4F88C2052
:109E9800616721670AD05A68110207D553E8002F75
:109EA80022F0806243E800210029F7D1E26E012AFE
:109EB80014D10022E26653E8002F22F0100243E892
:109EC80000210029F7D1DA69B4F85C10D20644BF42
:109ED80010221A622046FFF7A1FD55E72046F8F741
:109EE800FFFF51E79A6942F008029A616EE700BFE6
:109EF800FEFFFFEF00800040F59A000838B50446E1
:109F080003682169A2681D68C0690A4361690A4338
:109F18007749024329400A431A605A68E16822F4E3
:109F280040520A435A60734AA16993421CBF226A8D
:109F380011439A6822F06E4222F430620A439A6012
:109F4800DA6A616A22F00F020A43DA626A4A9342C5
:109F580019D14FF0B043694AD3F8883003F00303AE
:109F680043F44033934200F0B480B3F1031F24D08C
:109F7800013A934240F0B580B0F5004F40F08F8031
:109F8800FEF786FA6EE05E4A93421CD14FF0B0436A
:109F98005C49D3F8883003F00C0343F440228A422A
:109FA80000F0978006D8002B7CD0574B9A42E3D01C
:109FB800012026E0B2F10C1FFAD1B0F5004F53D0C2
:109FC8004FF4004075E04B4A9342F1D14FF0B04353
:109FD800D3F8883003F44063B3F5006F18D006D87F
:109FE8005BB1B3F5806FE3D1FEF752FA07E0B3F542
:109FF800406FDDD14FF400400BE0FEF741FE40B961
:10A0080000204FF00113A3660023C4E91D3338BDB7
:10A018003E4865683E4B626A05EB450133F81220FD
:10A02800B0FBF2F39942C3D8B3EB053FC0D8002385
:10A038001946F7F769FD090241EA10616B08000249
:10A04800C0182A464FF0000341F10001F7F75CFD04
:10A05800304BA0F540729A42AAD82368D860CFE75F
:10A06800FEF70EFE0028CBD06168294B626A33F8F0
:10A078001220B0FBF2F24B0803EB42034FF6EF72EB
:10A08800B3FBF1F3A3F11001914291D823F00F0231
:10A09800216892B2C3F342031343CB60B0E7FEF7E3
:10A0A800F7F904E0B0F5004FDAD0FEF7E9FD002833
:10A0B800A6D06368616A164A32F81120B0FBF2F044
:10A0C80000EB5300B0FBF3F04FF6EF73A0F1100272
:10A0D800C1E7B0F5004F0D48EBD1C5E7FEF7E0FD4D
:10A0E800C0E7B0F5004FF9D0FEF7DAFDDFE700BFB3
:10A0F800F369FFCF008000400038014002000300F0
:10A108000044004008000C0004000C000024F40087
:10A11800603B0108FFFC0F00836ADA0710B506D51B
:10A128000168C46A4A6822F4003222434A609C07E4
:10A1380006D50168046B4A6822F4803222434A60DB
:10A14800590706D50168446B4A6822F480222243E5
:10A158004A601A0706D50168846B4A6822F40042EF
:10A1680022434A60DC0606D50168C46B8A6822F47B
:10A17800805222438A60990606D50168046C8A6871
:10A1880022F4005222438A605A060FD50168446CB3
:10A198004A6822F480122243B4F5801F4A6005D130
:10A1A8004A68846C22F4C00222434A601B0606D522
:10A1B8000268C16C536823F400230B43536010BD3D
:10A1C8002DE9F843DDF8209005460F4616469846D7
:10A1D8002A68D36937EA03030CBF01230023B3427B
:10A1E80001D0002029E0B9F1FF3FF2D0F8F744FC94
:10A1F800A0EB080048452C6802D8B9F1000F1ED121
:10A2080054E8003F23F4D07344E80032002AF7D121
:10A2180004F1080353E8003F23F0010304F10801A7
:10A2280041E80032002AF3D12023C5F88830C5F868
:10A238008C30002385F884300320BDE8F883236838
:10A248005A07C5D5E3691B05C2D54FF400632362DD
:10A2580054E8003F23F4D07344E80032002AF7D1D1
:10A2680004F1080353E8003F23F0010304F1080157
:10A2780041E80032002AF3D12023C5F88830C5F818
:10A288008C30C5F89030D4E773B504460026C0F882
:10A298009060F8F7F1FB23681B681A07054619D484
:10A2A80023681B685B070AD56FF07E430093002282
:10A2B8002B464FF480012046FFF782FFB0B90020FB
:10A2C8002023C4F8883084F88400C4F88C30E06611
:10A2D80020670CE06FF07E430093324603464FF44C
:10A2E80000112046FFF76CFF0028D9D0032002B0E8
:10A2F80070BD10B5044650B3D0F888301BB980F84B
:10A308008430F8F70BFD22682423C4F888301368DA
:10A3180023F0010313602046FFF7F0FD012816D053
:10A32800A36A13B12046FFF7F7FE23685A6822F4A0
:10A3380090425A609A6822F02A029A601A6842F09B
:10A34800010220461A60BDE81040FFF79DBF0120BA
:10A3580010BD000030B581658168A0F85C2000233D
:10A36800B1F5805FA0F85E20436735D10369002B03
:10A3780040F2FF1318BFFF23A0F860300023C0F895
:10A3880090302223C0F88C30016801F1080353E8AB
:10A39800003F43F00103083141E800340368002C12
:10A3A800F2D1456E84680169B5F1005F32D1B0F829
:10A3B800685095422ED8B4F5805F244A03D1244CC6
:10A3C800002908BF22464267B1B153E8002F42F482
:10A3D800807243E80021F7E729B90369002B14BF0D
:10A3E8007F23FF23C8E7B1F1805FC5D10369002B44
:10A3F80014BF3F237F23BFE703F1080252E8002F71
:10A4080042F0805203F1080040E800210029F3D10E
:10A41800002030BDB4F5805F0E4A03D10E4C0029F0
:10A4280008BF2246426741B153E8002F42F49072B8
:10A4380043E800210029F7D1EAE753E8002F42F06A
:10A44800200243E800210029F7D1E1E7B99B000881
:10A45800619D0008299A0008F59A0008D0F88C3008
:10A46800202B30B415D1B9B1B2B100230468C3664A
:10A478000A4B9C420AD063681B0207D554E8003F88
:10A4880043F0806344E80035002DF7D130BCFFF776
:10A4980061BF022030BC70470120FBE7008000400C
:10A4A800436E30B52BB90123A0F86A30A0F86830A4
:10A4B80030BD0368094D9A689968094C490FC2F381
:10A4C80042626B5C615CDB00B3FBF1F3A0F86A30BD
:10A4D800AB5CA25CDB00B3FBF2F3E7E7803B01086F
:10A4E800783B01081FB504AB03E9060090F88430F7
:10A4F800012B04463AD0012380F884302423C0F885
:10A50800883003681A6822F001021A609A6822F4F7
:10A5180040120A439A6071B95A68BDF80C009DF858
:10A528000E1022F0100202435A605A6822F07F424D
:10A5380042EA01625A601A6842F001021A60F8F7AA
:10A548009BFA6FF07E42034600924FF4800100228E
:10A558002046FFF735FE38B92023C4F88830002399
:10A5680084F8843004B010BD0320F8E70220F9E72E
:10A5780090F88430012B0FD0012380F884300168D3
:10A5880051E8002F42F0020241E80023002BF6D1E7
:10A5980080F88430184670470220704710B590F84C
:10A5A8008430012B044617D02423C0F88830036870
:10A5B8001A68196821F00101196042F000524FF041
:10A5C800005141661A60FFF76BFF2023C0F88830FE
:10A5D800002084F8840010BD0220FCE770B590F8D4
:10A5E8008430012B044617D005682423C0F888302E
:10A5F8002E682B6823F001032B60AB6823F06043BF
:10A608001943A960FFF74CFF20232E60C0F888305B
:10A61800002084F8840070BD0220FCE738B5084D9E
:10A62800052455F8043B2BB9013C14F0FF04F8D17C
:10A63800204638BDDB6898470028F5D0F9E700BF09
:10A6480028100020034BD870034B1B681B6C03B108
:10A6580018477047101000200C100020034B187486
:10A66800034B1B685B6C03B1184770471010002040
:10A678000C100020F0B5314D314B95F90420314EC6
:10A6880091B00C46012795F905108DF80470022841
:10A698008DF809208DF80A1010D18DF80800D871AE
:10A6A8001C7202F063FD337803B114B101A803F002
:10A6B800C1F9254B059A1A6011B0F0BD59714FF4D4
:10A6C80080711A71D9801C7233788DF8087053BB69
:10A6D8001F2306A88DF81C208DF8183002F024FFDF
:10A6E80020238DF8183006A82B798DF81C3002F03D
:10A6F8001BFF22238DF8183006A86B798DF81C30C3
:10A7080002F012FF21238DF8183006A86B798DF816
:10A718001C3002F009FF29238DF8183006A80B4BCE
:10A72800079302F001FF02F021FD012306A88DF82E
:10A7380018308DF81C3002F0F7FEB4E71010002036
:10A7480060080020EC0E0020E00F0020000400014B
:10A758007FB5092301A88DF8043003F06BF90038A0
:10A76800044B059A1A6018BF0120404207B05DF8F3
:10A7780004FB00BFE00F002070B504460B461449E7
:10A7880062784A700020A2780A7208701A884A72A1
:10A798009A788A72DB780B746368CB600D4B1B6800
:10A7A800DA6A2AB1237803F0FB030A2B00D090471A
:10A7B800094E002556F8043B1BB15B6A0BB12046D5
:10A7C80098470135EBB2052B6DB2F3D170BD00BFD0
:10A7D800300800200C1000202810002070B5044616
:10A7E80011480123037063784370A3788372E36888
:10A7F800C360E378037623694376237943720B4B6E
:10A808001B689B6A03B19847094E002556F8043B1C
:10A818001BB19B690BB1204698470135EBB2052B5C
:10A828006DB2F3D170BD00BF440800200C100020A9
:10A8380028100020014B1868704700BFE00F002067
:10A8480000B58BB0012368468DF8003002F046FD54
:10A8580038B99DF80400003818BF01200BB05DF826
:10A8680004FB0020FAE7000008B501F037FE40B904
:10A87800FFF7E6FF012806D0054B197AD879FFF7CC
:10A88800F9FE012008BDBDE80840FFF7C7BE00BFBC
:10A89800600800202DE9F04186B005460E461746AF
:10A8A80001F01CFE002873D101F030FE044640B9C7
:10A8B800FFF7C6FF01280AD03D4B197AD879FFF770
:10A8C800D9FE6FF00204204606B0BDE8F081DFF83B
:10A8D800E48088F80860003E18BF01268DF80460FF
:10A8E800354E687833798DF81230694602F094FC59
:10A8F80000283FD08DF804400394ADF810406FF065
:10A90800060495E803002D4B83E80300337988F8A3
:10A918000A30394601A803F091F9294B059A1A60C3
:10A9280011283FD801A353F820F000BF9FA90008C1
:10A9380099A90008ADA90008ADA90008ADA90008AB
:10A94800ADA90008ADA90008CBA80008ADA900086A
:10A95800ADA90008ADA9000893A90008ADA9000891
:10A96800ADA9000899A9000899A9000899A90008A3
:10A97800B3A900082B788DF808306B78ADF8103043
:10A988006B6803934FF0FF34BBE76FF005049AE759
:10A998006FF0010497E70B4B00221A70E31D18BFF4
:10A9A800144690E74FF0FF348DE76FF004048AE710
:10A9B80060080020440800201010002054080020DF
:10A9C800E00F0020DF0F002037B501F0A9FD134D7F
:10A9D800052455F8043B4BB11A693AB19B682BB171
:10A9E800984718B155F8043C1B699847013C14F086
:10A9F800FF04EED1FFF712FE68B9094D2B7853B169
:10AA0800084BADF80040D978019422466846FFF714
:10AA180041FF00B92C7003B030BD00BF28100020E2
:10AA2800DF0F00201010002030B58BB0044601F075
:10AA380055FD0546002835D1FFF702FF012834D11E
:10AA480068468DF8005002F049FC40BB9DF8043080
:10AA5800A34204D0012C22D0022C12D014B1002021
:10AA68000BB030BD002BFAD068468DF8044002F0D8
:10AA78005BFDA0B90E4B1B681B6B002BEFD09847F2
:10AA8800EDE763B968468DF8044002F04DFD30B932
:10AA9800074B1B681B6B002BE1D02046EFE74FF0FC
:10AAA800FF30DDE76FF00100DAE76FF00200D7E76B
:10AAB8000C10002010B504468AB018B94FF0FF30CA
:10AAC8000AB010BD002368468DF8003002F006FC7D
:10AAD8000028F3D19DF804302370F1E77FB50022F8
:10AAE8000B4620498DF8072001220A7042784A70E7
:10AAF8000446002A33D102790A721A884A729A786F
:10AB08008A72DB780B740369CB60C378164D8DF8B5
:10AB18000830037B8DF80930836803932B68DB6A60
:10AB28000BB102A898472B689B6B13B1227E02B128
:10AB380098470E4E052556F8043B1BB1DB690BB14F
:10AB480020469847013D15F0FF05F4D10DF10700A7
:10AB5800FFF7B0FF637913B1054B01221A7004B0F7
:10AB680070BD00BF300800200C1000202810002005
:10AB7800DF0F002010B504468AB018B94FF0FF3037
:10AB88000AB010BD202368468DF8003002F0A6FBFD
:10AB98000028F3D1024A9DF9043023701371EFE7BE
:10ABA8001010002000B58BB02323019068468DF863
:10ABB800003002F0B9FC003818BF012040420BB049
:10ABC8005DF804FB70B5654C01468EB0182220462E
:10ABD80006F0C0F8624B00221A70F9F783F923785F
:10ABE8004068012202FA03F1014004D15D4B084696
:10ABF80008F09CF8FEE75C495C481A4602F0F8F851
:10AC080018B14FF0FF300EB070BD272304A88DF89F
:10AC1800103002F089FC564E564D002870D10123A1
:10AC280033702B68DB690BB100209847272304A8F1
:10AC38008DF8103002F052FB059B93F848202270E3
:10AC480093F8182193F81A316270A370464BD3E930
:10AC5800020105F06FFF05460028D2D1464E0623B3
:10AC680004A88DF8103002F039FB059B736104A825
:10AC780002F05AFC022304A88DF81030059602F061
:10AC88002DFB0836032304A88DF81030059602F032
:10AC980025FB0F2606F014F8012304A88DF81430BC
:10ACA8008DF8106002F040FC10230DEB03008DF8C6
:10ACB80010308DF8145002F037FC04238DF8103052
:10ACC80004A8A3788DF8143002F02EFC3A238DF8EE
:10ACD800103004A86369059302F026FC02A92078C5
:10ACE8008DF8086004F09CF8003818BF0120E07166
:10ACF8001420FFF757FFE07903F062F9284682E74E
:10AD080028238DF810302B681B6943B104A802F082
:10AD1800E5FA2B6805981B6940F2C4519847272328
:10AD280004A88DF8103002F0FFFB50B9012304A8E5
:10AD38008DF8103002F0D2FA9DF81430002B7FF411
:10AD48006EAF3378002B7FF46CAF052204A88DF822
:10AD58001020059302F0E8FB78E700BF10100020F0
:10AD6800DF0F0020883B0108E40F0020FC0F0020C3
:10AD7800EC0E00200C1000204C10002037B50023EA
:10AD88000D4601930446D0B900F0A8FB0190019B41
:10AD9800D3B10F4A42F824300E4A9A620E4A12681A
:10ADA800916B1963916C596392690C49D9625A6124
:10ADB80028465B680A49F2229847002006E001A964
:10ADC80000F092FB0028E2D04FF0FF3003B030BD16
:10ADD800281000207DA600080C10002059A70008A4
:10ADE800ED0E0020194B07B51860194B194A1A6067
:10ADF800194A5A60194A9A60194ADA60194B026866
:10AE08001A6042685A6082689A60C268DA60164AB4
:10AE18001A6182695A61154BC26B5A60144A0191D2
:10AE280019609A601946134ADA600020FFF7A6FFF6
:10AE380048B901A800F056FB003818BF012040426D
:10AE480003B05DF804FB4FF0FF30F9E70C10002069
:10AE5800FC0F0020E5A70008E5AA0008F9AE0008E5
:10AE680081A70008E40F0020D9ED00083C1000205D
:10AE78004DA6000865A6000849B118B1012804D0FC
:10AE880000207047034B0B60FAE7034BFBE74FF0DA
:10AE9800FF307047000400010100010208B503F00B
:10AEA800ABF8002814BF6FF00100002008BD08B5FA
:10AEB80002F084F9002814BF6FF00100002008BDDB
:10AEC80010B504468AB018B94FF0FF300AB010BD6B
:10AED800212368468DF8003002F000FA0028F3D1EB
:10AEE800024A9DF9043023705371EFE710100020D7
:10AEF8002DE9F0412F4D304F00232B7043786B70B4
:10AF08003B689B6A8AB004460BB128469847DFF82D
:10AF1800AC80002658F8043B1BB11B6A0BB12046D5
:10AF280098470136F3B2052B76B2F3D12378052B77
:10AF38002FD00B2B35D0012B25D1214C0623684669
:10AF48008DF8003002F0CAF90199E07905F038FE71
:10AF580010B91C4B019A5A611B48FFF70BFE1B489E
:10AF6800FFF7AEFF6B788BB9A371194B5878FFF7D1
:10AF78005BFD3B685B6A0BB1114898476B7813B966
:10AF8800E07905F0AFFE0AB0BDE8F081FF23A371B8
:10AF9800EFE7104B01225A74227A9A74627ADA74B3
:10AFA800F1E76378002BEED00AB0BDE8F041FFF777
:10AFB800CFBB00BF440800200C1000202810002040
:10AFC800600800204C10002064080020650800205C
:10AFD800101000203008002030B58BB0FFF767FF55
:10AFE8000446F0B903F0FCFE831C1DD0F8B9134DDC
:10AFF8002B685B69DBB1272368468DF8003002F0C7
:10B008006DF92B6801985B694FF4B961984703F0B3
:10B01800F9FE78B92CB9094B1B68DB690BB1012023
:10B02800984720460BB030BD6FF00704EFE74FF0AC
:10B03800FF34ECE74FF0FF34F3E700BF0C100020BB
:10B04800014B1878704700BF80100020014B5878DA
:10B05800704700BF8010002070470000044B9A7AA8
:10B068000AB101225A70034B5B6903B11847704754
:10B07800801000206C08002073B5224C6378002BE8
:10B0880033D008F03BF966680546FFF7D3FB064462
:10B09800AE4214D2A37A93B1E0228DF800208DF845
:10B0A8000130217AE368019301226846FFF7F2FB39
:10B0B80008B1073010D100236370A372656094F85B
:10B0C8003430EBB1002384F834300F4B5B6BBBB1E9
:10B0D80002B0BDE87040184740F2DC510B4808F058
:10B0E800D9F90A4808F09CF9E8E794F83520002ACD
:10B0F800E5D094F8360084F83530FFF795FCDEE7A4
:10B1080002B070BD801000206C0800206410002080
:10B1180037B5104D104CC8B1C1B16272012300227D
:10B128002860E16023700D480D4B00924FF0FF310D
:10B1380008F0CAF800250B4825822022294605F088
:10B148001DFE6570A574A58603B030BD00232B6075
:10B158002370EFE77C10002080100020641000208E
:10B1680065B00008941000202DE9F0478E4C237834
:10B178008CB0002B56D0C2780AB9837B13B1238ACE
:10B1880001332382437B002B4CD0E02A4AD1002391
:10B19800A372876897F80080B8F1220F27D8B8F112
:10B1A800220F30D8DFE818F04100FB0052005A00A7
:10B1B80061006E0075008E009D00B400C7002F006E
:10B1C8002F002F002F002F002F002F002F002F00FF
:10B1D8002F002F002F002F002F002F002F002F00EF
:10B1E8002F002F002F002F00C900D000D400B8F185
:10B1F8007E0F00F0CC80B8F17F0F00F0DF80B8F14F
:10B208007D0F00F0AB80A57A002D00F05B81674CC4
:10B21800637A3BB94FF47A71204608F03BF920462F
:10B2280008F0FEF80CB0BDE8F087E36801220021C1
:10B23800A2721970A37AE1689818A0720620C854FF
:10B24800A37AE1689818A072CA54DCE7584B9B6A45
:10B25800002BD8D0012102209847D4E77B7884F8C6
:10B268003630012384F83530CDE704238DF80430D7
:10B278007B78003B18BF012301A88DF8083002F045
:10B2880053F9C0E77878003818BF012002F098FE1B
:10B29800B9E7484E0FCE01AD0FC50FCE0FC596E8E2
:10B2A800070085E807007B780A2BACD8424A126869
:10B2B8005268002AA7D00CA901EB830353F82C0C81
:10B2C8009047A0E77878431E012B9CD83A4B013869
:10B2D8001B6818BF012020729B68002B93D09847E9
:10B2E80091E7E26801230821A3721170627A057B55
:10B2F800A17AAA4228BF2A46934284D285685A1C5A
:10B30800EB5CE56801334E1CA6726B54D3B2EDE7D3
:10B31800E3680122A27209221A70A37AE268218ADC
:10B32800581CA072D154A27A238AE1681B0A501CC7
:10B33800A0728B5467E7238265E705238DF80430F4
:10B3480001A802F077FB5EE7194BDB6A98475AE7DA
:10B35800194B78781B686075DB68BEE7037B072BA1
:10B368007FF451AF06238DF80430B7F80130ADF8FB
:10B3780008307B793A791B0443EA0223FA781343AD
:10B38800642253430393BB798DF81030D8E73B22EE
:10B3980001A88DF804208DF8083002F0C5F80123C3
:10B3A80084F834302FE700BF80100020641000209C
:10B3B8006C080020743901087C1000202A2301A899
:10B3C8008DF8043001F08AFF94F80A90E6689DF839
:10B3D80008009DF809509DF80A709DF80BC09DF86B
:10B3E8000D309DF80E209DF80F109DF80CE009F126
:10B3F800010A84F80AA006F80980354E94F80A90E4
:10B408003668D4F80C8009F1010A84F80AA096F885
:10B4180003A008F809A094F80A90D4F80C8009F160
:10B42800010A84F80AA096F802A008F809A094F87E
:10B438000A90D4F80C8009F1010A84F80AA096F859
:10B4480001A008F809A094F80A9009F1010A84F803
:10B458000AA096F80080E66806F8098094F80A8041
:10B46800E66808F1010984F80A9006F808C094F81B
:10B478000AC0E6680CF1010884F80A8006F80C7026
:10B48800A77AE66807F1010C84F80AC0F555A57A91
:10B49800E6686F1CA7727055A07AE568461CA6720C
:10B4A8002954A17AE0684D1CA5724254A27AE16839
:10B4B800501CA0728B54A37AE268591CA17202F83E
:10B4C80003E0A0E6034807F05DFF6570AAE600BF49
:10B4D8007C1000206410002070470000004870476E
:10B4E8006C080020002070474FF0FF3070470000C4
:10B4F800044B054A93F81831022B18BF062382F82B
:10B508009034704724170020E81C0020034BD3F820
:10B51800483313B15B6903B118477047E81C002032
:10B52800034A137843F004031370FFF7EFBF00BF1B
:10B53800CC1000201FB50A4B8DF8090093F87C2029
:10B548008DF80A2093F88C2093F848000D3202A950
:10B558008DF8082003F064FCC0B205B05DF804FB68
:10B568002417002008B5074807F00CFF064B93F88E
:10B578001A2412B1012283F81924BDE80840FFF704
:10B58800C5BF00BFE8200020E81C002010B50C4C07
:10B59800D4F8403343F08003C4F8403394F81A34A5
:10B5A80013B10020FFF7DEFF94F8913423F0120363
:10B5B80043F0120384F89134BDE81040FFF798BFB8
:10B5C800E81C00202DE9F041DFF8AC8098F818312C
:10B5D800022B06460D4602D0284BDB6A984702F03C
:10B5E800A6FD044628B1022002F097FD002002F0D3
:10B5F80099FD98F81831012B17D102F09AFD0746EA
:10B6080030B1002002F08AFD002002F08CFD3C469B
:10B6180002F091FD48B1002002F081FD002002F007
:10B6280083FDBDE8F041FFF763BF002CF9D1144C4E
:10B6380094F8902494F81A34BAB90BB184F8416498
:10B64800304602F017FFD8F82C0007F061FED4F856
:10B65800B4339842E5D30B4807F094FE94F891343C
:10B6680043F0100384F89134DBE70BB184F84154BC
:10B67800284602F0FFFEF1E72417002004430108E2
:10B68800E81C002080200020074A10B5137843F0FA
:10B6980002031370FFF73AFFBDE81040034B012285
:10B6A8000021022007F042BBCC100020D13B01084A
:10B6B800074A10B5137843F008031370FFF726FF05
:10B6C800BDE81040034B01220021022007F02EBBE9
:10B6D800CC100020E13B01082DE9F0410F46164649
:10B6E8001D46804607F00AFE0B4A0C4C137827814A
:10B6F80023F0110343F01103C4E9000813706681B5
:10B708002573FFF703FFBDE8F041054B0122002137
:10B71800022007F00BBB00BFCC100020B81000209F
:10B72800F13B010813B507F0E9FD0D4B6C461860B5
:10B73800204607F037FD94E803000A4A0A4B83E8DD
:10B748000300137843F020031370FFF7DFFE074B65
:10B7580001220021022002B0BDE8104007F0E6BA3D
:10B76800C8100020CC10002020200020FE3B01083B
:10B778002DE9F04192B0064602F0D9FC002840F0CD
:10B788005881AD4D95F81831012B09D02B6BAB4C76
:10B7980093B194F80431BBB1042B6FD0032003E0BC
:10B7A80002F0C7FC18B10F2012B0BDE8F08102F01A
:10B7B800C2FC0028EAD0F6E7B5F82031D4F81C24FA
:10B7C800013B53432B63E4E79D4803F060FA0028EC
:10B7D80040F0128194F80C3123802B6B0C930DF1FF
:10B7E800180895F839308DF83830404695F81C31EE
:10B7F8008DF83A3007F0FCFCD5F82831009302AFF9
:10B8080098E80600D5F82431384607F088FC97E810
:10B8180003000FAB83E80300EB6A0D9300238DF858
:10B8280044302388ADF8463095F8303101228DF840
:10B8380039201BB98DF844208DF83930814B00939D
:10B84800814B95F84800A3F179020CA903F05DFB40
:10B85800C0B10B28A8D1D4F8941499B1002EA3D064
:10B86800D4F84033794843F02003C4F8403307F054
:10B8780011FE764807F0D4FD002095E7704803F0E4
:10B888003AFAA4E795F8487095F9693095F939209E
:10B8980095F87D106E4E384603F044FB009641B291
:10B8A800EB6C95F850203846183603F0DFFA00960E
:10B8B800EB6C95F8502095F9701095F8480003F056
:10B8C800D5FAD4F8C413AB6DD4F8DC230B44C4F810
:10B8D800B033EB6D1344C4F8B43394F80431042B3B
:10B8E80007D02B6E0B44C4F8B0336B6E1344C4F806
:10B8F800B4330023089395F83031002B40D100234E
:10B908008DF8133095F839308DF8213095F83830A6
:10B918008DF82230D5F880300993D5F884300A9311
:10B928002388ADF82C3095F8303194F81B648DF8E5
:10B938002E3095F84800474B8DF820600DF1130222
:10B9480008A903F0A7FA012384F8413495F839309F
:10B9580084F842349DF8133084F84334D4F81C3406
:10B96800C4F85064C4F84834C4F8583402F0E5FB0D
:10B97800C8B1D4F81C0402F0F2FBA0B1102013E700
:10B9880008A802F0A7FC60B995F9390094F8376265
:10B998009DF82070FFF7CEFD3E44B042AFD208209C
:10B9A80002E7132000E795F81831012B01D102F0C6
:10B9B800D8FB02F0C5FB0023059394F8043195F9F0
:10B9C800395094F81B649BB1042B7FF4E7AE05A8AB
:10B9D80002F0B4FE58BB94F8183413B1059B013B30
:10B9E8000593174B05983246E9B202F00DFF02E0C5
:10B9F800134802F0DDFE08B11120D5E6D4F8403333
:10BA080094F80C11218043F00203C4F8403394F8F1
:10BA1800183411480133DBB284F8183484F84534FB
:10BA28000E4B00259B6AC4F89854984724E71220C7
:10BA3800BAE60E20B8E600BF24170020E81C002054
:10BA4800F01D0020541700207C21002050200020E9
:10BA5800A020002004210020EA1C00200443010843
:10BA680073B5134D134E0096EB6C95F8502095F96D
:10BA7800781095F8480003F0F9F995F830313375E6
:10BA880095F8480040F2012306F13C0231467382E2
:10BA980003F0F8F950B196F83C3086F88230064B3E
:10BAA80000205B6B9847F37C86F8A83002B070BD25
:10BAB80024170020D020002004430108F8B5324C98
:10BAC80094F81831012B05460ED0022B4ED0002BCE
:10BAD80057D138B9D4E91B0104F1740383E8030092
:10BAE8000020F8BD012806D102F02CFB0028F8D16F
:10BAF80084F81851F5E7022843D1244E84F8180138
:10BB080006F5747CBCE80F0006F57A770FC79CE849
:10BB1800030094F8E92094F8003187E8030086F8D8
:10BB2800FB53D2B1022B18D1D4F804316367C6F89D
:10BB3800EC3394F87D3094F8082186F8F83394F8BB
:10BB48008C3084F8782086F8F93396F81B2486F828
:10BB5800E82340F20133A6F8FA33002386F81A34B2
:10BB68000B4BDB6A9847FFF77BFFB9E748B9074BF0
:10BB780084F81801062283F89024054BDB6A98475D
:10BB8800AEE70320ADE700BF24170020E81C002023
:10BB980004430108F0B5504C504EB4F8DC2022871D
:10BBA800D4E92D0194F8B12084F8692004F16C02DD
:10BBB80082E80300D4E92F0104F1740282E803004B
:10BBC800B4F8C420A4F87C2091B0D4F8CC20D4F8E0
:10BBD800C810C4F884200025D4F8D020C4F88820E0
:10BBE8000123A4F82031C4F8801084F83051A562EC
:10BBF80084F81B5184F83A5084F81D5184F81E517A
:10BC0800C4F83451C6F89854A6F8185486F81A544B
:10BC1800A4F838518DF8183004F50973039304F526
:10BC28000A7394F84800049303A92D4B84F84551EE
:10BC3800C4E94F55A4F84651059303F0FFF8E36EA5
:10BC4800C6F8D43394F87D3086F8E03394F88C3015
:10BC580086F8E1334FF48073A6F8E23386F8D053C0
:10BC680094F8303186F8E43306F574770FCF06F58B
:10BC78007A740FC497E8030040F2012384E80300B4
:10BC8800A6F8FA33D6F8483386F81B54CDE901559F
:10BC98001BB15A685B6901920293124B0793A3F197
:10BCA80048020892A3F1140209920F4A0B92293311
:10BCB8000A93A2F19C030C93A2F198030D93131D10
:10BCC8000E9301A902F14C0307A802F599620F939C
:10BCD80002F022FA11B0F0BD24170020E81C002061
:10BCE800D01000205021002008180020F8B50D4F72
:10BCF8000D4E0C4607F046FB3B6B98470B4A96F8EF
:10BD08004800214603F0BEF850B1094D706D95F812
:10BD1800243485F86A347B6B9847E37C85F8903443
:10BD2800F8BD00BF04430108241700200C2100209F
:10BD3800E81C00200F4890F81B3480F8B8330E4BED
:10BD480093F8692080F8BB2393F87D2080F8C823F6
:10BD580093F88C2080F8C92393F8303180F8CC33DD
:10BD68000022A0F8CA2300F56E7100F56070FFF795
:10BD7800BDBF00BFE81C002024170020114890F820
:10BD88009034EBB190F81B3480F8D0330E4BDA6E58
:10BD9800C0F8D42393F87D2080F8E02393F88C2012
:10BDA80080F8E12393F8303180F8E4334FF480725F
:10BDB800A0F8E22300F5747100F56670FFF796BFEE
:10BDC800704700BFE81C00202417002070B5344CD1
:10BDD8002421204604F0D4FF636A984218BF6062A9
:10BDE8004FF01C012F4814BF0125002504F0C8FF9F
:10BDF800636C984218BF60644FF480712A4818BF7A
:10BE080045F0020504F0BCFFD4F84831984218BF49
:10BE1800C4F848014FF0D401244818BF45F0040580
:10BE280004F0AEFFD4F82032984218BFC4F82002BC
:10BE38004FF000011E4818BF45F0080504F0A0FFA8
:10BE4800D4F82432984218BFC4F824024FF4607121
:10BE5800184818BF45F0100504F092FFD4F8A8352B
:10BE6800984218BFC4F8A8054FF01401124818BF2B
:10BE780045F0200504F084FFD4F8C03598420F4BF4
:10BE880018BFC4F8C005D3F8483318BF45F04005BB
:10BE98002BB11B691BB12846BDE87040184770BD1F
:10BEA800241700204C1700206C1700207018002061
:10BEB800481900204C190020D01C0020E81C002044
:10BEC8002DE9F04F8FB04FF00009012B06460F46C1
:10BED80090468DF80D90ADF8109002D84C46BC42B3
:10BEE80002D30FB0BDE8F08F305D02F033FA204482
:10BEF800B842F6DC335D651C023BEDB2112BF0D87D
:10BF080001A252F823F000BF59BF000883BF000800
:10BF180081C00008A9C0000827C100084DC1000859
:10BF2800B3C10008DBC1000861C20008EBBE00080D
:10BF3800EBBE0008B5C20008EBBE0008EBBE000867
:10BF48005DC3000885C30008BDC30008F1C300082D
:10BF5800052002F0A7FA70B10521002002F068FA66
:10BF6800725DBA4BE51C0234E4B283F85C24325D9E
:10BF780083F85D24EDB22C46B1E700238DF80E302E
:10BF88008DF80F308DF814308DF81830B9F1000F96
:10BF98006DD1AF4C4FF0050994F87C208DF8312015
:10BFA8006B1E94F839208DF83320334494F83820E8
:10BFB8000B938DF8342094F81A3194F868208DF892
:10BFC8003520D4F82C218DF832300A9273B37B1CBB
:10BFD8005B1BDBB28DF8303006AB019305AB0093E9
:10BFE80094F848000DF10F030DF10E020AA902F0B2
:10BFF8005DFF8DF80D0000F00700072813D194F9B4
:10C0080039209DF90E3084F839309A429DF80F3066
:10C0180084F83830B8BF01229DF81430B8BF84F8CE
:10C028001D2184F868304FF0000A09E00523D1E7A4
:10C0380001220DF10D01032002F0A4F80AF1010A12
:10C048005FFA8AF29DF81830B3FBF9F19142EFD804
:10C058002B44DDB26B1EDBB29F420BD9F25C032A84
:10C068009AD0AF4288BF1D464FF0010983E70534D7
:10C07800E5B2F9E71D46F7E7735D754903F00F036D
:10C08800012281F81B31023402FA03F3A1F82031AE
:10C09800E4B2002204A9042002F074F825466AE7F5
:10C0A80007238DF80D30735DC3F3021203F00F03FD
:10C0B8008DF82830E31CDBB28DF82920F25C231DB3
:10C0C800DBB2651DF35C0234E4B21B0443EA0223CD
:10C0D800325D5F4C13436422534394F848000B933A
:10C0E8000AA902F0F2FE00F00703072BEDB28DF863
:10C0F8000D000CD19DF8283084F8703084F8783021
:10C108000B9BE36663679DF8293084F869308DF8E6
:10C118001000012204A9052002F034F82BE74B4B4C
:10C12800D3F8483363B11B6853B1984708F03F030D
:10C138008DF810008DF81130022204A90620EBE7D3
:10C14800FF20F3E703238DF80D30735D8DF81C3065
:10C158000AAB0693E31CDBB2A51DF25C231DDBB220
:10C1680006A9F35C1B0443EA0223A21CD2B20534DD
:10C17800B25C134364225343E4B20A9300230B9343
:10C18800335D8DF83030324B93F8480002F0A3FE4F
:10C19800C3B20028EDB28DF80D30FFF6ECAE8DF885
:10C1A8001030012204A90720B6E7735D03F00F03DE
:10C1B800012B4FF47A7238BF01235343244A0234C7
:10C1C800936503F57A73D365E4B2002204A90820C5
:10C1D80062E7735D1E4DC3F340128DF8152095F884
:10C1E8004800C3F3001205A903F00F038DF81420CB
:10C1F8008DF8163002F075FE02340130E4B23FF4D7
:10C208004DAFBDF81430134AA5F87C309DF81630B0
:10C218009DF814A0D05CF5F7F9FB0223C5F880005F
:10C228000AA995F848008DF828308DF82AA002F060
:10C23800F7FD95F93930069040B29842B8BF1846D4
:10C2480085F83900002204A9092025E7E81C002008
:10C25800241700200B3C010803238DF80D30735D73
:10C268008DF82830E31CDBB2651DF25C231DDBB2C0
:10C278000234F35CE4B21B0443EA0223325D134345
:10C28800642253430B93644B0AA993F8480002F0C5
:10C298002EFEC3B20028EDB28DF80D30FFF66BAE5E
:10C2A8008DF81030012204A90A2035E7092002F090
:10C2B800F9F8DFF868B1002849D00921002002F018
:10C2C800B7F80023ADF81E30A31CDBB2F25CE31C08
:10C2D800DBB216F803A0735D4FEA0A4A4AEA022A5B
:10C2E8004AEA030A231DDBB2A51D0534F35CE4B258
:10C2F8004AEA036A335D4FF47A7253430AAC1B125D
:10C308002046ADF81C3006F04DFF454B53440693CC
:10C31800DBF83C3300930DF1180A9AE80600DBF8C5
:10C32800383308A806F0FBFE099B009394E8060042
:10C33800089B504606F0D8FE9AE8030006F00AFF6C
:10C3480001F00AFF0123EDB28BF8383413E68BF8BD
:10C35800380410E60C2002F0A5F800283FF40BAED4
:10C368000C21002002F064F82C4B93F89034043B25
:10C37800012B7FF600AE01F0EBFEFCE5A31CDBB25F
:10C38800725DF15CE31CDBB2651DF35C0434E4B25E
:10C398001B04305D43EA012313436421594300F031
:10C3A8000F0001F0D6FEEDB28DF81000012204A9AD
:10C3B8001120B1E60D2002F075F800283FF4DBAD3E
:10C3C8000D21002002F034F8A31CDBB2154AF05C02
:10C3D800735D1268251D0334E4B243EA0020315D21
:10C3E800EDB201F0B8FEC6E5725DA31C251D03344D
:10C3F800DBB2E4B2F15C335D1B0443EA012313436F
:10C408006420584301F0A9FEEDB28DF81000012216
:10C4180004A9132080E600BF24170020E81C002090
:10C42800803DD512B81000200E4B93F89124920746
:10C4380003D593F88F24012A08D90B4991F81A21BA
:10C4480022B18A6A501C18BF01328A620022A3F8FE
:10C45800182483F81A24D3F8402322F00202C3F8E0
:10C4680040237047E81C00202417002070B5184CA2
:10C478001848194D06F086FFD4F84033D4F89804CC
:10C48800D5F8906023F02003C4F8403338B106F0A3
:10C498003FFF864203D2002385F83A3070BD012061
:10C4A800FFF766F90028F9D00B28F7D095F839304E
:10C4B80084F84234092094F8183484F8453484F810
:10C4C800410401F0D7FFBDE87040FFF7ADBF00BFE2
:10C4D800E81C00205020002024170020094BD3F826
:10C4E8004023012A0AD008490978C90708D43AB96B
:10C4F80093F89204013818BF012070470020704754
:10C5080001207047E81C0020CC100020034BD3F812
:10C518004003431E58425841704700BFE81C0020A2
:10C528002DE9F04FA9B0EFF3108272B6DFF8F0B240
:10C538000021DBF80030CBF8001082F31088B94CEA
:10C54800002B00F0E180DAB29B06039264D5B64D69
:10C5580095F81831022B02D0B44BDB6A9847EFF3F9
:10C56800108872B6B24F06F0C9FE3E68D4F8B01310
:10C57800361A3144AF4806F08DFFAE4806F050FF3A
:10C58800D4F8B413AC48314406F084FFAA4806F046
:10C5980047FF88F3108894F81A34002B00F06B8159
:10C5A800152312A995F848008DF8483002F038FC98
:10C5B800D4F8B4130F900144A04806F06BFF9F48CD
:10C5C80006F02EFF3B6894F81B24EB620DAF38464B
:10C5D8008DF870201D9306F00BFED5F828310093D6
:10C5E80006AE97E80600D5F82431304606F097FDE8
:10C5F80096E803001FAB83E80300D4F81C341E93AD
:10C6080095F8303195F84800003B18BF01231CA964
:10C618008DF8713002F00DFC039BDF0648D5824D82
:10C62800DFF81CA2D5F8E42004929BF80020BAF9A0
:10C638000A809AF90C90A4F88C84002363F3000212
:10C648000A9384F84434A4F8223484F82534C4F8CE
:10C658002834A4F82C3484F82E34C4F8303484F800
:10C668002034C4F8343484F83834C4F83C346F4B7C
:10C678008BF8002094F89024DB6A84F88E9484F870
:10C688008F24DAF80470BAF80860984794F88F3461
:10C6980013B9694806F076FE3146384601F045FD83
:10C6A8008346002800F0EA80A4F87E8484F8809409
:10C6B800039B19071AD55C4B93F81831022B02D04B
:10C6C8005A4BDB6A98470220FEF712FF84F84104B0
:10C6D80001F0D0FE94F81A3413B1012384F8193408
:10C6E80094F8913443F0100384F89134039B5A076B
:10C6F80003D506210520FEF765FF039B9B0703D59D
:10C7080004210320FEF75EFF01F02DFD94F891242B
:10C71800D7065FD5002384F89234D4F840331E0638
:10C7280044BF23F08203C4F8403312F0050F00F031
:10C73800FB820B2001F0B6FE002800F0F58294F889
:10C748009134DD0700F1F082580740F10783D4F8EF
:10C75800403323F00203C4F84033D4F8402382BBAB
:10C7680094F8915415F001011EBF2B4662F30003A3
:10C7780084F8913494F891345E0744BF6FF38203D0
:10C7880084F89134012384F8923421B1D4F84433E5
:10C798002C481B6898476D070BD52B4801F08EFE77
:10C7A80001F0BCFE28B194F8913443F0040384F8F6
:10C7B800913401F0C6FC94F891346FF3041384F8B3
:10C7C8009134012384F8923494F8913443F020038F
:10C7D80084F8913494F8913418070AD56FF3C30399
:10C7E8001A4984F89134D4F84433A1F12400DB6861
:10C7F800984794F8913499070AD56FF34103134980
:10C8080084F89134D4F84433A1F16C005B689847FC
:10C8180094F89034022B1BD1FFF722F918E000BFDF
:10C82800CC100020E81C0020241700200443010835
:10C83800C81000206820002080200020E820002068
:10C84800B8100020282100203C210020742100205D
:10C8580094F891349A0640F1C4826FF3451384F832
:10C868009134D4F84033002B40F0BB8229B0BDE8A6
:10C87800F04FFFF7ABBA84F84134A3E695F81831C6
:10C88800012B0CD101F055FC804668B1584601F0E7
:10C8980045FC584601F047FC042384F88F347EB9E0
:10C8A800012384F821344FE101F045FC0028F6D03B
:10C8B800404601F034FC404601F036FC0523ECE725
:10C8C8003B7805935B09013B062B00F21782DFE8F2
:10C8D80013F00700150295001502920015020602D2
:10C8E800102EDDD995F830311297F6B28DF84C60DC
:10C8F800002BD5D11CA804F055F912AA1CA9FF20B9
:10C9080002F09EF89DF85830C3F3030307468DF8EC
:10C918002C3095F8480095F87D308DF82D30072299
:10C928000BA902F090FA002F5DD100285BD09DF88A
:10C9380053309DF852201599C5F8E4101B0443EABA
:10C9480002239DF8512002201343C5F8E03004F07B
:10C9580037F99DF8583095F8480085F82E71C3F3DB
:10C968000212C3F3030385F8703085F878309DF818
:10C97800593085F86920012B38BF01234FF47A72AA
:10C988005343AB651344EB650DF15A034FF00108AF
:10C998001093113E94F81B348DF83C300FA985F89C
:10C9A80068808DF8446002F056FA0223404685F804
:10C9B800303101F077FD18B14146384601F038FDB5
:10C9C80094F88F34012B00F2A78194F81A34002BC5
:10C9D80040F09A8194F8913443F0100384F891342C
:10C9E800FEF786FD64E6012001F05CFD0028E7D033
:10C9F80001210720E2E7012384F8203495F87D30EF
:10CA08008DF82E3094F824348DF82D3095F88C302C
:10CA180095F848000D330BA98DF82C3002F000FA78
:10CA2800A6F10D031BB2099023EAE37300B2834217
:10CA38003FF736AF0B2E7FF633AFBA4B25931CA8C2
:10CA4800FF231C978DF874608DF8983002F0C4F8B5
:10CA5800074600287FF424AF95F81831012B13D12D
:10CA680001F067FB002872D0384601F057FB3846C2
:10CA780001F059FB04239DF87C101E9884F88F342C
:10CA8800C1F3001101F06EFB9DF87C301E99C4F8CB
:10CA9800341413F00F0203D09DF89000002862D1DF
:10CAA8009DF89800002861D0002A7FF4F9AE9DF81F
:10CAB8009020002A14BF4FF003084FF0020800220C
:10CAC8000A92D5F8EC2095F8E900914251D1002856
:10CAD8004FD0D5F80C1195F8EAB009680A9195F885
:10CAE8001811022902D1032184F88F14B8F1030F19
:10CAF8007FF4D6AE13F0600F7FF4D2AE0492012714
:10CB080095F82E31BBF1000F36D0BBF1010F13D1D0
:10CB1800012B33D16FF0090646FA08F606F0010634
:10CB2800C6F10206F6B2BDF87E100AAA304601F038
:10CB380011FE38B3072823D0012384F821340A9B37
:10CB4800C4F83034C4F86C34FEF720FDB0E501F0C9
:10CB5800F2FA002898D0384601F0E1FA384601F098
:10CB6800E3FA052387E74FF00008A8E74FF001082C
:10CB7800A5E74FF0010BC3E70426D4E70326D2E765
:10CB88000823DAE71CAB009304990A9B32465846FF
:10CB980001F0A2FE20B1022814BF0B230A2380E66D
:10CBA8000A9BC4F83034C4F86C349DF87C3084F89F
:10CBB8002104C3F3401384F82E3484F8443494F8E1
:10CBC8008F3484F82274012B9EBF0122A86285F855
:10CBD8001E21012FC4F8280484F82C0484F8410489
:10CBE80038D1022284F8202495F83A20002A4AD124
:10CBF8009DF87C20D60646D4012B94F840149DF865
:10CC08007C2005D8012901D1900601D501F04CFB03
:10CC1800B8F1020F94F88F3443D0B8F1030F0AD05B
:10CC28009DF87C10B8F1010F4A4601F00F0120A8C9
:10CC38003BD0FFF745F99DF8903084F82334259BC5
:10CC4800C4F828349DF8983084F82C34012384F8EB
:10CC58002D3430E0059A02F0E002A02A1BD195F8A5
:10CC68002E11012285F83A2009B927996963012B09
:10CC780084F8202407D9D5F89020C4F83C24DAF8A1
:10CC88000020C4F8982495F81821002AB4D101226C
:10CC980084F82524B0E7002285F83A2084F8202477
:10CCA800A6E79DF8981025984A46FFF709F99DF8D8
:10CCB800903084F823349DF89020E02A08D195F824
:10CCC8001F312BB984F82324C4F82834A4F82C3451
:10CCD80094F8913443F0020384F8913470E6114DCE
:10CCE800013EB2B2791C284604F034F80323A4F8B4
:10CCF8002034C4F8285484F82C64E9E7012384F824
:10CD08002134FEF743FC5BE694F84434002B3FF4EF
:10CD180061AE0020FEF726FC94F88F34022B3FF416
:10CD28005FAE57E6201F002094F89134590715D5B7
:10CD3800012001F0B7FB60B1012001F08BFB08B9BD
:10CD480084F81804D4F8403323F00203C4F84033BD
:10CD580004E0062001F0A6FB0028F3D194F89134F2
:10CD6800DA077FF5FAAC94F840240AB1032A18D1FF
:10CD78001D4A94F8181492F86820914205D29B072E
:10CD880023D594F88F34012B1FD8184806F0FAFAE7
:10CD9800D4F8403323F02003C4F84033FFF744FBB2
:10CDA800DBE4012A11D194F81924002A3FF4D5AC08
:10CDB8000D4A94F8181492F868209142E5D29F071A
:10CDC80003D594F84434002BDFD194F89134002033
:10CDD8006FF3041384F8913484F81904FFF746FBC1
:10CDE800BBE429B0BDE8F08F2417002050200020B4
:10CDF8002DE9F04F89468DB090460746002800F08F
:10CE08008F81002900F08C810368002B00F0888155
:10CE18004368002B00F084818368002B00F0808138
:10CE2800C368002B00F07C81104601F0F5FF002854
:10CE380000F07881BD4CBE4D384601F0AFFA40F2A3
:10CE4800C4520021204603F099FF40F21C520021F1
:10CE5800284603F093FFB74BC4F82C3104F5097347
:10CE6800089304F50A7300264046099308A9B24BB3
:10CE780084F848800A9384F8186184F88C608DF8E7
:10CE88002C6001F0DBFF0F2306A994F848008DF809
:10CE9800183001F0C5FF801B18BF01204FF00A0BA6
:10CEA80084F81C0106A994F848008DF818B001F020
:10CEB800B7FF4FF0060A84F8DC0006A994F848008A
:10CEC8008DF818A001F0ACFF102384F8DD0006A946
:10CED80094F848008DF8183001F0A2FF1123C4F827
:10CEE8009C0006A994F848008DF8183001F098FFC6
:10CEF8001223C4F8A00006A994F848008DF8183049
:10CF080001F08EFF1323C4F8A40006A994F8480082
:10CF18008DF8183001F084FF1423C4F8A80006A97E
:10CF280094F848008DF8183001F07AFF1623C4F8F9
:10CF3800AC0006A994F848008DF8183001F070FF8D
:10CF4800172384F8B10006A994F848008DF8183022
:10CF580001F066FF18230DEB0301C4F8B400C4F810
:10CF6800BC0094F848008DF8183001F059FFC0B2A1
:10CF78001D2384F8B80084F8C00006A994F8480076
:10CF88008DF8183001F04CFF1E2384F8C40006A960
:10CF980094F848008DF8183001F042FF1F2384F8F8
:10CFA800C50006A994F848008DF8183001F038FF3C
:10CFB8002023C4F8C80006A994F848008DF8183052
:10CFC80001F02EFF0B23C4F8CC0006A994F8480002
:10CFD8008DF8183001F024FF0C2306A9A4F8D0001E
:10CFE80094F848008DF8183001F01AFFD4F89C30F6
:10CFF8006365D4F8A030A365D4F8A430E365D4F809
:10D00800A83023664FF00108D4F8AC300590A4F896
:10D01800D200636684F8B080C4F894B084F898A00D
:10D02800C4F84CB084F850A084F8688084F81F8154
:10D03800C5F84893FEF7AEFDC5F84473C4E90B661E
:10D048003E4B84F8198185F89164C5F840833246CF
:10D058004FF0FF31009605F55A7006F035F9384B58
:10D06800009632464FF0FF3105F5607006F02CF956
:10D07800344B009632464FF0FF3105F5667006F0E6
:10D0880023F902AF304B009632464FF0FF3105F5D9
:10D09800806006F019F9384606F0AAF897E8030008
:10D0A80004F5927383E80300284B294F1E60294B2F
:10D0B800C5F84C33284BC5F85433284BC5F85C33B6
:10D0C800274BC5F85033274BC5F8583305F553702F
:10D0D8003B68984704F5A67003F080FB20B1112641
:10D0E80030460DB0BDE8F08F204601F003FB002864
:10D0F800F5D101F039F8B8B91B4801F04DFB0646E7
:10D108000028ECD17B69984703F002FEBB6D94F8C8
:10D1180019019847FB6A9847012385F89234DFE79D
:10D128000326DDE70926DBE71326D9E724170020C5
:10D13800E81C002000040001D010002075C400087D
:10D148003DBD000885BD00086DB50008CC10002065
:10D15800044301082DB70008E1B6000829B5000806
:10D16800B9B6000891B600080C18002008B5034BA2
:10D178000020C3F84003FEF7BBF908BDE81C0020F7
:10D1880010B5FFF7ABF90A4C60B90A4B93F81831A0
:10D19800022B02D1084BDB6A98470123C4F84033BD
:10D1A800002010BDD4F84003013818BF0120F8E76B
:10D1B800E81C0020241700200443010838B5124C4D
:10D1C800204606F0DFF804F1180006F0DBF804F159
:10D1D800300006F0D7F804F1980006F0D3F800F014
:10D1E800AFFF0A4B0025DB6A984744F8285CFEF736
:10D1F800EDFD0749074840F2C45203F0ABFD012397
:10D2080044F8283C284638BD502000200443010833
:10D21800241700206011002070B52E4B8AB00546F7
:10D2280093F8DD008DF8090093F8DC008DF80A000A
:10D2380029489A6A90F81804039200268DF80B0082
:10D2480004960C46002940D00692D3F8882007920D
:10D258001A8F93F81A118DF8151052BAADF82020CC
:10D2680093F87C2093F848308DF8243003AB8DF880
:10D2780022008DF8232000930DF10A020DF10B0313
:10D288000DF1090105A88DF8146000F0D7FE9DF98D
:10D298000900FEF74FF9607004A801F01BF8B0B957
:10D2A800049A0F2A0DD863789A420AD81544AB42DB
:10D2B800A3EB02012CBF002001202170C0000AB09E
:10D2C80070BD002323700820F9E70320F7E7132037
:10D2D800F5E700BF24170020E81C00201FB504460E
:10D2E800002800F010810378412B00F20781DFE865
:10D2F80013F0420049004D005100550059005E00EE
:10D3080005010501050105010501050105010501E5
:10D31800650069006D0078007F00820085008A0042
:10D3280088008C0090009300960099009C009F0054
:10D33800AE00B200BA00B600BE00C100C500CE0003
:10D34800CA00CC000501D20005010501050105014F
:10D358000501050105010501050105010501050195
:10D36800050105010501DA00DE00E200E700EB0037
:10D37800EF00F300FC00664B93F81831237100208E
:10D3880004B010BD624B93F83031F7E7406803F002
:10D39800C3FBF4E7406803F005FCF0E75C4B93F847
:10D3A8001A31EBE75A4BD3F8E0306360E7E7584BA4
:10D3B800011D93F8300103F00DFCE0E7544B93F89E
:10D3C8001931DBE7524B93F88C30D7E71C238DF8E3
:10D3D80008304F4B02A993F8480001F021FD606026
:10D3E800CDE74C4B043493E8030084E80300C6E718
:10D3F800494B0434F7E7494B0434F4E7484B043409
:10D40800F1E71A23E3E71923E1E7414B93F8683082
:10D41800B4E73F4B5B6DC8E73D4B9B6DC5E73C4BA5
:10D42800DB6DC2E73A4B1B6EBFE7394B5B6EBCE75F
:10D4380002238DF80830364B02A993F87C2093F824
:10D4480048008DF80A2001F0EBFC207197E7304B7B
:10D4580093F8DD3092E72E4B93F839308EE72C4B5A
:10D4680093F8DC308AE72A4B93F8383086E7284B64
:10D47800DB6C9AE7264B93F850307FE7244BD3F8C0
:10D48800843063607BE7224B8FE7264B8DE7204B88
:10D49800D3F8CC30F5E71E4BD3F82C31436001F0BC
:10D4A8004DFDA0606BE71A4BD3F890307DE7184B21
:10D4B80093F81F3162E7164BB3F88830A3805EE714
:10D4C800134BB3F88A30F9E7114BB3F8D030F5E7CE
:10D4D8000F4BB3F8D230F1E70D4B93F848200AB15F
:10D4E800062A12D1B3F8A035E8E7094B93F848208B
:10D4F8000AB1062A09D1D3F8A43556E704B0BDE825
:10D50800104000F021BE03203AE7182038E700BF9A
:10D518002417002090170020D81700209817002003
:10D52800E0170020601100207FB5044610B90320E1
:10D5380004B070BDA34DD5F840339A0700F16F824F
:10D548000278412A00F26882DFE812F042004700C0
:10D5580055005B005F006400690076008100870069
:10D568008D00930099009F00A500AB00B5006602EE
:10D57800BA00DC00EF0016013801290142014B0115
:10D588004F01530157015B0166025F017101990167
:10D598008701AB01B101B801BD01C20166022802D1
:10D5A8006602660266026602660266026602660233
:10D5B8006602660266026602660266026602660223
:10D5C800340239023E02430248024D0252025C0212
:10D5D8000079FEF773FA30B1AAE70379022BA6D0D7
:10D5E800794A82F8303195F8913443F0200385F870
:10D5F800913400209CE7406803F080FA0028F2D0BC
:10D6080095E7406803F0BEFAF8E76F4B027983F8B4
:10D618001A21E8E76C4B4268C3F8E020E3E76A4E5A
:10D62800416896F8300103F0CBFA00287FF47FAF09
:10D638006368C6F8E430D6E7416800293FF477AF5D
:10D64800002001F0DDF90028CDD0112070E74168F5
:10D6580000293FF46CAF0120F3E7416800293FF44B
:10D6680066AF0820EDE7416800293FF460AF092064
:10D67800E7E7416800293FF45AAF0C20E1E7416829
:10D6880000293FF454AF0D20DBE7416800293FF43F
:10D698004EAF0E20D5E7416800293FF448AF0F2070
:10D6A800CFE74A4C484B007983F81901A36D984796
:10D6B800E36A984797E7444B027983F88C2092E70E
:10D6C800414E037A8DF8043096F8480096F87D307C
:10D6D8008DF80530072201A901F0B5FB00283FF4B9
:10D6E80026AF636896F848000193002201A901F06B
:10D6F800AAFB00283FF41BAF6C36D4E9010186E889
:10D70800030070E7304E037A8DF8043096F848002D
:10D7180096F87D308DF80530072201A901F093FBBA
:10D7280000283FF404AFB436E7E7274E037A8DF8B4
:10D73800043096F8480096F87D308DF805300722B9
:10D7480001A901F080FB00283FF4F1AED4E9010102
:10D7580006F1740383E8030096F81831022B7FF46E
:10D7680042AF96F83031002B3FF43DAF174BDB6AE0
:10D778009847FEF775F936E7134E037A8DF80430AB
:10D7880096F8480096F87D308DF80530072201A9F3
:10D7980001F059FB00283FF4CAAEBC36ADE7436838
:10D7A800029301238DF80C30074B02A993F8480027
:10D7B80001F056FB00287FF416AFB8E643680293E1
:10D7C8000023EFE7E81C0020241700200443010889
:10D7D80003795A1E0E2A3FF6AAAE934A82F8683099
:10D7E80001E7914B42685A65FDE68F4B42689A659E
:10D7F800F9E68D4B4268DA65F5E68B4B42681A66A6
:10D80800F1E6894B42685A66EDE6874C037994F84D
:10D8180048008DF80430062201A901F014FB002805
:10D828003FF485AE9DF8043084F8DD30DBE67E4CAD
:10D8380003798DF8043094F8480094F87C308DF81A
:10D848000630052201A901F0FEFA00283FF46FAE68
:10D858009DF8043084F83930C5E6734C037994F8A0
:10D8680048008DF804300A2201A901F0ECFA0028DA
:10D878003FF45DAE9DF8043084F8DC30B3E66A4CC2
:10D88800037994F848008DF80430092201A901F0C1
:10D89800DAFA00283FF44BAE9DF8043084F83830AB
:10D8A800A1E6614B4268C3F89420DA649BE65E4BBC
:10D8B800027983F8982083F8502094E65A4B4268FE
:10D8C800C3F884208FE6584B4268C3F8CC208AE618
:10D8D800012B40F0A480554C2421204603F050FA37
:10D8E800636A984201D0172022E61C2104F128001F
:10D8F80003F046FA636C9842F5D14FF4807104F155
:10D90800480003F03DFAD4F848319842EBD1D421CD
:10D9180004F5A67003F034FAD4F820329842E2D124
:10D92800002104F5097003F02BFAD4F82432984248
:10D93800D9D14FF4607104F50A7003F021FAD4F8D4
:10D94800A8359842CFD1142104F2AC5003F018FA4C
:10D95800D4F8C0359842C6D1334E2146304640F2FD
:10D96800C45203F0F7F9204640F2C452002103F0F4
:10D9780005FA95F81B3485F8E833736FC5F8EC336E
:10D9880096F87D3085F8F83340F20123A5F8FA338C
:10D99800274B96F819019B6D984724E68379012B4C
:10D9A8003FF6C5AD204B42684068C3F82C2100F013
:10D9B800BDFE48E61C4B4268C3F8902013E61A4B9C
:10D9C800027983F81F210EE6174B8288A3F8882076
:10D9D80009E6154B8288A3F88A2004E6124B828850
:10D9E800A3F8D020FFE5104B8288A3F8D220FAE5EF
:10D9F8000D4B93F848200AB1062A12D1A288A3F841
:10DA0800A025F0E5084B93F848200AB1062A08D16A
:10DA18006268C3F8A425E6E500F098FBDBE5012081
:10DA280086E5182084E500BF241700206011002037
:10DA3800044301082DE9F04387B00023ADF8003016
:10DA48000646002800F0EE800361FEF747FD20B18E
:10DA58000124204607B0BDE8F08300F065FD0028EA
:10DA6800F6D100F05BFD014618B96F48142203F0A7
:10DA780085F96E4D95F89134012243F0040385F839
:10DA8800552485F8913433788DF804300021013B12
:10DA98008DF80520ADF806100C2B00F2BB80DFE8EE
:10DAA80003F007B9B9B97982B9B990B9AD9AA900A3
:10DAB800D5F8407317F02007CAD196F80480B8F15A
:10DAC800020F46D1DFF868815A4CFEF763F896F9E1
:10DAD800051098F848003A4601F00FFA88F839001E
:10DAE800B37988F83830384607238DF80530FDF7C4
:10DAF800E5FFFF2304F58670A5F80C31C5F8084149
:10DB080085F8047103F04EF804F58A7003F004F800
:10DB18003846FDF72DFE0446002839D096F9051041
:10DB280098F84800012201F0E8F988F83900D5F89A
:10DB380094343361002C71D000F0F0FC002888D1B7
:10DB480095F8913485F81A0460F3820385F89134C6
:10DB58007FE7B8F1010F4FF00204E8D1DFF8D09069
:10DB68008DF8144099F8480089F81D7102A901F050
:10DB780065F9337989F830318DF805708DF80680AC
:10DB8800FDF7C4FC95F8913443F0100385F89134FF
:10DB98000024CCE700226946022000F0F3FA0028AE
:10DBA800F6D01324C3E7244BB288DB6B96F90C102C
:10DBB800B0689847D5F8403343F00203C5F84033BE
:10DBC800E6E702A90D2000F053FB0028E0D0002270
:10DBD80069460D20E1E7164B93F81831D3B934792B
:10DBE80004F0070000F0ABFA8DF800400122694606
:10DBF8001020D2E7002269461220CEE78DF80720D0
:10DC080000F08EFA044638B900F087FA204600F092
:10DC180089FABDE702248AE7012488E701A800F011
:10DC2800D1FB16E7032414E73C210020E81C002060
:10DC380024170020EA1C0020044301082DE9F04FB6
:10DC480099B08046059118B9032019B0BDE8F08F46
:10DC580000230361FEF742FC0446002840F0A5803B
:10DC680046460FCE0EAD0FC51422524898F800A0B4
:10DC7800B8F80C7098F90EB04F4E214603F07EF8B4
:10DC88004E4B012283F8412496F83021022A25467A
:10DC98000BD196F81821022A07D196F81E2122B92D
:10DCA800BAF1010F38BF4FF0010ABAF1010F2BD0BA
:10DCB800BAF1030F2AD0BAF1000F33D102229DF82E
:10DCC8003C30DDF84090029362F34715012496F842
:10DCD8007C108DF8321002220CA996F848008DF8B5
:10DCE800302001F09DF896F81A3196F830C196F870
:10DCF8001D1140B2002B63D0BCF1010F57D1002990
:10DD080055D1002C61D153E00422D8E70023DDF877
:10DD18003C90BDF840709DF942B0029365F01F0534
:10DD28000124D4E74FF0000BD946CDF808B0CEE770
:10DD38004FF0010084F81A04D2E005F29A420BA9C8
:10DD480000F0D4FA002800F015811320049B3387D3
:10DD58001A4B002283F81A2423E105F29A452A4631
:10DD68000BA900F0C3FA0028EFD10B9B84F8280117
:10DD7800C4F82C5184F83031FCE0B9F1000F00F000
:10DD8800F980002A00F0F6804946E01C02F0E2FF24
:10DD980094F8373201332380ECE01220D6E70220D2
:10DDA800D4E70720D4E71320D2E701204DE7FCB9D8
:10DDB8000220F6E02821002024170020E81C00207B
:10DDC800002CF5D05845B8BF584696F87C308DF8E9
:10DDD8002000052296F848008DF8223008A901F0A5
:10DDE80032F800283FF430AF9DF8203086F83930FB
:10DDF8006F4A704BD2F89804D3F8904038B105F0C8
:10DE080087FA6C4B84423CBF002283F83A20198F72
:10DE18001A8F93F830010491996A099152BA00282F
:10DE2800BFD093F81B0100B9186393F81801ADF837
:10DE38005820013893F87C2093F81A411491D0F1B6
:10DE4800000BD3F888108DF85B204BEB000B93F890
:10DE5800482093F83A0093F868308DF85A3009ABA7
:10DE68000093554B03904FF001008DF84C0015912D
:10DE78008DF85C20A3F12F01A3F1300213A88DF8CF
:10DE88004D4000F0DBF8039B4FEA0B1B4BEA431BAA
:10DE980000264BEA801B4BEAC413B145444C03935C
:10DEA80008BF37463A46494604F59C70CDE90A66EC
:10DEB8009B46268084F81A6402F04CFFE9B2A570EC
:10DEC800C5F34215FAB2042D3A4E039B84F8372263
:10DED8003FF42EAF072D3FF450AF022D7FF45FAF14
:10DEE800364D84F80D110420029984F80401FF20AE
:10DEF80084F80C0184F8281184F81431D6F8E41059
:10DF0800C4F8085105F59B730AA8C4F8101184F8E1
:10DF18003021C4F82C3100F011FC00287FF43DAF0B
:10DF28000A9BA4F844040BA8A4F81631C4F84C348E
:10DF380000F0D0F900287FF408AF0B9BD3B196F915
:10DF48003900FDF7F7FA94F83732002B3FF405AFA4
:10DF58000B9B0F2B3FF6F1AE05F58B720BA90F202B
:10DF680000F0C4F900287FF4F0AE0B9B63F3030BB9
:10DF780084F814B10598FDF7FBFB00287FF4E6AEA2
:10DF8800099B86F83A00B36200F080F900287FF414
:10DF98000AAF94F8913484F840A443F0010384F85C
:10DFA8009134034BD3F89434C8F810304DE600BFD1
:10DFB800E81C0020241700208C170020EA1C0020F1
:10DFC80037B50B4D8DF8040004460F2295F848002C
:10DFD80001A900F038FF40B1064A85F81C4192F8C3
:10DFE800913443F0200382F8913403B030BD00BF70
:10DFF80024170020E81C002010B5FFF7C1F80446DC
:10E0080088B90A4805F0BEF9094805F0BBF909487E
:10E0180005F0B8F900F094F8FDF7BCFD064BDB6A93
:10E028009847204610BD0124FBE700BF5020002080
:10E038006820002080200020044301082DE9F04FCB
:10E048008BB047780093149B90F90C8090F90D6081
:10E0580090F80EB08A464168196004469146002F30
:10E0680058D002238DF8103004A9C37B007C8DF8AA
:10E07800123000F0D5FEB4F808C0618943B2606878
:10E08800984545466144B8BF1D46604534BF0027E2
:10E098000127884209D30A218DF81010207C0193AA
:10E0A80004A900F0BDFE019B46B2B4F808C060891F
:10E0B80061680CEB400E714519D3A1EB0C01B1FB63
:10E0C800F0FC00FB1C1191B9984503DC2378CBB90F
:10E0D8004FF0010B21238DF81030207CE37B8DF865
:10E0E800115004A98DF8123000F09AFE45B2009B39
:10E0F8008AF80050384689F8006083F800B00BB001
:10E10800BDE8F08F0223207C8DF8243006A900F0AA
:10E1180095FEDDE74546EAE7704770477047704768
:10E1280000207047704770477047002070470020F4
:10E1380070470020704700207047002070477047E4
:10E1480070477047022070470220704702207047CE
:10E1580070470020704770477047002070470020C4
:10E16800704770477047704710B5054C4FF40372FD
:10E178002046002102F002FE0020C4E9000010BD84
:10E18800042200202DE9F8438146904600293CD01E
:10E198001F4C2023224604F1100012F8017F6FBBA8
:10E1A8008242FAD11B4E3368013403B93460736874
:10E1B80003B11C6000252560C4F8088074601FFA4C
:10E1C80088F284F80490601D02F0C4FDB9F1110FC3
:10E1D8004FF0000398BF104D6373D6F8083298BF0C
:10E1E80025FA09F503F1010398BF05F00105434439
:10E1F8002573C6F808323846BDE8F883013B13F0AA
:10E20800FF030446C6D10227F5E70127F3E700BF5D
:10E218000B220020042200202007020010B518B3AA
:10E22800124A1368984204D103681360002305E07A
:10E238000B46002BFAD019688842F9D151688842F8
:10E2480008BF53600BB101681960D2F808328168C1
:10E25800013B00245B1A04602146C2F808321022F0
:10E2680002F08CFD204610BD0120FCE704220020AE
:10E27800054B1B6813B11A798242FAD1002B0B6047
:10E288000CBF0320002070470422002010B5054B66
:10E29800186800B910BD037B04680BB9FFF7BEFF0F
:10E2A8002046F6E70422002038B5084B084C1868C9
:10E2B80000B938BD03790568112B05D824FA03F392
:10E2C800DB0701D5FFF7AAFF2846F1E70422002063
:10E2D8002007020028B1044BD3F80832036000205D
:10E2E80070470120704700BF042200202DE9F0414B
:10E2F80007460E46154642B339B3154B1C68002332
:10E308002CB93046FFF7E6FF0020BDE8F081A2688F
:10E31800F91A0132914215D32279EA54581C2289FC
:10E328005FFA80F8611D55FA80F002F013FDA368CA
:10E33800246898445FFA88F3E2E720462568FFF7E7
:10E348006DFF2C46002CF8D1DBE70120DDE700BF8C
:10E35800042200200238C0B211289ABF014B185C71
:10E36800002070471B3C010830B50B4B93F8202068
:10E378000446084672B100211C330578A54208D02E
:10E3880001319842CDB214BF04301038AA42F4D8F3
:10E39800002030BD1046FCE71024002010B5084CC2
:10E3A80000232060142204F10C00FF2184F820309F
:10E3B800C4E9010002F0E2FC012384F8213010BD19
:10E3C8001024002010B50E4A92F82010042915D800
:10E3D800936804781C7044785C70C478807898706E
:10E3E8000131DC7082F8201002F11C018B4214BF4D
:10E3F800043302F10C039360012010BD0020FCE7F8
:10E4080010240020094B93F8200068B15A6803F1E2
:10E418001C018A4200F1FF3014BF043203F10C02E0
:10E4280083F820005A600120704700BF10240020A4
:10E4380010B5074B93F820200446084632B15968B6
:10E44800FFF792FF10B101234470837010BD00BF25
:10E458001024002008B5064B93F820202AB15968EB
:10E46800FFF782FF08B1407808BD0120FCE700BF34
:10E478001024002030B50A4A92F82010536882F818
:10E48800210061B1916801241C32DD78587005B90A
:10E498009C70934214BF0433103B9942F5D130BDB0
:10E4A8001024002008B5044B5968FFF75DFF0038B9
:10E4B80018BF012008BD00BF10240020F7B50422B2
:10E4C800154E044600210DEB020096F8207002F06C
:10E4D80055FC0025EBB29F4201D803B0F0BD73682C
:10E4E800197821705A786270987838B13368204664
:10E4F8009B689847FFF786FF0135EBE7DB788DF8D7
:10E5080004108DF805208DF80730FFF77BFF01A870
:10E51800FFF758FFF0E700BF10240020014B93F8E5
:10E528002000704710240020034B93F82000042893
:10E5380094BF002001207047102400201FB500243C
:10E54800CDE90244C41F8DF800408DF801100C0A73
:10E55800ADF80420090C120C8DF803108DF8062074
:10E568008DF8073002461B0A012168468DF80240E3
:10E578008DF8083002F05DFA002818BF0E2004B0AC
:10E5880010BD2DE9F04188B090460D460F9A074618
:10E59800002847D000240121CDE904448DF810104B
:10E5A8009DF838108DF81510ADF81630190CCDE916
:10E5B80000441B0ECDE902448DF81930ADF81A203D
:10E5C800130C120E07948DF818108DF81C308DF866
:10E5D8001D20E3B21E01002DF6B203DC002008B0B6
:10E5E800BDE8F081013310218DF81F3042466B469B
:10E5F8000DEB010002F0B3F90346A8B9102D284627
:10E608003E44A8BF10206946327811F801CB013387
:10E6180082EA0C02984206F8012BF5DC103D2DB277
:10E628000134D6E70920DAE70E20D8E701380328B5
:10E6380015D8DFE800F002080C100A4B1B681B69AC
:10E648000B6000207047074B1B685B69F8E7054BB8
:10E658001B689B69F4E7034B1B68DB69F0E705203F
:10E66800704700BF342400202DE9F041C4B00C46A7
:10E678004A9E17461D468046B8B3B1F5807F36D806
:10E688004FF488720021684602F078FB4923009312
:10E698004FF48073ADF804302B0C8DF80830330C30
:10E6A800ADF80650ADF80A608DF80C30224600230C
:10E6B800414604A82D0E360E8DF80E308DF80950FF
:10E6C8008DF80D608DF80F4002F044FB04F1100145
:10E6D8004B9A3B4689B2684602F02BF910B10128E3
:10E6E80018BF0E2044B0BDE8F0810920FAE70D20DC
:10E6F800F8E7000010B590B10A4C282200212060EC
:10E7080002F03CFB2368084A1A6000204FF0FF32F1
:10E71800C3E90302C3E90522C3E9072210BD0820A3
:10E72800FCE700BF3424002000010101024B1B68F4
:10E7380018600020704700BF3424002030B1044B1B
:10E748001B68DB68013303600020704709207047AD
:10E758003424002013B500230C460193CAB101A943
:10E76800FFF764FF18B9019B591C02D1146002B06D
:10E7780010BD99B2611A002901DD5C18F6E702D1D3
:10E7880013600720F3E71B0C1B0403F580331C44BC
:10E79800ECE70920EBE7000028B1044B1B681C33A9
:10E7A8004362002070470920704700BF34240020CE
:10E7B8001FB5044600B3002303A8039302F090F9A1
:10E7C800104ABDF80C30126820469380E38200F0AE
:10E7D8005EFA98B904F11803009321680123132203
:10E7E80002F09CF860B9204600F051FA003818BFD2
:10E7F8000120000104B010BD0920FBE71020F9E753
:10E808000E20F7E734240020F0B5054687B01C46F3
:10E8180013B9092007B0F0BD2E4E3368DB68834278
:10E8280055D894F82020002A0CBF082209228342D8
:10E8380005D3204600F05FFA68B11020EAE700230C
:10E8480001900093A36894F82810606AFFF799FE76
:10E858000028EED0DEE723792168B4F808C0A7685D
:10E86800043B9AB20029D4D0B2F5807F2DD8ADF8F8
:10E878000EC08DF817304FEA174C04F12C033F0EE9
:10E888008DF8117000932F0C08234FF0490EADF846
:10E898000C008DF814708DF816002F0E0DEB030088
:10E8A800CDF808E08DF810C0ADF812508DF815704D
:10E8B80002F034F808B10E20ACE7204600F01BFA4D
:10E8C8000028BAD13368DD60A4E70D20A2E706204E
:10E8D800A0E700BF342400202DE9FF410A9D8046AF
:10E8E8000F4616461C46002D5AD0002303A9104691
:10E8F8000393FFF79BFE18B1062004B0BDE8F08132
:10E90800039B9C4201D80133F6D1284600F064F9F4
:10E91800002847D1264B1A78424503D01A79424538
:10E9280042D10120AA68BA4240D103EB8002EB6AC7
:10E9380092F801802979CDE9004304399278286852
:10E948003B4689B2FFF790FE0028D6D195F82030D3
:10E958000194002B4FF00103009314BF4246082294
:10E9680095F82810686A3B46FFF70BFE0028C4D1CB
:10E97800013E032EC1D8DFE806F002070B0F0D4B4E
:10E988001B681C611C62B8E70A4B1B685C61F9E7ED
:10E99800084B1B689C61F5E7064B1B68DC61ACE71C
:10E9A8000920AAE70F20A8E70B20A6E70220A4E782
:10E9B800A4080020342400201FB50B294FF00003C1
:10E9C800CDE90033CDE902330A4607D00C2914D02B
:10E9D8000A2910D00A2005B05DF804FB012802D1ED
:10E9E80020238DF800300021684602F022F8002824
:10E9F80018BF0E20EFE73023F3E70B21F4E7000000
:10EA080038B5054602F010F8044610B10E24204629
:10EA180038BD002DFBD1094B1B680B219878FFF7F7
:10EA2800CBFF0028F2D10C21FFF7C6FF0028EDD15B
:10EA38000A21FFF7C1FF0028E9D0E7E734240020C6
:10EA48002DE9F04380468FB00C461746002A6BD05C
:10EA5800002969D0002529461D2206A8059504F03D
:10EA6800A7FE8DF81350344D2B680DF114099E88BC
:10EA7800CDF804900DF1130302933B7900933B68A2
:10EA880032462146404601F0F0FF00284ED1386852
:10EA98003A79494602F05EF9384600F04FF8002806
:10EAA80046D13C7AFA79BB79240444EA02241C430F
:10EAB8002B689A6894423DD99C609DF813000B21FD
:10EAC800FFF77AFF034658BB0C21FFF775FF034693
:10EAD80030BB0A21FFF770FF034608BB7B7ABA7A7E
:10EAE800FF7A3F0447EA02271F433A463346214646
:10EAF8000920FFF723FD034690B933463A462146DD
:10EB08000820FFF71BFD034650B92A689DF813102B
:10EB180091700021D1604FF0FF31C2E90411916179
:10EB280018460FB0BDE8F0830923F9E70E23F7E78D
:10EB38000F23F5E70323F3E73424002010B5044638
:10EB4800002845D00168002942D011F8013B4371E3
:10EB58000322063002F0FEF82046032250F8091B73
:10EB6800043102F0F7F82168CB79E3600A7A43EAC6
:10EB78000223E3604A7A43EA0243E3608A7A43EA7B
:10EB88000263E360CB7A23740B7B63742379212BB4
:10EB98001AD110220D3104F1120002F0DBF81D2207
:10EBA8002168501C8B5C6362085C43EA0023901C5C
:10EBB8006362085C033243EA004363628A5C43EAA7
:10EBC80002636362002010BD112B03DC0D22E7E70E
:10EBD8000220F8E70120F6E710B50446002854D0D3
:10EBE8000168002951D00B7843714B7883608A788B
:10EBF80043EA02238360CA7843EA024383600A79BE
:10EC080043EA026383604B7903738B79C381CA79C2
:10EC180043EA0223027BC38102F00F02083110305D
:10EC280002F098F8237B002203F00F0384F82020D9
:10EC380084F82820227903F10800111A04290DDD2F
:10EC480021680933043AD21A085C84F82000D2B249
:10EC5800606A84F82820194402F07CF82379226835
:10EC68001A44002012F8043CE36212F8031C43EA39
:10EC78000123E36212F8021C43EA0143E36212F83B
:10EC8800012C43EA0263E36210BD0220FCE710B5E1
:10EC9800044660B3036853B30279162A29D9427926
:10ECA8001A700146082251F8060B013002F05CF890
:10ECB8002146082251F80E0B093002F055F8236856
:10ECC800E28A5A74E38A22681B0A93742368A26949
:10ECD800DA74A36922681B0A13752368628B5A7554
:10ECE8002368E27E9A7517232371002010BD012046
:10ECF800FCE70220FAE738B50446002863D001682B
:10ED0800002960D0037B90F8282003F00F03002A25
:10ED180057D10833207904321344984255D3637984
:10ED28000B702368A2685A70A36822681B0A937044
:10ED380023686289DA702368E27A1A712368227B71
:10ED48005A712368E2899A71E38922681B0A21466D
:10ED5800D371227B51F8100B02F00F02083001F03A
:10ED6800F9FF237B94F8282003F00F0303F108052B
:10ED78002AB1226894F82010515503F1090520683A
:10ED880094F82820616A284401F0E4FF94F82830B8
:10ED98002268E16A2B44D1545A1CE16A206892B275
:10EDA800090A81549A1C2168E08D92B28854DA1CB1
:10EDB800216894F82F0092B20433885423710020FC
:10EDC80038BD0933A6E70120FAE70220F8E700007A
:10EDD800024B1A8810431880704700BF382400205F
:10EDE80008B5074B1B883BB1FEF7CAF9002814BFCA
:10EDF8006FF00200002008BD6FF00100FBE700BFC4
:10EE08003824002010B5034B00241C80FEF7AEF90F
:10EE1800204610BD38240020B0FA80F04009704721
:10EE280082B018B9084602B000F0CAB8002002B093
:10EE3800704710B9084600F077B9704710B908460E
:10EE480000F08EB970470346084611460BB900F02A
:10EE5800E5B90020704710B9084600F06DBD70474D
:10EE680010B9084600F006BA0020704710B40446EE
:10EE7800084611461A46019B14B910BC00F014BA92
:10EE880010BC70470346084611460BB900F03EBA5D
:10EE98000020704710B40446084611461A4614B9B3
:10EEA80010BC00F0ABBA002010BC704730B4054667
:10EEB800084611461A46DDE902341DB9029430BCF1
:10EEC80000F02ABB002030BC704710B9084600F09B
:10EED800DBBB0020704710B9084600F06BBD00206E
:10EEE800704710B9084600F0EABB0020704710B917
:10EEF800084600F0E7BB0020704703460846114665
:10EF08000BB900F001BC0020704710B40446084655
:10EF180011461A46019B14B910BC00F0F7BB092032
:10EF280010BC704710B40446084611461A4614B976
:10EF380010BC00F061BDC8B210BC704700487047F3
:10EF480001000102064B10B51B6A0446984730B110
:10EF58000448054B204498428CBF0020012010BD76
:10EF68000443010840C220C980B92A00F0B5114BFA
:10EF780085B00C4610491F56054601F04BF80F4B5B
:10EF8800E4B25E6A072D4FF00103CDE90243014662
:10EF98000AD105220023CDE900234FF47A727A437F
:10EFA8001846B04705B0F0BD08220020CDE9002082
:10EFB8003A46F5E7E83C0108C83C01080443010863
:10EFC8001FB5002300930378013B372B21D8DFE8D6
:10EFD80003F01C242020201E202020204143454EE1
:10EFE8002055585B5E6164206C1E6E73787A202011
:10EFF8007D81262020202020202020202020202045
:10F0080083858A2020838A208C90C3780BB10223C1
:10F018000093009805B05DF804FB8378F6E7437821
:10F028008DF8043005238DF805308378003B18BF30
:10F0380001235B008DF8063010238DF80730304B24
:10F048001B6801A803F55872CDE9022300F0C2FF3E
:10F058000090DEE74023DBE72023D9E7827890F9A8
:10F06800013012B9274AD35CD2E7274AFBE78278F6
:10F0780090F90130002AF8D1244AF4E740F6B83371
:10F08800C6E74FF47A73C3E74FF4FA63C0E741F277
:10F098008833BDE741F27073BAE71D484FF47A71BF
:10F0A80001F03CFE00F5FA60D2E71A4BB0E7144BCA
:10F0B8001B6803F55873ABE7114B1B6803F55B73CB
:10F0C800A6E71023A4E70E4B1B68A1E74FF0834384
:10F0D80000939EE7104BFBE7104B99E740F21113A2
:10F0E800ADF8003095E7032392E790F901300C4A18
:10F0F800B9E70C4990F9010000F08CFFA8E700BFC0
:10F1080040240020BD3C0108AD3C0108B53C010885
:10F1180018FCFFFF00EA06379A99094040F70937BB
:10F12800E83C0108C83C010837B50B4B02781B685E
:10F138000C2101FB02335B7A03EB4304074B1D6888
:10F1480003690093C3684278816805EBC40000F046
:10F15800DDFC03B030BD00BF402400203C2400206B
:10F1680070B586B0027B6423ADF80030012A4FF0F9
:10F178000003CDE90133CDE903338DF802308DF872
:10F18800143030D0022A39D05ABB03684BB34368D5
:10F198003BB31F4D80682B601E4B182269461860D0
:10F1A80001F0D8FD1C4B2C6893E807000C3384E869
:10F1B800070093E8070004F10C06032386E807001C
:10F1C800A4F86C33012204F55B7104F5587000F063
:10F1D8008EFC2B684FF6B072A3F878230522C3F88B
:10F1E8007C2306B070BD0A4908684360036100F5D6
:10F1F8005B7100F5587000F07AFCF2E7044B1B686D
:10F20800B3F86023B3F86C130A43A3F86023E8E764
:10F21800402400203C240020A039010808B50346FA
:10F228000A2924D8DFE801F006232323230B161B21
:10F2380023212100BDE808400068FFF783BE90F94C
:10F2480000009978052271B900F011FC003818BF48
:10F25800012008BD052293F900000021F4E790F988
:10F2680000005978EEE70221EEE70722F3E70020D5
:10F27800EFE7000008B502791AB1012A0BD0002087
:10F2880008BD084B01681B68012203F5587000F09F
:10F298002EFC0120F4E7034B01681B6803F55B7043
:10F2A800F5E700BF40240020F7B50528144D1C469B
:10F2B800A8BF052058700E462946174600F0AAFE3A
:10F2C80094F90130A070072B13D1322000F0A2FD71
:10F2D8000C4BDB6D0546984704F10C0208340346D5
:10F2E800019200943A463146284600F098FD03B052
:10F2F800F0BD054A55F82310D05C00F083FDE7E720
:10F30800C83C010804430108E83C01082DE9F04F16
:10F31800344F90F901607B68D0F804908BB00446B4
:10F32800884698470546002859D1E37C73B92E4A88
:10F338002378126803EB4303990002EB8303D3F8A5
:10F348000490B9F1000F01D152F80190274B4846BB
:10F3580013F906B0FB689847A37C2289D7F818A050
:10F368000993072E28D100230121CDE90223204A41
:10F378000693CDE90431CDE907330521CDE9002114
:10F388004FF47A7202FB0BF24CF250311846D04718
:10F39800637C13B3174B995D7B6D0D31C9B2284659
:10F3A8009847E07C3246494600F046FE88F80060FF
:10F3B80001200BB0BDE8F08F002101250823CDE91D
:10F3C8000013CDE90715CDE90511CDE90311029226
:10F3D800A1782B465A462846D9E7074BDBE7002099
:10F3E800E7E700BF0443010840240020E83C010887
:10F3F80085450100B53C0108BD3C01082DE9F04FE9
:10F408008DB090F90130DFF8FCA0DFF8FC90CDE971
:10F418000A123E4A12F903B00278DAF800300C25D5
:10F4280005FB02333A4A5B7A126803EB430302EBAB
:10F43800C303044693F9021090F9020000F0E5FDB9
:10F448003449064694F9010000F0E4FDA2686168B9
:10F458008046304600F00BFD2178DAF80020D9F814
:10F468000C306943074650589847D9F81C309C46D9
:10F4780094F901300025072B4FF47A63CDE907533F
:10F48800CDE905552DD10123CDE903530523CDE958
:10F4980001534FF47A7303FB0BF300933946434649
:10F4A80046F2A81228466746B8472378DAF80020BB
:10F4B8000C214B4394F90110D05800F0DFFDA189CD
:10F4C80094F90100FFF752FD0B9B217B1860D9F8D6
:10F4D8005430284698470A9B01201E700DB0BDE89D
:10F4E800F08F01200823CDE90350CDE901032A4616
:10F4F800CDF800B0654643463946A8470120054681
:10F50800D3E700BF4024002004430108E83C010879
:10F518003C240020C83C01082DE9F04F8FB000249E
:10F5280005468A46914698460494ADF81440ADF8CD
:10F53800024007264FF0010B2B7AA34206D96868D0
:10F5480004A9204400F0F6FB00285ED102238DF8C0
:10F55800083002A86B7A8DF80A30FFF731FDAB7AD4
:10F568008DF81D309DF811308DF81E309DF8123041
:10F578008DF81F309DF810308DF82030EB7A8DF81B
:10F5880021302B7B8DF822306B7B8DF823301023B4
:10F598008DF81C608DF824303A4E8DF82C000DF152
:10F5A80002030A9305238DF82D3033680C93072343
:10F5B800ADF834302B6806930DF1120204AB0DF14F
:10F5C800110106A800F0D0FB072805460BD13068CA
:10F5D8000C22002100F5587001F0D0FB3368BDF80B
:10F5E8000220A3F860239DF811308AF800309DF8B6
:10F5F800123089F800309DF8103088F80030189BD8
:10F6080028461C700FB0BDE8F08F9DF81330BDF888
:10F618001470ADF802702044C4B2F3B917B3194A94
:10F6280000201168072602464FF00C0C062B1BD150
:10F638000CFB00FE51F80EE0BEF1000F04D00BFAEF
:10F6480000F23A4397B2012201301028EED1002A85
:10F658003FF472AFADF802706EE75A1E042A01D962
:10F66800062BDCD0062667E747FA00FE1EF0010FDE
:10F67800EAD00CFB00FE51F80EE0BEF1000F08BF07
:10F688000626E1E74024002038B505464068FFF724
:10F6980059FC0522841D002195F90000E4B200F010
:10F6A800E6F908B904F0FD0495F9010007220021E4
:10F6B80000F0DDF908B904F0FB04204638BD00204D
:10F6C8007047000010B503780F2B044618D840681F
:10F6D800FFF738FC22780B4902EB42020968831CC9
:10F6E80001EB820051F82220DBB21AB903F0FD03C6
:10F6F80058B210BD032B06BF626842600223F7E7C9
:10F708000020F6E740240020022070472DE9F04F42
:10F71800DFF838810446D8F8000099B089461746C2
:10F7280000211E460122032300F55870CDE9061179
:10F73800CDE908118DF814108DF81510ADF81630B4
:10F7480000F0B7F938B9D8F80020B2F8603343F0C0
:10F758000303A2F86033D8F80020637A8DF82830C4
:10F7680002F55871CDE90B12394A94F9083012683C
:10F778000D920DF116020F92226810926268119292
:10F78800D4E90301A27A8DF8482001228DF8492096
:10F7980013AA82E803001025227DE18A8DF829301A
:10F7A80018468DF85420ADF83850FFF7DFFB0AAB48
:10F7B80017930DF11503169000933146019705AB89
:10F7C80006AA10A800F0C2FB064698BB9DF81410C4
:10F7D800204F013901F0A2FA1F4B1B690393C4B2F1
:10F7E8004FF00C0B04F160036B44D8F8000013F8D9
:10F7F80048AC9DF814300BFB0AFC01343946B4FBC5
:10F80800F3F203FB1244D0F87C33B0F9782350F8B4
:10F818000C00DDF80CC0E4B2E04728B189F800A07C
:10F82800304619B0BDE8F08F013D15F0FF05D9D17C
:10F838000D26F5E70C2801BFD8F80020B2F8603390
:10F8480043F00303A2F86033EAE700BF4024002036
:10F858003C240020400D030004430108F8B5067954
:10F86800012E054648D90F2E48D80368187A40F368
:10F8780003000522002140B200F0F9F82B68044685
:10F88800187A40F303100522002140B200F0EFF887
:10F89800B8B1B4FA84F4640929680B7A086843F3A8
:10F8A800030243F303135BB252B29A42C8BF012466
:10F8B800FFF748FB80F00103DBB224B10533D8B26F
:10F8C800F8BD0124E8E7DBB90E4F29683B6806EB71
:10F8D800460003EB80000C2201F03CFA3A680C2346
:10F8E80003FB062320465C72B2F860130123B34081
:10F8F8000B43A2F86033E3E70620E1E70320DFE7E4
:10F908000420DDE74024002010B4017801290ED935
:10F91800084B18680C234B43C4180022C250C4E992
:10F92800012200F5587010BC102200F0A9B8002080
:10F9380010BC7047402400202DE9F04186B05023C8
:10F948008DF81430037A102B074630D14368DD7BDD
:10F958006DBB0224A8466426062C14D87A68535D29
:10F9680003932A44517843EA01230393927843EAA4
:10F9780002437343CDE9033863B968468DF8004004
:10F98800FFF7C2FF0DE0CDF80C808DF81480CDF89C
:10F998001080F2E703AB01A801938DF80840FFF748
:10F9A8005DFF0134E4B2102C05F10305D4D106B093
:10F9B800BDE8F0811FB502680379116849B901A84B
:10F9C8008DF80430FFF7A0FF78B1032005B05DF88B
:10F9D80004FB02A802928DF80C30FFF73FFF0428C1
:10F9E80005D0052805D00028EFD00020EEE702203A
:10F9F800ECE70120EAE70000C90020B9034B0B44FB
:10FA08009856C0B27047024BF9E700BF6D3C010839
:10FA18002D3C0108F0B59A42069D03DB9DF9143090
:10FA28009A4220DD0020F0BD03EB430331F814C0F7
:10FA380005EB830300264CFA06F7FF0707D51F7A64
:10FA480007F00F0E964502DCB2EB171F0DDD0136ED
:10FA5800102E03F10C03EED10134E4B22301DBB222
:10FA68009842E1D8DEE70024F8E70120DBE7884286
:10FA780004DB9042CCBF0020012070470020704773
:10FA880010B51409B4EB111F03464FEA11100ED339
:10FA980091420CD202B201F00F0133F8124001205A
:10FAA80000FA01F124EA010123F8121010BD002028
:10FAB800FCE7F0B528B100EB410501270020914291
:10FAC80000D3F0BD002435F802CB234607FA04F62C
:10FAD80036EA0C0608BF013304F1010408BFDBB2A3
:10FAE800102CF3D118440131C0B2C9B2E7E710B500
:10FAF80000B149B910BD31F8134020F81340013363
:10FB0800DCB2A242F7D8F5E70023F9E782B030B5B6
:10FB180004880493D2B9B3F5616F15D349F6AF25BC
:10FB280042F21072AB4298BF4FF47A72944238BFD7
:10FB380014466143BDE83040C3688B428CBF5B1AF2
:10FB48000023C36002B070476422EFE7012C38BF7E
:10FB58000124EEE72DE9F04F8FB01546199F039366
:10FB68009DF8603007930C46804603F0C7FB6A4A4D
:10FB78000590A7F5F633303BB3FBF2F3534303F597
:10FB8800F63B0493182313FB05430BF1300B069344
:10FB980000254FF0FF3A069B9C4207D1002D14BF69
:10FBA80050464FF0FF300FB0BDE8F08FBDF9683018
:10FBB800ADF82430099919973846089703F02EFBB9
:10FBC8002688B8F1000F5FD1B7F5616F5AD349F6AF
:10FBD800AF2242F21073974298BF4FF47A739E4255
:10FBE80038BF1E46642E59D1DFF83091A060A16855
:10FBF8000CA803F035FB0D9B0093DDE908120C9B64
:10FC08000AA803F08CFA039A0A9B0AB9079A2AB140
:10FC180022694A4502D1424A93420ED9414BC4F85F
:10FC28000C909F4209D90023ADF82C300B99CDF8E0
:10FC380028B0584603F0F2FAA060606808B9C4F822
:10FC48000C90C4F81090B8F1000F04D003F060FBDA
:10FC5800E3680344E360D4E903329342059B88BF19
:10FC6800E26063601B9BE1687343994204D2039886
:10FC7800E8B9B8F1000F1AD001231D442375EDB27D
:10FC8800183488E76423AAE7039B0BB9234BE36086
:10FC9800012EDFF8889038BF0126CEE7B6F57A7FC7
:10FCA8000ABFDFF88490DFF88490A0609FE7002007
:10FCB8009342207506D85B1A9A4505F1010528BFBD
:10FCC8009A46EDB2B8F1000FDAD1642E184AADF8B1
:10FCD8002C801DD049F6B023B6F57A7F18BF13469D
:10FCE800974281BF049A02F5A83202F5C0729B18A8
:10FCF8000A931A9B00930AAE96E80600199B3046B1
:10FD080003F00DFA96E8030003F088FA8246B7E795
:10FD18004FF46163E4E700BF8051010040771B00A6
:10FD28007F5101002FEC010080A81201002E9302E0
:10FD380030EC01000378032B14D1437803F00F0251
:10FD48001B098A704B7083788B80C27843EA022340
:10FD58008B800379C3F3021203F00F03CA700B7090
:10FD680005207047002070472DE9F3479A464379EC
:10FD7800057990F907609146044690F9062088466F
:10FD8800D3B190F90870002D37D00F2A1BD194F900
:10FD980009200F2E27D194F90A00072D02D1002F30
:10FDA80008BF012788F8002089F8000028468AF84B
:10FDB800007002B0BDE8F08790F90B7090F9092047
:10FDC80090F90A60DFE7A369019394F9153000936D
:10FDD80094F914302169207BFFF71CFE0028D8D144
:10FDE80005F0FD05D5E794F91D00B042D5DC94F97E
:10FDF8001C30B34203DA05F0FB053046D2E7304643
:10FE0800CBE70000024B03FA00F0B0FBF1F07047BB
:10FE180040420F004FF4FA53B3FBF0F0704730B58F
:10FE28004FF47A750C1F6A4300FB042252001EBF70
:10FE380000F1FF341219B2FBF0F2914238BF1146BB
:10FE4800039A1160820048431CBF013040084FF4F8
:10FE58007A71121A01FB1323002BCABF03F2E7338E
:10FE680093FBF1F1B3FBF1F1049B196030BD38B598
:10FE7800400014460D46F1F7C9FD01462846F1F742
:10FE880013FD2146F1F710FDF1F702FC03F0DCFC4D
:10FE9800F1F7DEFC40B238BD2DE9F74F019300239E
:10FEA8009C469E46048A1E01F6B2B44246D906EB29
:10FEB80046054FEA4309AD000024476837F8097042
:10FEC8002741FF0729D5876807EB050A7F5927B31C
:10FED800077837B9476927B137F809702741FF070D
:10FEE8001BD59AF8087090F901B047F303084FFA48
:10FEF80088F8D84511DC47F303177FB25F450CDB60
:10FF08009AF8097007EB4708C76807EBC8073F7DF1
:10FF18005FB90CF1010C5FFA8CFC0134102C05F16F
:10FF28000C05CAD10133DBB2BCE70EF1010706EBC1
:10FF3800040801F80E805FFA87FEEEE7019B82F85D
:10FF480000E083F800C003B0BDE8F08F2DE9FF475B
:10FF580004464068DDE90C671D468A46914603F071
:10FF6800D7F923681B1A3B604FF000080123337050
:10FF780085F80080636813B12368834224D8D4F8D5
:10FF88001CC0CAF80080A3699CF800E00393D4E978
:10FF9800030101AB83E80300237D0093DCF80C1018
:10FFA800237A627A7046FFF7D5FD334638602A46D1
:10FFB800E0694946FFF770FF2B782BB1C7F800803E
:10FFC800002004B0BDE8F0873378002B0CBF0C206C
:10FFD8000B20F6E737B590F9002090F902509542CA
:10FFE80004460FD0013A52B295420BD0A368019350
:08FFF80094F9013000936168E7
:020000040801F1
:10000000E0782B46FFF70AFD0028EFD0104603B03A
:1000100030BD8842B8BF08467047000051F8200044
:10002000054B984205D0054BC31A58425841400031
:1000300070470120704700BF90D0030020A1070047
:1000400005281FB50ED80C4B53F820300093CDE98E
:1000500001120A4B01220021022002F06BFE05B0C2
:100060005DF804FBCDE90012054B012200210220BE
:1000700002F060FEF3E700BF5C3D0108F03C0108C0
:100080000F3D010807B5054BCDE900010122002114
:10009000022002F04FFE03B05DF804FB2B3D010887
:1000A00010B5102204460021F13000F06BFE002153
:1000B000C4F814112046F022BDE8104000F062BEE2
:1000C00002460846102100F0A5B92DE9F043044688
:1000D000D0F8140185B00E46154604F2011988B314
:1000E000C0F110089045474628BF1746BAB24844A9
:1000F00000F034FED4F814313B440F2BC4F8143113
:100100002DD9A8452BD204F1F00304F5807113F822
:10011000012F187C8B4282EA00021A70F7D104F199
:10012000F10810224146684600F018FE2246694652
:10013000684600F0F1F910226946404600F00EFED4
:100140003E44ED1B04F5807804F1F107102D09D829
:10015000AAB23146484600F001FEC4F8145105B079
:10016000BDE8F08304F1F003711E13F8012F11F8BC
:10017000010F434582EA00021A70F6D11022394677
:10018000684600F0EBFD22466946684600F0C4F977
:1001900010226946384600F0E1FD1036103DD5E7E3
:1001A000F0B589B00C46102200210546684600F0E3
:1001B000E9FD22466946684600F0AEF99DF9003037
:1001C000002B6A464FF0000143DA137812F8010F52
:1001D00001315B0043EAD0130F2902F8013CF4D14E
:1001E0009DF80F305B0083F08703D4F81401DBB275
:1001F00010288DF80F303BD104F58073694604F563
:10020000887013F8016F11F8012B984282EA0602F8
:100210001A70F6D104F1F00304F5807113F8012F80
:10022000187C8B4282EA00021A70F7D110220DEB83
:10023000020004F1F10100F091FD2246294604A8D4
:1002400000F06AF910220021684600F09BFD09B019
:10025000F0BD137812F8010F01315B0043EAD013AF
:100260000F2902F8013CF4D19DF80F305B00BCE788
:100270009DF90030002B6A464FF0000137DA137801
:1002800012F8016F01315B0043EAD6130F2902F81F
:10029000013CF4D19DF80F305B0083F08703471CCD
:1002A000DBB28DF80F30102F04EB0003C0F10F0606
:1002B0004FF0800288BF002600F5817083F801218D
:1002C0000021324620443E4403F076FAC4F814611B
:1002D00004F58073694604F5887013F8016F11F80E
:1002E000012B984282EA06021A70F6D192E713783F
:1002F00012F8016F01315B0043EAD6130F2902F8AF
:10030000013CF4D19DF80F305B00C8E70A78037810
:10031000534003704A784378534043708A78837817
:1003200053408370CA78C3785340C3700A79037905
:10033000534003714A794379534043718A798379F1
:1003400053408371CA79C3795340C3710A7A037ADF
:10035000534003724A7A437A534043728A7A837ACB
:1003600053408372CA7AC37A5340C3720A7B037BB9
:10037000534003734A7B437B534043738A7B837BA5
:1003800053408373CA7BC37B5340C373704710B51C
:100390000B7814786340037054784B786340437053
:1003A00094788B7863408370D478CB786340C37043
:1003B00014790B796340037154794B79634043712D
:1003C00094798B7963408371D479CB796340C3711D
:1003D000147A0B7A63400372547A4B7A6340437207
:1003E0008B7A947A63408372D47ACB7A6340C372F7
:1003F000147B0B7B63400373547B4B7B63404373E1
:10040000947B8B7B63408373CB7BD27B5340C373E2
:1004100010BD0000A1F11003DBB2102B2DE9F04755
:10042000044604D83A4820FA03F3DB0705D4002336
:1004300082F8F030FF20BDE8F087561E254615F8FB
:10044000013B06F8013F631B0B4413F0FF00F6D19C
:1004500001F11C039B005FFA83FCC3F30313013B10
:10046000DFF8B09082F8F030884653184FF0010E54
:10047000B8FBF1FA01FB1A8A1AF0FF0A13F8047CA0
:1004800013F8036C13F8025C13F8014C30D119F81F
:1004900006A019F8056019F8045019F807404FEA4A
:1004A000DE1707EB47078EEA0A0A07EBC7074FEA92
:1004B0004E0EFFB25FFA8EFE87EA0E0E574692F896
:1004C00000A087EA0A071F7057787E405E70967812
:1004D00075409D70D57808F104085FFA88F86C4083
:1004E000C445DC7002F1040203F10403C0D8A2E7A2
:1004F0001829E4D9BAF1100FE1D1DFF818A01AF8E1
:1005000007701AF806601AF805501AF80440D6E782
:1005100001010100743F01082DE9F04FA3B092F8EA
:10052000F0301D911B920193002B00F05381014686
:100530001EA8FFF72CFF1B9BA74CA84DA84E1033FD
:100540000293002303939DF87C0004909DF886009D
:100550000590205C06909DF87B000790205C089039
:1005600004989DF881C0205C099014F80C000A9052
:100570009DF880000B909DF885009DF878809DF88F
:100580007DE09DF882A09DF887900C909DF87A0000
:10059000029B1C9314F80A2014F8093014F8081070
:1005A00014F80E700D90205C0E909DF87F000F9057
:1005B000205C10900B98205C11900C98205C12909D
:1005C0009DF8840013909DF8790014909DF87E00AA
:1005D0001590205C16909DF883001790205C189071
:1005E0001398205C19901498205C1A90039801309D
:1005F00003900298DDF804B0103002909DF80C00D2
:10060000834536D88DF878108DF87A2009990E9A9E
:100610008DF87C108DF882201199069A8DF8801043
:100620008DF87E201999169A8DF884108DF8862001
:100630000A99189A8DF87D108DF887201299109AD2
:100640008DF87B301B9B8DF881108DF883201A99D3
:10065000089A1D988DF885108DF87F201EA903EB50
:100660000B128DF87970FFF792FE002023B0BDE8E1
:10067000F08F15F808B082EA03008BEA000016F844
:100680000EB080EA0B008DF8780015F80E004B4094
:10069000434016F80A0043408DF8793081EA070399
:1006A00015F80A10594016F80930594016F8083064
:1006B0008DF87A107A40534015F8092053408DF890
:1006C0007B30089A069B5340049AAA5C534016F864
:1006D0000C2053408DF87C30DDE908325A4015F883
:1006E0000C305340059AB25C53408DF87D30DDE903
:1006F00009325A40059BEB5C5340079AB25C534069
:100700008DF87E30069B0A9A5340049AB25C5A4098
:10071000079BEB5C5A408DF87F200E9B109A53404C
:100720000B9AAA5C53400C9AB25C53408DF880300F
:10073000DDE910325A400C9BEB5C53400D9AB25CE1
:1007400053408DF88130DDE911325A400D9BEB5C4E
:1007500053400F9AB25C53408DF88230129A0E9B30
:1007600053400B9AB25C5A400F9BEB5C1C995A4069
:100770008DF88320169B189A5340139AAA5C534015
:10078000149AB25C53408DF88430DDE918325A4037
:10079000149BEB5C5340159AB25C53408DF8853046
:1007A000DDE919325A40159BEB5C5340179AB25C55
:1007B00053408DF886301A9A169B5340139AB25CB8
:1007C0005340179AAA5C1EA853408DF88730FFF754
:1007D0009DFDB8E6FF2049E7743F0108743E01081B
:1007E000743D010808B538B1044A05491060D822A3
:1007F00000F0B4FA002008BD0220FCE744240020E9
:10080000A44401080A4B1A6870B5002302F11805C8
:1008100003EB03142E5D864204D1183422440A608F
:10082000002070BD01330B2BF2D10320F9E700BF8C
:10083000442400202DE9F041CCB00646DDF8488183
:1008400017461C460D4631B3B8F1000F23D006A859
:10085000FFF726FC204601A9FFF7D4FF0446B0B9F4
:10086000019906A80131FFF72BFC26B11022314671
:1008700006A8FFF72AFC3A46294606A8FFF725FCFA
:1008800006A902A8FFF78CFC029BC8F8003020469E
:100890004CB0BDE8F0810224F9E7000030B595B016
:1008A00013A90446FFF7AEFF002830D11B4B0C21E3
:1008B00001FB00F2D5189A5CA2422AD1139B1A7C44
:1008C0001092DA7B0F929A7B0E925A7B0D921A7BD2
:1008D0000C92DA7A0B929A7A0A925A7A09921A7AD6
:1008E0000892DA7907929A7906925A7905921A79DA
:1008F0000492DA7803929A7802925B78019300224C
:10090000AB6800931146064B022002F013FA15B0B3
:1009100030BD01300B28CBD1F9E700BFEC41010815
:100920007440010810B40B2B019C03D8019410BC37
:10093000FFF780BF032010BC704730B50D4685B06F
:100940001446014668B103AA002000922A4603908B
:10095000FFF770FF18B90398001B18BF012005B0FE
:1009600030BD0220FBE72DE9F0430D46BFB0144631
:100970009946804620B31BB311F00F0122D1F0221B
:1009800001A800F0FFF920466946FFF73BFF044647
:1009900048B9009801AA10210130FFF73BFD2E460F
:1009A000AF1BFFB21EB920463FB0BDE8F08301AADD
:1009B00009EB070108EB0700FFF7AEFD103EEFE77C
:1009C0000224F0E70524EEE7F0B5184E346802463D
:1009D00085B00846002304F1180103EB03154F5DB1
:1009E00097421ED10D2A05F1190513D10023CDE937
:1009F0000033CDE902330C2210216B46FFF7B3FF21
:100A00000446306810226946284400F0A7F92046C1
:100A100005B0F0BD01461022601900F09FF90024D6
:100A2000F5E701330B2BD8D10324F0E74424002051
:100A300009B1FFF7C9BF022070471FB51446A0B126
:100A40000C2A01D10B2912D10023CDE90033CDE9C5
:100A500002330A466B461021FFF785FF18B9694635
:100A60002046FFF7B1FF04B010BD0220FBE70320D2
:100A7000F9E7F8B51E46DDE907479DF818505BB366
:100A800054B34FB3212D29D819462A46204600F0E9
:100A900065F90122631C691EB018FFF764FFF8B9FD
:100AA000E37ADB093B70EBB96319204613F8012C9C
:100AB00013F8021C120642EA014213F8041C0A430E
:100AC00013F8031C012342EA0122291FFFF735FF17
:100AD000003818BF0120F8BD0220FCE70520FAE726
:100AE0000720F8E70420F6E710B5044628B1044BC8
:100AF0005B6998472060002010BD0220FCE700BF22
:100B00000443010808B5014630B1044B08221868B7
:100B100000F024F9002008BD0220FCE74424002056
:100B200008B530B1044B0822196800F017F900200D
:100B300008BD0220FCE700BF442400207FB5124E10
:100B40000023044602A801930D46FFF7E9FF33682E
:100B50005B6901936CB102AA082312F8011B41B929
:100B6000013B13F0FF03F8D102A8A04702A8FFF74A
:100B7000C9FF35B1019B23B901A8A8473368019A81
:100B80005A61002004B070BD4424002008B501461D
:100B900038B1054B18680822104400F0DFF8002037
:100BA00008BD0220FCE700BF4424002008B538B18E
:100BB000044B19680822114400F0D0F8002008BD49
:100BC0000220FCE744240020034B1B6802280CBFD2
:100BD00019615961002070474424002049B1064B37
:100BE0001B68D3E90423022808BF13460B600020CA
:100BF00070470220704700BF4424002030B58FB0FA
:100C0000002405460CA80994FFF78AFF9DF83730A9
:100C100007939DF8363006939DF8353005939DF87F
:100C2000343004939DF8333003939DF832300293AF
:100C30009DF8313001939DF83030009322462146D3
:100C40001E4B022002F076F80AA8FFF7AFFF9DF8CE
:100C50002F3007939DF82E3006939DF82D30059385
:100C60009DF82C3004939DF82B3003939DF82A3087
:100C700002939DF8293001939DF828300093224675
:100C80000F4B2146022002F055F809A92846FFF72C
:100C9000A5FF9DF8243003939DF8253002939DF81D
:100CA000263001939DF8273000932246054B2146BC
:100CB000022002F03FF80FB030BD00BFD040010865
:100CC0000E4101084C41010808B50020FFF7E6FD80
:100CD0000120FFF7E3FD0920FFF7E0FD0820FFF703
:100CE000DDFD0020FFF78AFF002008BD10B5044697
:100CF0000B20FFF7D3FD0C20FFF7D0FD0920FFF7F5
:100D0000CDFD0820FFF7CAFD0A20FFF7C7FD2046EA
:100D1000FFF774FF002010BD014B1860704700BF43
:100D2000AC0800200B4A30B514680B4D43F2390370
:100D300005FB04331360091A6FF00042B3FBF2F2B3
:100D4000C2EBC27201319B1A93FBF1F201FB123329
:100D5000184430BDAC0800206D4EC64101380A442D
:100D6000914200D1704711F8013B00F8013FF7E7CD
:100D700010440A44914200D1704711F8013B00F839
:100D8000013DF7E702F018BD30B530B10A4D01441E
:100D90004FF0FF33814201D1D84330BD10F8012B11
:100DA0005340082243F30004013A2C4092B284EAF3
:100DB0005303002AF6D1EDE72083B8ED01207047F8
:100DC000054B4FF400529A62044B1B6813B15B68E9
:100DD00003B11847704700BF00040048D424002026
:100DE000054B4FF480529A62044B1B6813B1DB68C9
:100DF00003B11847704700BF00040048D424002006
:100E0000012070470120704701F03EB901F02CB974
:100E100010B501F00FFE0E21044640F61F1001F040
:100E200023F92046012101F0EFFDBDE8104001F05B
:100E3000CDBA000070B50C4E01EB40030D46B36512
:100E40004FF6FF71002304461A46084601F054FB92
:100E500096F85600002101F0D7FD29462046BDE84E
:100E6000704001F08BBA00BF7824002010B5044612
:100E700001F0A0FE01281CD101F0A4FE34B11248FB
:100E8000214602F00BFB104802F0CEFA0F4C104B3B
:100E900000214FF48052A1659A6194F8560001F048
:100EA000B3FD63786BB16FF07F40BDE8104001F097
:100EB00049BA002340F262211A46084601F01CFBA1
:100EC000DCE7A0688001F0E74824002078240020B7
:100ED00000040048002001F0B5B9000008B501F099
:100EE000BDF80438C0B2032896BF024B0020185C3E
:100EF00008BD00BFCE42010808B501F0B0FD0330C7
:100F000008BD01F03FB901F0FFB808B501F0F6FCEB
:100F100008BD000038B50D46144601F053FB2846C5
:100F200001F088FD0E21054640F61F1001F09CF8E7
:100F300028460121074D01F067FD01F047FA4FF403
:100F40007A716143284602F0A9FA2846BDE8384084
:100F500002F06ABA6024002001F034BB08B5084BE7
:100F6000002193F8560001F04FFD00234FF4C071AB
:100F70001A46084601F0C0FABDE8084001F01ABA66
:100F80007824002010B5044601F014FE01281CD17D
:100F900001F018FE34B11248214602F07FFA1048E1
:100FA00002F042FA0F4C104B00214FF48052A16521
:100FB0009A6194F8560001F027FD63786BB16FF0E9
:100FC0007F40BDE8104001F073B9002340F2622178
:100FD0001A46084601F090FADCE7A0688001F0E7C5
:100FE00048240020782400200004004808B54FF071
:100FF000040001F00DF9BDE808400220F1F748BDFA
:1010000008B500231A461946184601F075FABDE8DE
:10101000084001F063B900001D4B73B51D4D186009
:1010200000241D486C70C5E90144AC6501F08EFADE
:10103000AC8101F0F9F92146204601F041FC21463E
:101040000422012001F0F2FA144E154D4FF6FF7103
:1010500023462246084601F04FFAFFF7C7FF224613
:10106000104B00944FF0FF31304602F031F90E4B37
:10107000009422464FF0FF31284602F029F930460D
:1010800002F084F9284602B0BDE8704002F07EB953
:10109000D4240020782400204D2001086024002062
:1010A00048240020C10D0108E10D0108012808486D
:1010B00005D1084BC17719700E3001F09DBB437DFF
:1010C000012B03D1034B81751970F5E7704700BF01
:1010D00078240020B00800200D4B10B5044618738A
:1010E0005873012000F016F85CB134214FF4E86029
:1010F00000F0BAFF4421BDE8104040F2417000F01A
:10110000B3BF14214FF4E86000F0AEFF2421F2E7F2
:101110007824002038B5114C0546207001F057FDA9
:10112000052D04D8DFE805F0090B03171709032084
:1011300001F066FA0023637338BD0020F8E7012050
:1011400001F05EFA207B637B8342F5D06073BDE8DB
:101150003840FFF7C1BF0220EAE700BF7824002033
:101160002DE9F0431E4687B000230546CDE9013343
:101170000C46174601F01DFD032D5BD8DFE815F086
:101180007A00C1000C010400A27C082A69D8A16879
:1011900001A801F0D5FE2168002962D042F2107248
:1011A0009142E37C874D50D80322AA7385F83820FA
:1011B000E96385F844304FF002086368A17DDB00E5
:1011C0002B820423AB74A37CDB00EB7402294FF069
:1011D00000032B75637D02D0227D022A46D103F1E4
:1011E0000F02D2B2012A01D9012B3AD1764B774AAC
:1011F000196803944FF0010903A88DF8149001F0C9
:10120000D5FC70BB287685F817906875FFF762FEED
:101210004046FFF77FFF6E4801F082FA6D4801F00B
:10122000EBFA01A800F080FF208A00F051FFA089AE
:1012300000F096FF384601F0FDFB624C84F8560042
:1012400001F0BCFC666000200DE04FF00008E9638F
:10125000890885F80E8085F8388085F8443029643F
:10126000ABE74FF0FF3007B0BDE8F083EB752976B0
:101270006A75CBE72368002BF3D0A27C082AF0D84C
:10128000504DA16801A801F05BFE002385F83830BD
:101290002268EA63E27C85F84420A269AB732A6481
:1012A0006268D2002A820422AA74A27C2B75D20022
:1012B000EA74A27D022A02D0237D022B1CD1627D1A
:1012C00002F10F03DBB2012B01D9012AC9D13E4B38
:1012D0003E4A196803944FF0010803A88DF8148062
:1012E00001F064FC0028BCD1287685F81780687569
:1012F000FFF7F0FD00208CE7617DE9752A766B75BC
:10130000F6E7304D012185F83810227885F8502015
:10131000637885F85130A37885F85230E3788B42B2
:1013200002D0022B03D03BB985F8533004E00B3ACE
:10133000012A29D885F853104FF0010885F80E804E
:10134000A388AB83A379AB77E37985F82030237A40
:1013500085F82130FFF7BEFD4046FFF7DBFE1C4855
:1013600001F0DEF91B4801F047FA95F85130062BE1
:1013700040F689000AD100F087FE00F0FB0140F63C
:10138000890000F071FE55E70023CDE700F07CFEF8
:1013900040F00401C9B2F2E72368013BB3F57A7F5C
:1013A000BFF45FAF0320FFF7B5FE0648022380F8C5
:1013B000383023688364162380F84C30383001F0CD
:1013C000AFF937E778240020D424002060240020DF
:1013D000B024002086240020F0B51E4687B00023EC
:1013E000CDE90133144607460D4601F0E2FB002C1F
:1013F000724C16BF012300230026637027B1012F12
:101400007AD0002007B0F0BDAB68002B00F0D2808E
:10141000EB68002B00F0CE80AA7F082A00F2CA8079
:10142000296901A801F08CFD2868003818BF012047
:1014300000F0D6FF84F83870AB68E36395F820308D
:1014400084F84430686801F057FBA77384F84500BE
:10145000EB68DB002382EB7FA374AB7FDB00E374DC
:1014600095F82130237595F82230002B3ED12A7D46
:1014700095F82410A275022995F8232001D0022B9B
:1014800036D102F10F03DBB2012B02D9012A40F061
:10149000918000238DF81430494B4A4A196804950D
:1014A00003A801F083FB002840F08480012320760C
:1014B000E3756075FFF70EFD0020FFF72BFE424835
:1014C00001F02EF9414801F097F901A800F02CFE37
:1014D000A88B00F0FDFD288B00F042FE4FF4FA537C
:1014E000AA687343B3FBF2F3A3608AE7FF22BFE766
:1014F000E27521766375DDE72B8E002B5AD095F8C7
:101500003230A86A012B0CBF2F7DFF27003818BF8F
:10151000012000F065FFF0B200F06EFF012184F8B9
:10152000381095F82C2084F8502095F82D3084F848
:10153000513095F82E3084F8523095F82F308B4288
:1015400002D0022B03D03BB984F8533004E00B3AAD
:10155000012A27D884F853102B8EA38395F83230B4
:10156000A3770126AB8E2384A673E777FFF7B2FC3F
:101570003046FFF7CFFD144801F0D2F8134801F0D0
:101580003BF994F82130B34240F236700CD100F0B0
:101590007BFD00F0FB0140F2367000F065FD4FF678
:1015A000FF73A1E70023CFE700F06EFD40F00401D8
:1015B000C9B2F0E74FF0FF3024E700BF78240020E5
:1015C000D424002048240020B024002086240020B9
:1015D0002DE9F04F85B082460E9DBDF840809DF804
:1015E00044709DF84890019193461E4601F0E1FA3F
:1015F000BAF1010F524C54D0BAF1040F00F09180AF
:10160000BAF1000F3AD10B22304684F8442084F816
:1016100038A0E56301F070FA4FEAC803B9F1000F92
:10162000238241F6040363820CBF0123F223E37596
:1016300087F001070123237684F84500C4F840B001
:1016400084F80EA084F814A06775FFF743FC504699
:10165000FFF760FD04F1380001F062F804F10E00BC
:1016600001F0CAF8374A1068516802AB03C302A8F8
:1016700000F05AFD40F2FF1000F02AFD019801F041
:10168000D9F90E2184F8560040F61F1000F0ECFC4A
:1016900094F8560001F092FA169B636005B0BDE81D
:1016A000F08F294984F838A0EAB2895D84F8502087
:1016B00076BB0B3D012D8CBF00250125053A012A83
:1016C00004D8B8F10C0F38BF4FF00C081F4B9DF831
:1016D0003C201B7884F85350E37701259DF8543063
:1016E00084F8511084F8522084F82130A573A4F8AE
:1016F0001C80A77784F82090FFF7ECFB2846FFF7C3
:1017000009FD134801F00CF8124801F075F8B5E72F
:10171000012E04D1A5F10C035D425D41CEE7002509
:10172000CCE75046FFF7F6FC022384F8383004F18A
:1017300038001623A56484F84C3000F0F1FF9DE7D3
:1017400078240020B839010800430108B0080020BF
:10175000B0240020862400202DE9F04F87B0DFF868
:10176000B4B29DF864A09DF84C90029314469DF885
:1017700054309DF85020BDF84880039205468BF800
:1017800001A0BDF8446001930F4601F012FABAF1CE
:10179000000F18BF4FF00008DFF87CA2039AB9F1E0
:1017A000000F08BFFF22012D8AF8002000F0C8803A
:1017B000052D48D0002D40F0C080284600F010FED6
:1017C0000B2238468BF844208BF83850CBF83C403D
:1017D00001F092F9019B8BF8450041F60402002BC1
:1017E000ABF812209AF800208BF816200CBF0122CB
:1017F000F2228BF81720F600012289F001098BF8FC
:1018000018208BF80E50ABF810608BF814508BF842
:101810001590FFF75FFB2846FFF77CFC0BF13800C3
:1018200000F07EFF0BF10E0000F0E6FF7B49086838
:10183000496804AA03C204A800F076FC40F2FF1035
:1018400000F046FC71E0012000F0CAFD09224FF0D3
:1018500000098BF8442038464FF44872CBF84020FA
:101860008BF83890CBF83C4001F046F94FF48052A9
:10187000ABF812209AF800208BF845008BF8162060
:1018800028460122F6008BF817208BF80E90ABF853
:101890001060ABF814908BF81890FFF73BFC0BF13D
:1018A000380000F03DFF0BF10E0000F0A5FF5B4992
:1018B0008868C96804AA03C204A800F035FC40F295
:1018C000FF1000F005FC40F6B80000F0DDFB00F072
:1018D000EF0140F6B80000F0C7FB042140F6B90064
:1018E00000F0C2FB40F69B0000F0CEFB00F0E301ED
:1018F00041F0080140F69B0000F0B6FB40F2D160D9
:1019000000F0C2FB40F01801C9B240F2D16000F013
:10191000ABFB40F2AC6000F0B7FB00F08F0141F090
:10192000500140F2AC6000F09FFB4FF4FA5202FB12
:1019300008F2B2FBF4F2CBF8082007B0BDE8F08F54
:10194000002000F04DFD36498BF83850E2B2C95DF9
:101950008BF85020002F4DD10B3C012C8CBF002464
:101960000124053A012A02D80C2E38BF0C26029B0E
:101970009AF800208BF852308BF85340019B8BF87B
:101980001F2001249DF860208BF821208BF8511036
:101990008BF820308BF80E40ABF81C608BF81E9053
:1019A000FFF798FA2046FFF7B5FB1E4800F0B8FE97
:1019B0001D4800F021FF5FFA88F000F01DFD40F6A1
:1019C000A30000F061FB00EA040140F6A30000F070
:1019D0004BFB9BF82120A24240F2367013D100F05D
:1019E00053FB00F0FB0140F2367000F03DFB4FF678
:1019F000FF72A0E7012F04D1A4F10C035C425C410B
:101A0000AFE70024ADE700F03FFB40F00401C9B2AE
:101A1000E9E700BF78240020B0080020B8390108A9
:101A200000430108B024002086240020F0B58BB0CC
:101A30000D46044617461E46FFF74CFA0020FFF7F6
:101A400069FB204600F0BEFD00240123CDE90843D8
:101A500003234FF4167229462046CDE90644CDE90A
:101A60000444CDE90244CDE900532346FFF774FE58
:101A70002046FFF787FAFFF73FFAF1F709F801F080
:101A800041FC0446204601F047FCB04205D3012446
:101A9000FFF720FA20460BB0F0BD00F02FFF874281
:101AA000F0DA0024F4E70000F7B500230C4640F21A
:101AB00001211A460646084600F01EFD644B654D9E
:101AC0004FF400529A6195F85600012100F09CFFF6
:101AD0002B78012B40F6890013D195F85130062B55
:101AE0000FD100F0D1FA00F0FB0140F6890000F0C0
:101AF000BBFA2B78042B6CD8DFE803F0524B527FF3
:101B0000090000F0C1FA40F00401C9B2EDE7524A01
:101B1000731E1046C6F101074FF0000CF9188C42F5
:101B20006FDC0022E7001346BA4271D19A0142EA03
:101B3000C3125B0183F020031343661C0355F6B206
:101B400002234648AB73AE7600F056FE0021F1202A
:101B500000F08AFA0021F02000F086FAAB6C642BCA
:101B600070D17021F32000F07FFA1D21F22000F0E7
:101B70007BFAE1008C1CF420090A00F075FA04F0ED
:101B8000FE01F52000F070FA33486FF07F423146D5
:101B90001DE0EC77314800F02FFE0022214615E0D1
:101BA00001F008F80128074625D121460DF107026A
:101BB000304601F004F80446A0B99DF807302748E4
:101BC000AB7500F019FE9DF807102246304600F074
:101BD00065FB6968224801F061FC214801F024FCA2
:101BE000002006E01F4B3A460021022001F0A2F837
:101BF000032003B0F0BDAC75CCE70223AB73AC7629
